:100000000C94C2040C9408050C9408050C94080583
:100010000C9408050C9408050C9408050C9408052C
:100020000C9408050C94A9180C9408050C94080568
:100030000C94782E0C9408050C9408050C94080573
:100040000C9408050C9408050C94CC140C94080529
:100050000C94620B0C9408050C942C0B0C94080562
:100060000C94791A0C9408050C9492290C940805A8
:100070000C944A6E0C9408050C94A9689E1AA31A55
:10008000A81AB11AC81ADF1AEF1AFF1A431B1E1D4D
:10009000DF1A191C2A1C3E1C5C1C791CC41C101D78
:1000A000111FF01F6320DC201421B72140229D2264
:1000B00018234923BF23ED231A24895DD45E595F99
:1000C0000D60AD5FDD5FC85D985E0D602D5E0A0D51
:1000D0003D3D3D3D3D3D3D3D3D3D3D3D3D3D3D3D50
:1000E0003D3D3D3D3D3D3D3D3D3D3D3D3D3D3D3D40
:1000F0003D3D3D000A0D426174743A0020256420A4
:1001000043656C6C732000204C6F77207761726EB2
:10011000696E673A2025642E2564560020204175BB
:10012000746F2D43483A2025642E25645600202004
:100130004175746F6C616E64696E673A2025642E38
:10014000256456000A0D4F6C6420464320486172B6
:100150006477617265206E6F7420737570706F7252
:100160007465642062792074686973204669726DD1
:100170007761726521000A0D466F756E6420424CEE
:100180002D4374726C3A20002564000A0D0A0D217B
:1001900021204D495353494E4720424C2D43545240
:1001A0004C3A202564202121000A0D43616C6962CC
:1001B000726174696E672070726573737572652001
:1001C00073656E736F722E2E004F4B0A0D000A0D71
:1001D000466C696768742D74696D65202575206D9E
:1001E000696E20546F74616C3A2575206D696E00DC
:1001F000416E676C654E69636B20202020202020B3
:10020000416E676C65526F6C6C202020202020208E
:100210004163634E69636B20202020202020202032
:10022000416363526F6C6C2020202020202020200E
:100230005961774779726F202020202020202020CC
:10024000416C746974756465205B302E316D5D207E
:100250004163635A202020202020202020202020BD
:1002600047617320202020202020202020202020D3
:10027000436F6D706173732056616C75652020202B
:10028000566F6C74616765205B302E31565D20209F
:100290005265636569766572204C6576656C2020D1
:1002A0004779726F20436F6D706173732020202037
:1002B0004D6F746F722031202020202020202020BC
:1002C0004D6F746F722032202020202020202020AB
:1002D0004D6F746F7220332020202020202020209A
:1002E0004D6F746F72203420202020202020202089
:1002F00031362020202020202020202020202020D7
:1003000031372020202020202020202020202020C5
:1003100031382020202020202020202020202020B4
:1003200031392020202020202020202020202020A3
:10033000536572766F20202020202020202020204E
:10034000486F76657267617320202020202020206E
:1003500043757272656E74205B302E31415D2020D2
:100360004361706163697479205B6D41685D202031
:1003700048656967687420536574706F696E74208E
:100380003235202020202020202020202020202046
:100390003236202020202020202020202020202035
:1003A0003237202020202020202020202020202024
:1003B0004932432D4572726F722020202020202068
:1003C000424C204C696D6974202020202020202080
:1003D0004750535F4E69636B20202020202020204F
:1003E0004750535F526F6C6C20202020202020202B
:1003F00021212120494E434F4D50415449424C4503
:1004000020212121002E005B25695D005B25695DAF
:10041000002B204D696B726F4B6F70746572202BCF
:100420000048573A5625642E25642053573A2564D0
:100430002E25303264256320005365743A256420EC
:10044000257300424F4154004D6978657220457212
:10045000726F722100486172647761726520457223
:10046000726F7220313A2564202121004D69737327
:10047000696E6720424C2D4374726C3A25642021CA
:10048000210021204E432D4552523A20253264202E
:10049000212000493243204552524F522121210050
:1004A000424C2D53656C6674657374204572723AC4
:1004B000253264004865696768743A2020253569EB
:1004C00000536574706F696E743A25356900507217
:1004D0006573737572653A253569004F6666736595
:1004E000743A2020253569006163742E20626561AD
:1004F00072696E67004E69636B3A202020202020CD
:1005000025356900526F6C6C3A2020202020202570
:10051000356900436F6D706173733A202020253573
:1005200069004B25693A25346920204B25693A2515
:10053000346920004E693A2534692020526F3A25EB
:100540003469200047733A253469202047693A25E9
:100550003469200050313A253469202050323A2540
:100560003469200050333A253469202050343A252C
:10057000346920004779726F202D2053656E736FA8
:1005800072004E69636B202534692028253469295F
:1005900000526F6C6C2025346920282534692900AD
:1005A00059617720202534692028253469290041A4
:1005B0004343202D2053656E736F72004E69636B49
:1005C0002025346920282533692900526F6C6C205E
:1005D000253469202825336929005A202020202528
:1005E000346920282533692900566F6C746167656A
:1005F0003A2020202533692E253169560043757233
:1006000072656E743A2020202533692E25316941A8
:1006100000506F7765723A202020202025346957DA
:10062000004469736368617267653A202535696DB6
:1006300041680052656365697665720052432D51C9
:1006400075616C6974793A202534690052432D43F1
:1006500068616E6E656C733A25346900556E646529
:1006600072766F6C74616765732020005761726EDB
:100670003A202532642E25645600486F6D653A2075
:100680002532642E256456004C616E643A20253272
:10069000642E25645600506F746925693A20202520
:1006A000336900506F746925693A20202533690049
:1006B000466C696768742D54696D65202000546F1D
:1006C00074616C3A2535756D696E004163743A202A
:1006D000202535756D696E00287265736574290073
:1006E0000A0D47656E65726174696E6720646566A0
:1006F00061756C7420506172616D65746572205310
:100700006574202564000A0D5573696E6720506179
:1007100072616D6574657220536574202564000AEA
:100720000D47656E65726174696E67206465666108
:10073000756C74204D69786572205461626C650037
:100740000A0D4D697865722D436F6E6669673A20B0
:100750002725732720282575204D6F746F72732904
:10076000000A0D414343206E6F742063616C69621F
:100770007261746564210D0A000A0D4779726F2059
:1007800063616C6962726174696F6E206461746127
:10079000206E6F742076616C69640D0A0000008F12
:1007A000001E01AD013B02CA025803E603740402B5
:1007B000058F051B06A7063307BE074808D2085B4E
:1007C00009E3096B0AF20A780BFD0B810C040D8614
:1007D0000D070E870E060F840F00107B10F5106EAC
:1007E00011E5115B12CF124213B31323149214FEBE
:1007F000146A15D3153B16A11605176717C81727D6
:10080000188318DE1837198E19E319361A871AD685
:100810001A231B6E1BB61BFD1B411C831CC31C0033
:100820001D3C1D751DAB1DE01D121E421E6F1E9A44
:100830001EC31EE91E0D1F2E1F4D1F691F841F9B07
:100840001FB01FC31FD31FE11FEC1FF51FFB1FFFAE
:100850001F00200A0D7777772E4D696B726F4B6FF3
:10086000707465722E646520286329204869537965
:100870007374656D7320476D6248000A0D74686576
:1008800020757365206F66207468697320736F66C6
:100890007477617265206973206F6E6C7920706562
:1008A000726D6974746564200A0D6F6E206F7269D1
:1008B00067696E616C204D696B726F4B6F70746508
:1008C000722D4861726477617265005573657200BC
:1008D000486F5454205634004143542044534C0034
:1008E0004A657469005370656B7472756D00505081
:1008F0004D000A0D52656365697665723A20007590
:100900006E6B6E6F776E2E205573696E6720505038
:100910004D2E2E2E006E6F7420737570706F727472
:100920006564206279206861726477617265210074
:100930000A0D202D204C4942204E4F5420434F4D4C
:1009400050415449424C452021212121000A0D46A5
:100950006C69676874436F6E74726F6C0A0D4861DE
:100960007264776172653A25642E25640A0D536FAF
:100970006674776172653A5625642E253032642597
:100980006320000011241FBECFEFD0E1DEBFCDBF3A
:1009900011E0A0E0B1E0EEE2F2EE02C005900D92AF
:1009A000A03BB107D9F719E0A0EBB1E001C01D925F
:1009B000A63AB107E1F74AEAE2E0F0E081E280938B
:1009C0005700549120EF37EFA6E7B3E09FE0F9011D
:1009D0002F5F3F4F84918D93915097FFF8CF5739F8
:1009E00011F40000FECFE6E7F3E09EE08191482796
:1009F0004095915097FFFACF80918503481721F0D9
:100A0000573911F40000FECF0E943D060C94167178
:100A10000C9400008EEC90E09F938F938EED91E10B
:100A20009F938F93E0918903F0918A0309950F902A
:100A30000F900F900F90089580912E06E82FFF27BA
:100A4000EE0FFF1FE350F84F808191818D5E9F4F25
:100A500014F010920401808191818A5B9F4FCCF445
:100A6000809104018823A9F481E08093040180919E
:100A7000BD038F5F8093BD03853038F088EE93E02F
:100A80009093E8018093E701089566E970E00E9481
:100A90007C300895CF93DF93C82F882311F184EF22
:100AA00090E09F938F938EED91E19F938F93E091D0
:100AB0008903F0918A030995809123019091240183
:100AC0006BE270E00E948970CB018F5F8093000120
:100AD0000F900F900F900F90873018F086E0809362
:100AE000000180915106823328F590910001989F72
:100AF000802D112480930201CC23F1F068EC70E08A
:100B0000892F0E947C308091000199279F938F93B9
:100B10008CEF90E09F938F938EED91E19F938F9355
:100B2000E0918903F0918A0309958DB79EB70696E7
:100B30008DBF02C0809302019091A106923340F4D0
:100B400080910001899F802D11248093B90102C0FA
:100B50009093B9013091A206323340F480910001A4
:100B6000839F802D11248093B80102C03093B80177
:100B70008091B90190910201981720F491509093BF
:100B8000B9019F5F8091B801891720F0915090932F
:100B9000B8019F5F8091B9012091B801821728F0B8
:100BA000332319F021502093B901CC2309F462C0FA
:100BB000892F6AE00E946970892F99279F938F93EC
:100BC000809102010E94697099279F938F9387E01B
:100BD00091E09F938F93CEEDD1E1DF93CF93E0919E
:100BE0008903F0918A0309958DB79EB708968DBF4A
:100BF0008091B8018823E9F06AE00E946970892F2A
:100C000099279F938F938091B8010E9469709927CB
:100C10009F938F938CE191E09F938F93DF93CF937A
:100C2000E0918903F0918A0309958DB79EB70896E4
:100C30008DBF8091B9018823E9F06AE00E94697054
:100C4000892F99279F938F938091B9010E94697092
:100C500099279F938F938EE291E09F938F93DF93D9
:100C6000CF93E0918903F0918A0309958DB79EB7E0
:100C700008968DBFDF91CF910895CFEFD0E1DEBF11
:100C8000CDBF88249924C1E07C2E14B815B88AE021
:100C90008AB98FE58BB9B7EECB2EB3E0DB2E2EEC05
:100CA0003FEFC20ED31ED7FEFACF189B06C0199B8A
:100CB00002C08DE005C08BE003C0199B04C084E135
:100CC0008093030107C08AE0809303018EE38AB911
:100CD00087E48BB981E887B93E9A8FEF88B98BE1B9
:100CE00084B981E085B9469A84B7877F84BF8091B3
:100CF00060008861809360001092600084EC99E04D
:100D00009093E8018093E7011092A1021092A00253
:100D100010920208109201081092A3021092A202EF
:100D20001092A5021092A40220910301243128F010
:100D300084EC94E0A0E0B0E004C08BE095E0A0E09B
:100D4000B0E08093410190934201A0934301B0939E
:100D500044012898293111F4299A01C029980E9448
:100D60001D160E94EE150E94E6110E943F2E0E9461
:100D7000D91981E00E943F290E942D5C0E942A66B9
:100D800087E00E94F36C80910301893111F4299A64
:100D900001C0299878940E946028809103018431D1
:100DA000E8F488E190E02CE00FB6F894A8958093E1
:100DB00060000FBE2093600084E491E09F938F93C6
:100DC0008EED91E19F938F93E0918903F0918A03D7
:100DD00009950F900F900F900F90EECF80913A02EF
:100DE000826080933A0210923D02C0E0D0E00E94FF
:100DF0005E3B85E090E00E94B4156C0180913A0260
:100E000080FD05C0C6010E94BD158823B9F3219657
:100E100031E0C43FD30758F386E791E09F938F9367
:100E2000AEEDAA2EA1E1BA2EBF92AF92E091890356
:100E3000F0918A030995C0E0D0E00F900F900F90D9
:100E40000F9008E417E0F3ECEF2EF6E0FF2EF70129
:100E5000808124E030E0E20EF31E1816ACF40BC0E3
:100E60000E945E3B80913A0280FD05C0C6010E944F
:100E7000BD158823B9F3C6010E94BD15882321F44E
:100E8000F8018381882364F7F801838187FF2CC0F0
:100E9000CE0101966AE070E00E9475709F938F9377
:100EA00088E891E09F938F93BF92AF92E09189037E
:100EB000F0918A0309958091B1018F5F8093B10110
:100EC000F801948584E6989FC00111242585280F98
:100ED0008DB79EB706968DBF222331F08091A50372
:100EE000281710F42093A5032196015F1F4FCC30E3
:100EF000D10508F4ACCFC0E0D0E008E417E0E3ECA3
:100F0000EE2EE6E0FE2EF801838187FD1DC0F7017D
:100F100080811816CCF42196DF93CF9321978BE82C
:100F200091E09F938F938EED91E19F938F93E0914A
:100F30008903F0918A03099582E08093E5012DB73A
:100F40003EB72A5F3F4F2DBFF801838180788383AE
:100F5000219624E030E0E20EF31E015F1F4FCC30FB
:100F6000D10588F20E940A0590912C068091B1016A
:100F7000981728F48091A30380618093A30399308C
:100F800020F088E080933B0102C090933B0189EA06
:100F900091E09F938F93CEEDD1E1DF93CF93E091DA
:100FA0008903F0918A03099588EE93E00E94B415B5
:100FB0006C010E94171A0F900F900F900F90C601AE
:100FC0000E94BD158823D9F389EC91E09F938F93FC
:100FD000DF93CF93E0918903F0918A03099580E034
:100FE0000E943131289880ED97E09093E80180933A
:100FF000E70185E58093BF038EE090E00E948426A0
:101000009927182F00278FE090E00E948426080F70
:10101000111D1093B7010093B6018AE090E00E9481
:1010200084269927182F00278BE090E00E948426C1
:10103000080F111D1093B5010093B4010F900F908C
:101040000F900F900F5F1F4F39F08091B601909174
:10105000B7018F5F9F4F41F41092B7011092B60114
:101060001092B5011092B4018091B4019091B50134
:101070009F938F938091B6019091B7019F938F9327
:101080008EEC91E09F938F93DF93CF93E091890350
:10109000F0918A0309950E948B1E88E893E1909352
:1010A0003A0180933901C1E0C093BE038C2F0E94A6
:1010B0004A05809154060E94466C0E940A0580ED04
:1010C00097E00E94B4156C018AEF90E00E94B4157D
:1010D00093E0909386051092B0018091A7062DB7FA
:1010E0003EB7285F3F4F2DBF84FF02C0C093BA01B7
:1010F00090933C0112BC11BC8091BC01882311F07B
:101100004798FECF8091EB01882309F494C2809127
:101110001501882309F48FC2F8948091EB01815066
:101120008093EB0178948091BD03882319F00E948D
:101130001C0502C00E940B3F0E945E3B28988091D4
:101140009402882331F0809194028150809394021C
:1011500042C080916F00806280936F001092FE0702
:101160001092FD078091A30388608093A303809170
:101170002E06A82FBB27AA0FBB1FFD01ED5BF74F63
:101180001182108280912F06E82FFF27EE0FFF1F9C
:10119000CF018D5B974FEC0119821882A350B84F95
:1011A00011961C921E92E350F84F1182108280918A
:1011B0003106E82FFF27EE0FFF1FE350F84F118293
:1011C000108280913006E82FFF27EE0FFF1FE350BB
:1011D000F84F118210828091390190913A01019764
:1011E00090933A01809339018091390190913A01AD
:1011F000892B21F080913B028823C9F1809139012C
:1012000090913A01892BD9F40E94702985E090E0F1
:1012100090933A01809339018091C0059091C10566
:1012200001969093C1058093C0058091A3038160CE
:101230008093A303809187058260809387058091C6
:101240000B0190910C018F5F9F4F91F4809193025D
:10125000882371F088EA91E69093E8018093E70192
:1012600080E890E090930C0180930B0101C02898D6
:101270000E94C26D8091EB01882309F0DAC1809150
:10128000E601882311F40E944E5C809111018823AD
:1012900011F00E9477160E9431120E94B70DC6010C
:1012A0000E94BD15882309F4C0C124E130E0C20EBC
:1012B000D31E0E94351680913B02882329F4809129
:1012C00078098E3150F405C08091A3038260809329
:1012D000A3038091870582600FC08091E701909100
:1012E000E801892B59F48091390190913A010797CF
:1012F00028F0809187058D7F809387058091BA01C2
:10130000882361F080919402873940F01092BA01ED
:1013100088E893E19093E8018093E70180910601CA
:10132000882321F08150809306012EC08093C90349
:101330001092670210926602109265021092640287
:101340001092630210926202809194028823E1F469
:1013500080910B0190910C018F5F9F4FA9F4209118
:10136000BA01223089F088E99AE39093E8018093EA
:10137000E70180E09CE090930C0180930B01222315
:1013800019F082E08093BA018091A001893C70F04D
:1013900081508093A0018091A3038B7F8093A3034E
:1013A0008091A60381608093A60351C08091FA08C2
:1013B0008823F9F08091A30384608093A30389E0DC
:1013C0008093420380910B0190910C018F5F9F4F9E
:1013D00081F480919302882361F088E99AE39093E5
:1013E000E8018093E70180E098EA90930C018093F4
:1013F0000B011092350310923403109233031092B4
:101400003203109231031092ED088FEF809362093E
:1014100010922C0910922B0910922E0910922D096E
:101420008FEF9FEF90932A098093290910928302EE
:101430001092840210928502109286021092870206
:101440008091A6038E7F8093A6031092A0016091E5
:101450000201262F33278091230190912401281720
:101460003907F4F080915B02806280935B02809187
:101470000B0190910C018F5F9F4F91F4809123019C
:10148000909124010B9764F080E797E19093E80135
:101490008093E70180E093E090930C0180930B012F
:1014A0008091BB018F5F8093BB01813309F074C0D1
:1014B0001092BB0180915B0281FF0AC08091B20152
:1014C0009091B30101969093B3018093B20104C04F
:1014D0005AEA852E55E0952E80915C0290915D022E
:1014E0008050944008F049C02091CF053091D0053C
:1014F0004091D1055091D20580911B0190911C0122
:10150000A0911D01B0911E01281739074A075B07FA
:1015100064F48091CF059091D005A091D105B09150
:10152000D2050596A11DB11D20C02091CF05309197
:10153000D0054091D1055091D20580911B01909129
:101540001C01A0911D01B0911E0182179307A407F1
:10155000B5079CF48091CF059091D005A091D1055D
:10156000B091D2050597A109B1098093CF05909359
:10157000D005A093D105B093D205862F9927019667
:101580002091230130912401821793072CF480913C
:101590005B028F7D80935B020894811C911C22E783
:1015A00082162BE0920609F040C0882499242091ED
:1015B000B6013091B7012F5F3F4F3093B7012093B1
:1015C000B6018091B4019091B50101969093B50157
:1015D0008093B401832F9927682F8EE090E00E94BA
:1015E0008C268091B6019091B7019070682F8FE0A2
:1015F00090E00E948C268091B4019091B501892FD2
:101600009927682F8AE090E00E948C268091B4018F
:101610009091B5019070682F8BE090E00E948C262D
:1016200084E190E00E94B4156C010E94BA610E94AE
:10163000646671107A94772039F40E947E61882361
:1016400019F08CE0782E56CD8091E601882309F0C0
:1016500051CD0E944E5C4ECD1F920F920FB60F924D
:1016600011248F939F93EF93FF9380910801882318
:10167000E1F48091D6019091D70101969093D70122
:101680008093D601FC01E655FB4FE081ED3019F067
:101690008C3D910539F41092D7011092D60181E06A
:1016A00080930801E093C60004C01092D701109205
:1016B000D601FF91EF919F918F910F900FBE0F90E8
:1016C0001F9018951F920F920FB60F9211242F930F
:1016D0003F934F935F936F937F938F939F93AF93BA
:1016E000BF93CF93EF93FF9390E08091BC01813043
:1016F00029F48091C6008093CE00D1C08091BC01B6
:10170000823029F48091C6008093CC03C8C08091B8
:10171000C6008093CE015091DC015C3D10F09093A7
:10172000DD018091CE018D3009F06AC08091DD012C
:10173000823009F065C09093DD01852F992784538D
:101740009C4FFC01329740812091D8013091D90102
:10175000241B3109DC0111978C91281B3109C90127
:101760009F709093D9018093D80146E09695879514
:101770004A95E1F7982F935C9093DA012F733070BC
:10178000235C2093DB018081981729F48C91281722
:1017900011F491E006C090E08091CB018F5F8093BF
:1017A000CB018091CD01882309F079C0992309F4F8
:1017B00076C081E08093CD01580F5093CA015150FB
:1017C000E52FFF27E453FC4F8DE080838091CE030B
:1017D000823509F064C0C0919302CC2309F05FC048
:1017E0000E948B1E88E190E02CE00FB6F894A8953B
:1017F000809360000FBE20936000C093E5014FC04E
:101800002091DD01822F992781309105F9F08230F6
:1018100091051CF4892B21F040C0029711F13DC0C5
:101820008091CE01833239F48091CD01882319F45F
:1018300081E08093DD018091CE018093CC0381E033
:101840008093DC018091CE01992722C02F5F2093E5
:10185000DD01E52FFF27E453FC4F8091CE0180830B
:1018600009C0E52FFF27E453FC4F8091CE01808310
:101870005C3D20F45F5F5093DC0102C01092DD01FB
:101880002091CE018091D8019091D901820F911DB4
:101890009093D9018093D80102C01092DD01FF918D
:1018A000EF91CF91BF91AF919F918F917F916F9168
:1018B0005F914F913F912F910F900FBE0F901F900E
:1018C0001895AC01A0E0B0E09D01A817B90748F455
:1018D000EAEAF4E08191280F311D1196A417B507AB
:1018E000C8F33F70FD01E655FB4FC90156E09695E0
:1018F00087955A95E1F7835C80831196FD01E65543
:10190000FB4F2F733070822F835C8083A555BB4FB4
:101910008DE08C93109208018091AA048093C600F8
:101920000895A0E0B0E0E7E9FCE00C94E2702C85BB
:101930009D850E85BB2483E28093AA049F599093D2
:10194000AB042093AC0433E0E32EF12C002309F424
:101950009EC0CF84D888BE016D5E7F4FA989BA89A9
:101960000150109709F493C01097B9F0F601EB0DF0
:10197000F11DB3949081119791F4002349F1FB017B
:101980006E5F7F4FDB01C080D1806E5F7F4F0D9017
:10199000BC91A02DBB24015002C090E019C010974B
:1019A000B9F0F601EB0DF11DB3944081119791F45C
:1019B000002341F1FB016E5F7F4FDB01C080D180CE
:1019C0006E5F7F4F0D90BC91A02DBB24015002C0D3
:1019D00040E018C01097B1F0F601EB0DF11DB39483
:1019E0001081119781F4002371F0FB013296DB0125
:1019F000CD90DC90BF016E5F7F4FA081B181BB2491
:101A0000015001C010E0F701E655FB4F892F869584
:101A10008695835C80830894E11CF11CF701E655F0
:101A2000FB4F892F99278370907024E0880F991FAE
:101A30002A95E1F755279A0194E0369527959A95CE
:101A4000E1F7822B835C80830894E11CF11CF70191
:101A5000E655FB4F4F705070440F551F440F551FF4
:101A6000812F992726E0969587952A95E1F7842B73
:101A7000835C80830894E11CF11CF701E655FB4F61
:101A80001F73135C10830894E11CF11C6ACFC7011B
:101A90000E94610CE9E00C94FE70A3E07A2F409163
:101AA000CA014650442309F458C0E72FFF27E453E6
:101AB000FC4F80818D537F5FE72FFF27E453FC4F5E
:101AC00020812D537F5FE72FFF27E453FC4F3081A8
:101AD0003D537F5FE72FFF27E453FC4F60816D5339
:101AE0007F5F9927880F991F880F991F522F529552
:101AF0005F70582B822F99278F709070F4E0880FB9
:101B0000991FFA95E1F7232F26952695282B832FE9
:101B1000992783709070E6E0880F991FEA95E1F7A6
:101B2000682B41504F3FC9F0EA2FFF27E453FC4F89
:101B30005083AF5F41504F3F81F0EA2FFF27E453BE
:101B4000FC4F2083AF5F41504F3F39F0EA2FFF2712
:101B5000E453FC4F6083AF5FA5CF8FEC93E090938D
:101B6000C9018093C801A350A093C7010895A2E0C2
:101B7000B0E0EDEBFDE00C94E8708091CD0188239E
:101B800009F418C40E944D0D8091CD03823609F0EE
:101B9000E4C28091CE0399278037910509F4AFC044
:101BA00081379105C4F48A36910509F441C28B3618
:101BB000910544F48B34910571F18636910509F451
:101BC0006AC1CBC28D36910509F469C08E36910584
:101BD00009F44DC0C2C28437910541F185379105A2
:101BE0004CF48137910509F491C08337910509F4CC
:101BF000EAC0B3C28737910509F4DCC18837910583
:101C00002CF48537910509F498C1A7C2893791054D
:101C100009F47DC1A2C2E091C801F091C90180819F
:101C200091819093900180938F0197C28091CA0116
:101C3000A091C801B091C901853140F080E1E7EA87
:101C4000F3E00D9001928A95E1F70DC08D919D9181
:101C50000D90BC91A02D8093A7039093A803A0930F
:101C6000A903B093AA0380EF8093C5014BC0809174
:101C700008018823E1F38DE490E09F938F9386EB36
:101C800096E09F938F9381E08F938F938EE48F9351
:101C90000E94910C8DB79EB707968DBF5EC2A09132
:101CA000C801B091C9011C91113081F48DE4E6EBBB
:101CB000F6E00D9001928A95E1F70E949B27198327
:101CC0008091A3038F7E8093A30301C0198280912A
:101CD00008018823E1F381E090E09F938F93CE0188
:101CE00001969F938F9381E08F938F938DE48F93D1
:101CF0000E94910CADB7BEB71796ADBF2EC281E062
:101D00008093D0018FEF8093060127C280919302C8
:101D10008823E1F5E091C801F091C901E0818E2F9F
:101D20008A508A3058F48983882311F481E003C0F3
:101D3000863010F085E0898361E00EC08E2F8451DB
:101D40008A3070F48983882311F481E003C08630DF
:101D500010F085E0898360E089810E941D2812C00F
:101D6000E983EF3F19F40E94FE2789838981882344
:101D700011F481E003C0863010F085E08983898109
:101D80000E94A22680E00E944A0503C00E94FE270E
:101D90008983809108018823E1F388E890E09F938C
:101DA0008F938DE296E09F938F9381E090E09F93D5
:101DB0008F93CE0101969F938F9382E08F9381E062
:101DC0008F9381E52DC12091C8013091C901D901BE
:101DD0008C918150853008F045C0F90181818736AA
:101DE00009F040C0809193028823E1F52F5F3F4FB7
:101DF00088E8EDE2F6E0D9010D9001928A95E1F7CD
:101E0000F90182910E940D2780916E069927AA27D9
:101E1000BB27BC01CD0124EC39E040E050E00E943A
:101E20004A70DC01CB018093870190938801A093D5
:101E30008901B0938A0180916F069927AA27BB2751
:101E4000BC01CD010E944A70DC01CB01809383016B
:101E500090938401A0938501B09386010E94FE2790
:101E6000898301C01982809108018823E1F381E010
:101E700090E09F938F93CE0101969F938F9381E083
:101E80008F938F9383E58F930E94910C8DB79EB7AC
:101E900007968DBF2BC080919302882309F05DC106
:101EA000E091C801F091C901E0818E2F8150853009
:101EB00018F48E2F0E94A2260E94FE27898380910B
:101EC00008018823E1F381E090E09F938F93CE0196
:101ED00001969F938F9381E08F938F9386E48F93E6
:101EE0000E94910CADB7BEB71796ADBF109193028B
:101EF000112341F46EE670E089810E947C30812FCD
:101F00000E944A05809154060E94466C26C119829F
:101F10002981A091C801B091C901EDEFF7E08D9141
:101F2000992787FD909593A382A3822F8F5F898342
:101F3000282F32968C3098F310C1E091C801F091AF
:101F4000C90180810E94AF2D8A83882319F481E022
:101F5000898301C01982809108018823E1F388E018
:101F600090E09F938F9380E497E09F938F9321E07D
:101F700030E03F932F938091C8019091C9019F93C6
:101F80008F933F932F93CE0102969F938F933F930E
:101F90002F93CE01820F931F9F938F9384E08F9393
:101FA00081E08F9385E58F930E94910CEDB7FEB78A
:101FB00073963CC08091C701893008F4CEC020914F
:101FC000C8013091C9012F5F3F4F88E0A0E4B7E01E
:101FD000F90101900D928A95E1F7D9018E910E9445
:101FE000092D8A83882319F481E0898301C019822D
:101FF000809108018823E1F321E030E03F932F93A3
:10200000CE0102969F938F933F932F93CE01820F21
:10201000931F9F938F9382E08F9381E08F9387E547
:102020008F930E94910CEDB7FEB73B96EDBF95C024
:1020300080919302882309F090C00E94FD6B8983F0
:10204000823019F0843009F088C020E430E0F89440
:102050008091C1008F738093C1008091C9008F73FC
:102060008093C9008091C100877E8093C1008091D8
:10207000C900877E8093C9008091C80087FF03C094
:102080008091CE00F9CF8091C00087FF03C080917E
:10209000C600F9CFE091C801F091C901E081E130BB
:1020A00021F482E08093BC012EC0E43611F421E8D3
:1020B00030E081E08093BC01832F99278093CD008D
:1020C0002093CC008091CD008093C5008091CC00FE
:1020D0008093C4008091CA008F7D8093CA00809154
:1020E000CA008F7E8093CA008091C9008B7F809345
:1020F000C9008091CA0084608093CA008091CA00A0
:1021000082608093CA008091CA00877F8093CA0052
:102110008091C200877F8093C2008091C9008E7F2A
:102120008093C9008091C10088618093C100809133
:10213000C90088618093C9008091C1008068809344
:10214000C1008091C90080688093C90010926E0020
:1021500010926F001092700078948091CE039927AE
:102160008436910509F4BBC085369105ACF48136FF
:10217000910509F46FC0823691052CF48B349105DA
:1021800009F45DC00FC18236910509F470C0833631
:10219000910509F47FC006C18C36910509F4EDC0A4
:1021A0008D3691054CF48736910509F4F8C08836D0
:1021B000910509F4B2C0F6C08437910529F086373D
:1021C000910509F4E8C0EEC08091CA01A091C80150
:1021D000B091C901803140F080E1E7EAF3E00D9071
:1021E00001928A95E1F70DC08D919D910D90BC9162
:1021F000A02D8093A7039093A803A093A903B09365
:10220000AA03809108018823E1F31F9280910501C0
:102210008F9384E58F930E94910C8AEF8093C50180
:102220008FEF8093060180EA9FE00E94B41590939F
:10223000BE018093BD010F900F900F90B3C0E0914D
:10224000C801F091C90180819181909390018093A0
:102250008F01A8C0E091C801F091C90180818093ED
:102260000701803298F08FE1809307010FC0A091A1
:10227000C801B091C9018BE0EFEBF3E00D90019242
:102280008A95E1F78091C8038093C8058FEF80930A
:10229000060188C08091C1019091C201892B89F407
:1022A000E091C801F091C901E081EE2351F08AE08C
:1022B000E89FC00111240E94B41590939A03809363
:1022C0009903E091C801F091C90190818AE0989F3B
:1022D000C00111249093C2018093C10115C08FEFFA
:1022E00080930601E091C801F091C90190818AE0D4
:1022F000989FC00111249093C4018093C301892B3E
:1023000019F081E08093D20180EA9FE00E94B41529
:102310009093BE018093BD0145C08FEF809306016D
:10232000E091C801F091C901908197FD08C082E059
:102330008093CF011092C0011092BF011AC09095F6
:1023400080913302892B8093330291818AE0989F98
:10235000C00111249093C0018093BF0184E0809359
:10236000CF0180EA9FE00E94B4159093BE01809354
:10237000BD0181E08093D30115C08FEF80930601EA
:10238000E091C801F091C90180818093340281E01D
:102390008093D40107C081E08093D10103C081E024
:1023A0008093D5011092CD011092C9011092C801FD
:1023B0001092C701E3E0CE5F0C940471982F8091D6
:1023C000C00085FFFCCF9093C60008950F931F9324
:1023D00088E18093C1008091C00082608093C0003A
:1023E0008091C10080688093C1008091C1008064A9
:1023F0008093C10000E010E00093C5008AE290E005
:102400008093C4008091C3019091C4010E94B415CF
:1024100090939C0380939B038CED90E00E94B415F5
:102420009093CB038093CA0382E080939D0388E05E
:1024300080939E031092A1038BE080939F031092E0
:10244000A0038FEF8093A503809103018093A403E1
:102450001093C9010093C8011092C7011F910F91F9
:102460000895A0E1B0E0E7E3F2E10C94E770809119
:102470000801882309F48CC28091BD019091BE01AE
:102480000E94BD15882361F01092C0011092BF0117
:102490001092C4011092C3011092C2011092C101A6
:1024A0008091BF019091C001892B41F08091A804D7
:1024B0009091A9040E94BD15882329F48091D3012D
:1024C000882309F460C080910801882309F45BC067
:1024D0008091CF010CED15E08430A8F00E94A11E80
:1024E00080E590E09F938F931F930F9381E08F93EC
:1024F0008F9388E48F930E94910C2DB73EB7295F8C
:102500003F4F2DBF34C01092350280EF93E09F9370
:102510008F9384E99EE19F938F93E0918903F091DB
:102520008A03099584E190E09F938F931F930F9303
:1025300081E090E09F938F938FEC91E09F938F9336
:1025400082E08F9381E08F9388E48F930E94910CB7
:102550008091CF01982F8F5F8093CF012DB73EB729
:10256000215F3F4F2DBF943010F01092CF0180912A
:10257000BF019091C0010E94B4159093A90480936B
:10258000A8041092D3018091D401882351F1809145
:102590000801882331F10E94A11E80E590E09F93FD
:1025A0008F938CED95E09F938F9321E030E03F93E4
:1025B0002F9385E291E09F938F933F932F9384E332
:1025C00092E09F938F9383E08F9381E08F938CE4CD
:1025D0008F930E94910C1092D4018DB79EB70F96E5
:1025E0008DBF8091D1018823D1F08091080188238B
:1025F000B1F08AE090E09F938F938DE993E09F93F1
:102600008F9381E08F938F9386E58F930E94910C37
:102610001092D1012DB73EB7295F3F4F2DBF80915A
:10262000D5018823D9F0809108018823B9F08BE087
:1026300090E09F938F938FEB93E09F938F9381E034
:102640008F93809105018F9387E48F930E94910C63
:102650001092D5018DB79EB707968DBF8091C301AB
:102660009091C401892B41F080919B0390919C0330
:102670000E94BD15882321F48091D201882341F165
:1026800080910801882321F10E948E2F82E490E03E
:102690009F938F9386E895E09F938F9381E08F932C
:1026A0008F9384E48F930E94910C1092D2012DB7E6
:1026B0003EB7295F3F4F2DBF8091C3019091C40168
:1026C000009731F00E94B41590939C0380939B0374
:1026D0008091C1019091C201892B09F497C080912A
:1026E000990390919A030E94BD15882309F48EC026
:1026F00080910801882309F489C080910009909194
:10270000010990938C0380938B038091020990912F
:10271000030990938E0380938D032091E2083091FA
:10272000E3084091E4085091E508DA01C90163E04B
:10273000880F991FAA1FBB1F6A95D1F7820F931F9D
:10274000A41FB51F820F931FA41FB51F2091410125
:10275000309142014091430150914401BC01CD01AF
:102760000E94BE703093900320938F038091B60235
:102770009091B702A091B802B091B90249E0B59525
:10278000A795979587954A95D1F780939103809166
:10279000B2029091B302A091B402B091B50239E0B7
:1027A000B595A795979587953A95D1F7809392031C
:1027B0008091BE029091BF02A091C002B091C1026F
:1027C00029E0B595A795979587952A95D1F7809398
:1027D00093038EE090E09F938F938BE893E09F9319
:1027E0008F9381E08F938F9383E48F930E94910C5A
:1027F0008091C1019091C2010E94B41590939A03F7
:10280000809399038DB79EB707968DBF809107017E
:102810008F3F79F1992704E0880F991F0A95E1F716
:1028200080519E4F40E150E0BC01CE0101960E94D4
:102830009D6E80E190E09F938F93CE0101969F93D0
:102840008F9381E090E09F938F9387E091E09F9337
:102850008F9382E08F9381E08F9381E48F930E9426
:10286000910C8FEF809307012DB73EB7255F3F4F47
:102870002DBF8091C8058823C9F080910801882365
:10288000A9F081E090E09F938F9388EC95E09F936F
:102890008F9381E08F938F9382E48F930E94910CAA
:1028A0001092C8058DB79EB707968DBF8091D00155
:1028B0008823D1F0809108018823B1F086E490E06C
:1028C0009F938F938DEF97E09F938F9381E08F93EA
:1028D0008F9380E58F930E94910C1092D0012DB7B9
:1028E0003EB7295F3F4F2DBF8091CA039091CB0324
:1028F0000E94BD15882309F44BC0809108018823EC
:1029000009F446C08091A001882361F580910009F7
:10291000909101099093B8038093B70380910209C5
:10292000909103099093BA038093B9038091700248
:102930008093BB0380916F028093BC0388E090E09A
:102940009F938F9387EB93E09F938F9381E08F9377
:1029500083E08F938BE68F930E94910C8DB79EB787
:1029600007968DBF8091BD03853018F086E0809377
:10297000BD038091E401882319F083E690E002C052
:1029800087EE93E00E94B4159093CB038093CA0323
:10299000E4E0C05F0C9403711F920F920FB60F9288
:1029A00011242F933F935F936F937F938F939F9304
:1029B000AF93BF93EF93FF938091E601882329F0B3
:1029C0008091E60181508093E6018091590388232C
:1029D00019F08150809359038091EE0181508093CA
:1029E000EE018F3F09F051C089E08093EE018091A4
:1029F000EC019091ED0101969093ED018093EC0133
:102A0000809112018F5F817080931201882349F4B5
:102A10008091EB01843028F48091EB018F5F8093EB
:102A2000EB01349903C081E08093E4018091E701D8
:102A30009091E801892B11F18091E7019091E801D3
:102A40000B9750F08091E7019091E8010A979093DD
:102A5000E8018093E70104C01092E8011092E701B9
:102A60008091E7019091E80120910B0130910C01D8
:102A700082239323892B41F0479A07C08FEF9FEF62
:102A800090930C0180930B0147988091E401882377
:102A900009F45AC02091A001222309F055C0809169
:102AA000D00883FF51C086B19927FC01E071F07016
:102AB00084FF13C08091E9019091EA0101969093FF
:102AC000EA018093E9018091E9019091EA01895E30
:102AD0009340D0F12093E40137C08091E9019091B7
:102AE000EA01892B69F18091E9019091EA018A5606
:102AF000914030F58091E9019091EA0169E270E03E
:102B00000E9475708091E9019091EA01860F971FEC
:102B10009093EA018093E9018091E9019091EA01A3
:102B20000B9750F08091E9019091EA010A979093F8
:102B3000900180938F0104C0F0939001E0938F0186
:102B40001092EA011092E901FF91EF91BF91AF91CC
:102B50009F918F917F916F915F913F912F910F90F6
:102B60000FBE0F901F9018952091EC013091ED0150
:102B7000280F391FC901019608952091EC01309169
:102B8000ED01821B930B892F992786958074907095
:102B90000895CF93DF930E94B415EC01CE010E94FB
:102BA000BD158823D9F3DF91CF910895CF93DF939B
:102BB0000E94B415EC0109C080911501882329F009
:102BC000909315018FEC80937A00CE010E94BD1581
:102BD000982F882389F3DF91CF9108959FB7F894B8
:102BE0005F983E9A469A8091B0008F708093B000B3
:102BF0008091B00083608093B0008091B1008B73AE
:102C00008093B1008091B1008B608093B1001092ED
:102C1000B2008FEF8093B3008091B0008068809302
:102C2000B000809170008A7F809370008091700066
:102C30008260809370009FBF08958AE090E00E94B8
:102C4000B4159093CA058093C90582E085BD83EBD6
:102C500084BD8FEF88BD84EB87BD86E086BD809103
:102C60006E00816080936E0008958091A606209189
:102C70006E0182FF30C090915D068CE3989FB00199
:102C8000112490915C0680E5989FA0011124922F59
:102C9000905897FD9D5F9595959586E09802C001A7
:102CA00011242091090130910A01281B390B30931E
:102CB0000A0120930901421753072CF050930A018F
:102CC0004093090108952617370784F070930A018D
:102CD000609309010895822F992736E0880F991F84
:102CE0003A95E1F790930A01809309010895EF92D4
:102CF000FF920F931F93CF93DF9380916406E82F89
:102D0000FF27E95BFE4F9681C081809111018130E0
:102D100009F021C18091A80687FF05C0C0E0D0E07E
:102D2000E0E0F0E046C0892F992787FD9095A92F14
:102D3000B92F2091D2023091D3024091D402509108
:102D4000D502BC01CD010E944A7097FF04C06158B2
:102D50007F4F8F4F9F4F7B018C0187E01595079523
:102D6000F794E7948A95D1F78C2F992787FD909552
:102D7000A92FB92F2091CE023091CF024091D002DD
:102D80005091D102BC01CD010E944A7097FF04C04E
:102D900061587F4F8F4F9F4FB7E0959587957795F7
:102DA0006795BA95D1F7F801E701C61BD70BE80B79
:102DB000F90B20913C0330913D03C901A3E0880F3A
:102DC000991FAA95E1F7821B930BAA2797FDA0955F
:102DD000BA2FC81BD90BEA0BFB0B80916C0199270A
:102DE000AA27BB27BC01CD019E01AF010E944A70FA
:102DF00097FF04C061507E4F8F4F9F4FFC01EB0146
:102E000079E0F595E795D795C7957A95D1F7109123
:102E1000A6066091090170910A0112FF05C0709326
:102E2000100160930F0118C040910F0150911001E3
:102E300080916306282F3327CB01841B950BB901A2
:102E40000E94897080910F0190911001860F971F49
:102E50009093100180930F0110FF14C080910F0117
:102E60009091100197FD0F9664E0959587956A956E
:102E7000E1F7AA2797FDA095BA2FC80FD91FEA1F1F
:102E8000FB1F15C080910F019091100197FD0F96C7
:102E900054E0959587955A95E1F7AA2797FDA09557
:102EA000BA2F8C1B9D0BAE0BBF0BFD01EC012091CB
:102EB0009806222321F133278091E0019091E101CE
:102EC000829FA001839F500D929F500D1124CA0133
:102ED000AA2797FDA095BA2F8C0F9D1FAE1FBF1F6D
:102EE0002F5F3F4F442737FD4095542FBC01CD0144
:102EF0000E94BE703093E1012093E00104C0D093A2
:102F0000E101C093E00180915C06282F3327220F56
:102F1000331F220F331F8091E0019091E10182174E
:102F200093077CF080915D06282F3327220F331FF3
:102F3000220F331F8091E0019091E101281739079A
:102F400024F43093E1012093E001809111018F5F1F
:102F500080931101F9C0892F992787FD9095A92F9A
:102F6000B92F2091CE023091CF024091D0025091E2
:102F7000D102BC01CD010E944A7097FF04C0615884
:102F80007F4F8F4F9F4F7B018C0187E015950795F1
:102F9000F794E7948A95D1F78C2F992787FD909520
:102FA000A92FB92F2091D2023091D3024091D4029F
:102FB0005091D502BC01CD010E944A709B01AC0129
:102FC00097FF04C021583F4F4F4F5F4FC7E05595C3
:102FD000479537952795CA95D1F72E0D3F1D401F70
:102FE000511F80916B019927AA27BB27BC01CD01F6
:102FF0000E944A7097FF04C061507E4F8F4F9F4FD1
:10300000FC01EB01B9E0F595E795D795C795BA9521
:10301000D1F780916D019927A6E0880F991FAA9595
:10302000E1F740910D0150910E0120916306332785
:10303000841B950BB9010E94897080910D019091BC
:103040000E01860F971F90930E0180930D018091C2
:10305000A60681FF14C080910D0190910E0197FD8D
:103060000F9674E0959587957A95E1F7AA2797FDD5
:10307000A095BA2FC80FD91FEA1FFB1F15C080915A
:103080000D0190910E0197FD0F9664E0959587953F
:103090006A95E1F7AA2797FDA095BA2F8C1B9D0B87
:1030A000AE0BBF0BFD01EC0120919906222321F10B
:1030B00033278091DE019091DF01829FA001839FE1
:1030C000500D929F500D1124CA01AA2797FDA0957B
:1030D000BA2F8C0F9D1FAE1FBF1F2F5F3F4F44277E
:1030E00037FD4095542FBC01CD010E94BE70309336
:1030F000DF012093DE0104C0D093DF01C093DE0125
:1031000080916006282F3327220F331F220F331F91
:103110008091DE019091DF01821793077CF080910E
:103120006106282F3327220F331F220F331F809170
:10313000DE019091DF012817390724F43093DF0175
:103140002093DE0110921101E6E0CDB7DEB70C94BA
:1031500001711F920F920FB60F9211242F933F937C
:103160004F935F938F939F93EF93FF938091EF0122
:10317000882309F0DDC08091B00086FF9FC0809158
:10318000B0008F7B8093B000E091F2012091620645
:10319000EE23D9F433278DED96E0289FA001299FD7
:1031A000500D389F500D1124CA012091F00130912B
:1031B000F101821B930B9093E3018093E201109243
:1031C000F1011092F001469AB0C02E1738F48AE04F
:1031D00090E09093E3018093E201A7C089EA93E035
:1031E0009093E3018093E2018E2F9927833091051C
:1031F000D9F08430910534F48130910549F002977B
:1032000061F020C08430910591F0059799F01AC0C3
:103210008091E0019091E10104C08091DE019091E4
:10322000DF0187559E4F1DC08091AC0805C080917D
:103230008D0802C08091B5089927880F991F880FC3
:10324000991FEFCFFF27EE0FFF1FE350F84F2081AC
:103250003181220F331F8091E2019091E301820FAF
:10326000931F9093E3018093E2018091E20190919A
:10327000E30155E08D3D950718F08CED95E005C014
:103280008757914030F487E791E09093E301809372
:10329000E2012091E2013091E3012C5B3040309358
:1032A000E3012093E2018091F0019091F101820FFE
:1032B000931F9093F1018093F00137C08091B0008B
:1032C00080648093B0008CEB90E09093E301809356
:1032D000E2018091F0019091F10184549F4F90930D
:1032E000F1018093F0018091E501882321F0809124
:1032F0009402882321F48091E501823011F44698EC
:1033000001C0469A8091F2018F5F8093F201282FCD
:1033100033278091620699270196821793072CF430
:1033200081E0809311011092F20181E08093EF011E
:103330002091E2013091E30141E02F37340730F072
:103340008FEF8093B3002F5F30400FC02F3F3105C8
:10335000C9F0C0F0A9014F5F50404F37510550F4FC
:1033600080E88093B300205830403093E3012093ED
:10337000E20112C08FEF8093B3005093E3014093BA
:10338000E2010AC08091E2018093B3001092E30150
:103390001092E2011092EF01FF91EF919F918F91B6
:1033A0005F914F913F912F910F900FBE0F901F9003
:1033B000189510927C008FEC80937A00089580918C
:1033C000520260911301709114012091030288232D
:1033D00079F0CB01AA27BB27332727FD3095432F50
:1033E000532FBC01CD010E944A70DC01CB0116C0F5
:1033F00084E0660F771F8A95E1F7CB01AA27BB27E8
:10340000332727FD3095432F532FBC01CD010E9458
:103410004A70DC01CB010497A109B1098093FB013B
:103420009093FC01A093FD01B093FE010895CF930A
:10343000DF93109203020E94DF1983E090E00E9464
:103440008426C82FDD27C03FD10508F42A96C7BDC2
:103450008C2F809588BD86E990E00E94D6158091DA
:10346000190190911A018152934010F0C0EFD0E001
:10347000C630D10510F1C7BD8C2F809588BD84E67C
:1034800090E00E94D61585E094E09F938F938EED97
:1034900091E19F938F93E0918903F0918A030995BD
:1034A0008091190190911A010F900F900F900F9039
:1034B0008152934010F42197DBCFC093D9056C2F34
:1034C00083E090E00E948C2680913A0680FF0AC03B
:1034D0008091D9058A508C3D28F08091A2038064A8
:1034E0008093A2038CE291E00E94D615DF91CF91E8
:1034F00008951F920F920FB60F9211242F933F93AE
:103500004F935F936F937F938F939F93AF93BF93EB
:10351000CF93DF93EF93FF9380911B02282F3327E4
:10352000442755278F5F80931B02F9012231310513
:1035300008F0CEC3E25CFF4F0C94107180917800CC
:103540009091790046C080917800909179007BC17C
:10355000809178009091790090931F0280931E02D1
:103560008BC18091DC029091DD0220917800309136
:103570007900821B930B9093CC058093CB058091AF
:10358000CB059091CC05909329028093280292C19B
:1035900080917800909179002091DE023091DF02D5
:1035A000821B930B9093D8058093D7058091D70504
:1035B0009091D80590932B0280932A028BC380911F
:1035C0002202909123022091780030917900820F9D
:1035D000931F909323028093220281E07CC3809109
:1035E0002002909121022091780030917900820F81
:1035F000931F909321028093200284E06CC38091FA
:10360000310290913202892B91F42091780030910F
:103610007900C901E3E0880F991FEA95E1F7820F6D
:10362000931F820F931F9093320280933102209157
:10363000780030917900C90173E0880F991F7A955D
:10364000E1F7820F931F820F931F20913102309177
:1036500032028217930718F02E5F3F4F02C02250AC
:1036600030403093320220933102809131029091A8
:1036700032026FE170E00E947570709324016093D4
:10368000230185E028C38091780090917900909380
:10369000CE058093CD058091CD059091CE054091CA
:1036A000D8025091D902841B950B2091D702332761
:1036B00027FD3095821B930B90930902809308029B
:1036C00080915202882309F06DC080910802909188
:1036D000090202977CF122E04E3E52070CF062C0D4
:1036E00020911C0230911D022B5F3F4F30931D0231
:1036F00020931C022550304080915C0290915D0225
:10370000845F914030F4215F3F4F30931D0220933E
:103710001C0280911C0290911D02853691050CF4CB
:1037200041C04F5F5F4F5093D9024093D8028456F7
:10373000904034C080910802909109028F5F9F4FA2
:103740008CF562E0473256076CF120911C023091F3
:103750001D022550304030931D0220931C022B5F28
:103760003F4F80915C0290915D02845F914030F404
:103770002F50304030931D0220931C0280911C0278
:1037800090911D022FEF8C39920764F44150504004
:103790005093D9024093D8028C599F4F90931D02A9
:1037A00080931C0280910802909109029C01442799
:1037B00037FD4095542F8091AE029091AF02A091B9
:1037C000B002B091B102820F931FA41FB51F809366
:1037D000AE029093AF02A093B002B093B1022091D9
:1037E000AE023091AF024091B0025091B10257FF4A
:1037F00004C021503C4F4F4F5F4F6AE055954795AD
:10380000379527956A95D1F78091AE029091AF02D6
:10381000A091B002B091B102821B930BA40BB50B27
:103820008093AE029093AF02A093B002B093B10226
:10383000F5C0809120029091210220917800309172
:103840007900820F931F909321028093200210929F
:103850001A0243C2209178003091790080911E02B3
:1038600090911F02280F391F8FEF97E0821B930B57
:1038700090930F0280930E0286E02DC28091DC02AD
:103880009091DD022091780030917900821B930B9A
:103890009093CC058093CB058091CB059091CC057E
:1038A0002091280230912902820F931F90930D02DC
:1038B00080930C0287E00FC280917800909179008C
:1038C0002091DE023091DF02821B930B9093D8058A
:1038D0008093D7058091D7059091D80520912A0231
:1038E00030912B02820F931F90930B0280930A0258
:1038F000F1C12091220230912302809178009091B1
:103900007900280F391F220F331F220F331F3093E6
:10391000230220932202C90137FD079643E09595C3
:1039200087954A95E1F79093130280931202809154
:10393000240290912502820F931F97FD0196959581
:10394000879590932502809324022091E80230917C
:10395000E902821B930B9093220180932101209115
:103960001802309119028091210190912201280FB3
:10397000391F37FF02C02F5F3F4F35952795309392
:1039800019022093180229CE2091200230912102A1
:103990008091780090917900280F391F220F331FF2
:1039A000220F331F3093210220932002C90137FDDB
:1039B0000796F3E095958795FA95E1F790931102B4
:1039C000809310028091260290912702820F931F0C
:1039D00097FD0196959587959093270280932602EF
:1039E0002091E6023091E702821B930B9093200115
:1039F00080931F01209116023091170280911F01C0
:103A000090912001280F391F37FF02C02F5F3F4FD1
:103A100035952795309317022093160283E05BC1FA
:103A200010921B0281E0809315018091FF0190911B
:103A300000020196909300028093FF01809178002C
:103A40009091790090931A01809319018091190146
:103A500090911A01AA27BB27C0912C02D0912D0268
:103A6000E0912E02F0912F02C80FD91FEA1FFB1F11
:103A7000C0932C02D0932D02E0932E02F0932F02DC
:103A8000809130028F5F80933002803108F422C130
:103A900080911B0190911C01A0911D01B0911E010C
:103AA0009C01AD0163E0220F331F441F551F6A952F
:103AB000D1F7281B390B4A0B5B0B2C0F3D1F4E1FF8
:103AC0005F1F8091FB019091FC01A091FD01B091DD
:103AD000FE01281B390B4A0B5B0B57FF04C0295F03
:103AE0003F4F4F4F5F4F93E055954795379527953B
:103AF0009A95D1F720931B0130931C0140931D012F
:103B000050931E01C091CF05D091D005E091D10511
:103B1000F091D20580911B0190911C01A0911D0193
:103B2000B0911E01C81BD90BEA0BFB0BC093F3012C
:103B3000D093F401E093F501F093F6012091040293
:103B400030910502409106025091070257FF04C0D0
:103B5000215F3F4F4F4F5F4F84E055954795379515
:103B600027958A95D1F78091040290910502A09142
:103B70000602B0910702821B930BA40BB50B809336
:103B8000040290930502A0930602B093070280916D
:103B9000040290910502A0910602B09107028C0FD9
:103BA0009D1FAE1FBF1F8093040290930502A09338
:103BB0000602B09307028091040290910502A09141
:103BC0000602B0910702B7FF03C00F96A11DB11DF9
:103BD000C4E0B595A79597958795CA95D1F720919B
:103BE000F3013091F401281B390B64E021303607D2
:103BF0001CF020E034E006C08CEF2030380714F4CD
:103C000020E03CEF8091010290910202809101023C
:103C10009091020297FF03C0909581959F4FA90153
:103C2000F3E0440F551FFA95E1F78D5B9240C4F025
:103C300080910102909102029C01E4E0220F331F67
:103C4000EA95E1F7281B390B240F351F37FF02C017
:103C5000215F3F4F74E0359527957A95E1F717C0BE
:103C600080910102909102029C0165E0220F331FB6
:103C70006A95E1F7281B390B240F351F37FF02C067
:103C8000215E3F4F45E0359527954A95E1F7309302
:103C900002022093010280912C0290912D02A091AA
:103CA0002E02B0912F02B7FF03C00196A11DB11DD6
:103CB000B595A7959795879580932C0290932D02A3
:103CC000A0932E02B0932F0288E08093300202C0AE
:103CD00010921B0282E080931A0280911A02809354
:103CE0007C0080911B02882319F08FEC80937A006E
:103CF000FF91EF91DF91CF91BF91AF919F918F9104
:103D00007F916F915F914F913F912F910F900FBED7
:103D10000F901F90189590E2ECEDF5E08FE49193F1
:103D2000815087FFFCCF089590913502903540F483
:103D3000E92FFF27E452FA4F80839F5F909335026B
:103D40000895A0E0B0E0E7EAFEE10C94E370209172
:103D5000330220FF0AC080913402882311F0815081
:103D600002C0809125018093340221FF0CC0909104
:103D7000340280912501981719F41092340203C07F
:103D80009F5F90933402822F992780FF04C081FFA8
:103D900002C0109234020E948B1E80913402282FA0
:103DA000332704E91EE1C0918903D0918A038A3048
:103DB00098F481E1809335023F932F9387E094E05C
:103DC0009F938F931F930F93FE0109952DB73EB7D5
:103DD0002A5F3F4F2DBF11C080E1809335023F9392
:103DE0002F938CE094E09F938F931F930F93FE018A
:103DF00009958DB79EB706968DBF20913402822F0C
:103E00009927AA27BB27FC010D9708F072C5E05B34
:103E1000FF4F04E91EE1C0918903D0918A030C94FD
:103E200010711092350281E194E09F938F9394E991
:103E3000E92E9EE1F92E1F930F93FE01099584E16F
:103E4000809335020F900F900F900F9081E690E0D5
:103E50009F938F9388E090E09F938F9382E090E010
:103E60009F938F93809103016AE00E946970892F6C
:103E700099279F938F93809103010E9469709927DE
:103E80009F938F9381E294E09F938F931F930F935F
:103E9000E0918903F0918A03099588E280933502C5
:103EA000EDB7FEB73E96EDBF87EB96E09F938F93FD
:103EB0008091010199279F938F9389E394E09F93C9
:103EC0008F931F930F93E0918903F0918A030995D3
:103ED000809159022DB73EB7285F3F4F2DBF81FF1C
:103EE00012C088E38093350283E494E09F938F931C
:103EF0001F930F93E0918903F0918A0309950F9026
:103F00000F900F900F908091A30384FF06C08CE365
:103F10008093350288E494E039C09091A2039923FC
:103F200051F08CE380933502892F99279F938F93CB
:103F300085E594E047C090913B02992351F08CE3D2
:103F400080933502892F99279F938F938CE694E075
:103F50002EC190914203992371F08CE38093350236
:103F6000892F99279F938F9382E894E09F938F9353
:103F7000FF92EF9252C38091390190913A010697D6
:103F800098F48CE38093350283E994E09F938F93B8
:103F9000FF92EF92E0918903F0918A0309950F90C7
:103FA0000F900F900F90AEC4909178099E3108F059
:103FB000A9C48CE380933502892F99279F938F930F
:103FC00080EA94E09F938F93FF92EF92E0918903B0
:103FD000F0918A0309958DB79EB706968DBF92C45E
:103FE0001092350280918E0290918F02A0919002E2
:103FF000B0919102BC01CD0125E030E040E050E0FD
:104000000E94BE703F932F9384EB94E09F938F9315
:104010001F930F93FE01099584E180933502EDB75C
:10402000FEB73696EDBF80918A0290918B02A091E7
:104030008C02B0918D02BC01CD0125E030E040E062
:1040400050E00E94BE703F932F9381EC94E09F93C9
:104050008F931F930F93E0918903F0918A03099541
:1040600088E2809335022DB73EB72A5F3F4F2DBFC0
:104070008091190190911A019F938F938EEC94E097
:104080009F938F931F930F93E0918903F0918A037D
:1040900009958CE3809335028DB79EB706968DBF48
:1040A00087B599279F938F938BED94E09F938F9380
:1040B0001F930F93E0918903F0918A030995EDB75F
:1040C000FEB736965AC31092350288EE94E09F935D
:1040D0008F9384E9E82E8EE1F82E1F930F93FE0153
:1040E000099584E1809335020F900F900F900F9007
:1040F0008091D2029091D302A091D402B091D502C6
:10410000B7FF04C081509C4FAF4FBF4F1AE0B59529
:10411000A795979587951A95D1F7BF93AF939F93DE
:104120008F9385EF94E09F938F93FF92EF92E091AE
:104130008903F0918A03099588E2809335022DB7AF
:104140003EB7285F3F4F2DBF8091CE029091CF02A6
:10415000A091D002B091D102B7FF04C081509C4F12
:10416000AF4FBF4FCAE0B595A79597958795CA956C
:10417000D1F7BF93AF939F938F9384E095E09F9384
:104180008F93FF92EF92E0918903F0918A03099552
:104190008CE3809335028DB79EB708968DBF8091D2
:1041A000D9089091DA089F938F9383E195E09F93CC
:1041B0008F93FF92EF927ECFF1E0FF2EC1E0D0E02F
:1041C0000FEF17E09F2D969584E1989FC001112471
:1041D00080933502F801828193819F938F9321967A
:1041E000DF93CF932197808191819F938F93DF936A
:1041F000CF9382E295E09F938F9384E99EE19F9312
:104200008F93E0918903F0918A0309952DB73EB70A
:10421000245F3F4F2DBF32E0F30E22960C5F1F4FFD
:1042200088E08F1578F66EC31092350280912F06C4
:10423000E82FFF27EE0FFF1FE350F84F8081918199
:104240009F938F9380912E06E82FFF27EE0FFF1F7D
:10425000E350F84F808191819F938F9384E395E0A1
:104260009F938F931F930F93FE01099584E1809391
:104270003502EDB7FEB73896EDBF80913106E82FD5
:10428000FF27EE0FFF1FE350F84F808191819F932E
:104290008F9380913006E82FFF27EE0FFF1FE3502A
:1042A000F84F8081918181589F4F9F938F9384E431
:1042B00095E09F938F931F930F93E0918903F09163
:1042C0008A03099588E2809335022DB73EB7285FAF
:1042D0003F4F2DBF80913306E82FFF27EE0FFF1FC2
:1042E000E350F84F8081918181589F4F9F938F9326
:1042F00080913206E82FFF27EE0FFF1FE350F84FA3
:104300008081918181589F4F9F938F9384E595E0A1
:104310009F938F931F930F93E0918903F0918A03EA
:1043200009958CE3809335028DB79EB708968DBFB3
:1043300080913506E82FFF27EE0FFF1FE350F84F5F
:104340008081918181589F4F9F938F9380913406F4
:10435000E82FFF27EE0FFF1FE350F84F8081918178
:1043600081589F4F9F938F9384E695E0FAC11092F6
:10437000350284E795E09F938F93E4E9EE2EEEE11A
:10438000FE2E1F930F93FE01099584E18093350261
:104390000F900F900F900F908091E8029091E9029A
:1043A0009F938F932091E8023091E90237FF02C07A
:1043B000295F3F4F73E0359527957A95E1F7809116
:1043C000120290911302821B930B9F938F9382E8AA
:1043D00095E09F938F93FF92EF92E0918903F09184
:1043E0008A03099588E2809335022DB73EB7285F8E
:1043F0003F4F2DBF8091E6029091E7029F938F93EC
:104400002091E6023091E70237FF02C0295F3F4F5B
:1044100063E0359527956A95E1F7809110029091B8
:104420001102821B930B9F938F9381E995E09F93D9
:104430008F93FF92EF92E0918903F0918A0309959F
:104440008CE3809335028DB79EB708968DBF80911F
:10445000E4029091E5029F938F938091E402909102
:10446000E50220910E0230910F02821B930B9F9365
:104470008F9380EA95E09F938F93FF92EF9275C19F
:10448000109235028FEA95E09F938F931F930F93BD
:10449000FE01099584E1809335020F900F900F90F3
:1044A0000F908091DE029091DF029F938F93809115
:1044B0000A0290910B029F938F938CEB95E09F9350
:1044C0008F931F930F93E0918903F0918A030995CD
:1044D00088E2809335022DB73EB7285F3F4F2DBF4E
:1044E0008091DC029091DD029F938F9380910C026A
:1044F00090910D029F938F938BEC95E09F938F93F8
:104500001F930F93E0918903F0918A0309958CE33F
:10451000809335028DB79EB708968DBF8091D802E3
:104520009091D9029F938F938091080290910902F4
:104530009F938F938AED95E014C11092350280917C
:104540002301909124016AE070E00E9489709F939A
:104550008F9380912301909124016AE070E00E9482
:1045600089707F936F9389EE95E09F938F931F934C
:104570000F93FE01099584E1809335022DB73EB774
:10458000285F3F4F2DBF80917209909173096AE0B7
:1045900070E00E9475709F938F9380917209909143
:1045A00073096AE070E00E9475707F936F938DEFDE
:1045B00095E09F938F931F930F93E0918903F09160
:1045C0008A03099588E2809335028DB79EB70896D5
:1045D0008DBF80917409909175099F938F9381E1AC
:1045E00096E09F938F931F930F93E0918903F0912F
:1045F0008A0309958CE380933502EDB7FEB73696B2
:10460000EDBF80917609909177099F938F9381E216
:1046100096E09F938F931F930F93E0918903F091FE
:104620008A0309952DB73EB72A5F3F4F2DBF6AC158
:104630001092350283E396E09F938F931F930F931D
:10464000FE01099588E2809335020F900F900F903C
:104650000F908091940299279F938F938CE396E01B
:104660009F938F931F930F93E0918903F0918A0397
:1046700009958CE3809335028DB79EB706968DBF62
:104680008091FC07992701979F938F938CE496E084
:104690000DCD109235028CE596E09F938F931F937A
:1046A0000F93FE01099584E1809335020F900F90DE
:1046B0000F900F90809102016AE00E946970892F2B
:1046C00099279F938F93809102010E946970992787
:1046D0009F938F938CE696E09F938F931F930F93F6
:1046E000E0918903F0918A03099588E2809335026D
:1046F0002DB73EB7285F3F4F2DBF8091B8016AE0CC
:104700000E946970892F99279F938F938091B80198
:104710000E94697099279F938F938AE796E09F93F1
:104720008F931F930F93E0918903F0918A0309956A
:104730008CE3809335028DB79EB708968DBF80912C
:10474000B9016AE00E946970892F99279F938F931E
:104750008091B9010E94697099279F938F9388E88F
:1047600096E09F938F931F930F93E0918903F091AD
:104770008A030995EDB7FEB73896EDBFC3C055E97A
:10478000C52E52E0D52E20E030E0E90143E0F42EC2
:10479000C0933502F60181916F0199279F938F9302
:1047A00089010F5F1F4F1F930F9386E996E09F9338
:1047B0008F9384E99EE19F938F93E0918903F09119
:1047C0008A0309952DB73EB7285F3F4F2DBFFA9456
:1047D00064969801F7FEDCCF95C099E9C92E92E066
:1047E000D92EC0E0D0E08E0183E0F82E0093350290
:1047F000F60181916F0199279F938F932596DF93FF
:10480000CF9383EA96E09F938F9384E99EE19F93F1
:104810008F93E0918903F0918A0309952DB73EB7F4
:10482000285F3F4F2DBFFA940C5E1F4F2497F7FE71
:10483000DDCF68C01092350280EB96E09F938F9396
:104840001F930F93FE01099584E1809335020F9029
:104850000F900F900F908091B4019091B5019F93AC
:104860008F938EEB96E09F938F931F930F93E0911E
:104870008903F0918A03099588E2809335028DB708
:104880009EB706968DBF8091B6019091B7019F9318
:104890008F938BEC96E09F938F931F930F93E091F0
:1048A0008903F0918A03099589E480933502EDB775
:1048B000FEB73696EDBF88ED96E09F938F931F93DA
:1048C0000F93E0918903F0918A0309958091330257
:1048D0000F900F900F900F9083FF14C01092B701AC
:1048E0001092B60160E070E08EE090E00E949D269C
:1048F00009C080912501281719F421502093250122
:104900001092340210923302E8E0CDB7DEB70C9477
:10491000FF70F999FECF92BD81BDF89A80B59927B5
:104920000895F999FECF1FBA92BD81BD60BD0FB643
:10493000F894FA9AF99A0FBE08954AEA20E030E016
:104940002617370740F4FC018191480F2F5F3F4F36
:1049500026173707C8F3842F99270895EAEA40E01D
:1049600050E04617570778F49C01F999FECF32BD05
:1049700021BDF89A80B5E80F4F5F5F4F2F5F3F4F23
:104980004617570790F38E2F9927089581E080935B
:10499000300682E080932F0683E080932E0684E029
:1049A0008093310685E08093320686E0809333065B
:1049B00087E08093340688E08093350689E0809311
:1049C00036068AE0809337068BE0809338068CE0C9
:1049D00080933906089587E680932D069CE0E9EAE6
:1049E000F6E0892F11928A95E9F78AE080934D06C7
:1049F000109271068BE1809349068EE480936E06D7
:104A000080936F06B0E2B09370061092A5068AE616
:104A100080933A0682E78093A70680E58093A806F4
:104A200084E0809354061092920610928F0678E0EC
:104A30007093470626EE2093480680E480934A064A
:104A400085E080933D06FEE1F0933B068EE6809381
:104A500042068FE080933E06F0933C06109240069B
:104A600070934106109243061092950680933F067C
:104A700010929E0690939F0610925606109257062B
:104A800010925806109259061092730610927406EE
:104A9000109275061092760690E890935A0642E3BB
:104AA00040935B06A2E0A093A60688E180935C0693
:104AB00020935D0683E0809362065DE75093650670
:104AC000509366065093670690935E06E5E5E09383
:104AD0005F0666E4609360068CED809361068CE36C
:104AE00080936306109264069AEA909377068CECA2
:104AF0008093790610927B0690937C0698E29093BF
:104B0000780690937A0610927D061092A306409341
:104B1000A406409368062AE52093690640936A0636
:104B200036E030937E0684E680937F06809380068D
:104B30002093810688E780938206909386068BE413
:104B400080938306E09384068093850630938706DE
:104B500070938806409389068AE280938A061092B1
:104B60008B0610928E069CE890938C06A0938D067F
:104B7000109290061092910681E480935206209341
:104B80005306109293061092940686E98093960637
:104B900050936B0684E380936C06109297061092F4
:104BA00098061092990690939A0660939B069093AC
:104BB0009C0660939D061092A006B09351068FE16B
:104BC0008093A206F093A10608950E94EB248AE048
:104BD0008093440680E18093450626E020934606B4
:104BE0009AE590934B0688E780934C0690934E0687
:104BF00080934F062093500680E2809355068CE305
:104C000080936D068BE48093720686E491E6A3E7B9
:104C1000B4E78093A9069093AA06A093AB06B0933D
:104C2000AC0668E870E08DE296E00E949D248093D7
:104C3000B5060895CF93DF930E94EB2488E080931C
:104C4000440630E13093450626E02093460694E67C
:104C500090934B0688E780934C0690934E06809382
:104C60004F06209350063093550686E480936D06D8
:104C700080937206A9EAB6E085E0E6E2F1E0ED0194
:104C8000019009928A95E1F768E870E0CD018C57B0
:104C900090400E949D248093B506DF91CF910895A6
:104CA0000E94EB2426E0209344068AE08093450688
:104CB00084E08093460694E690934B0688E78093C1
:104CC0004C0690934E0680934F062093500680E149
:104CD0008093550686E480936D068093720685E482
:104CE00091E6A3E7B9E78093A9069093AA06A0935B
:104CF000AB06B093AC0668E870E08DE296E00E94E7
:104D00009D248093B5060895F999FECF92BD81BD8B
:104D1000F89A80B599270895F999FECF1FBA92BDE8
:104D200081BD60BD0FB6F894FA9AF99A0FBE089546
:104D300069E874E20E94D86E089541E954E20E9445
:104D4000126F0895EF92FF920F931F93CF93C82F86
:104D50008150853008F0C3E089E8C89F80011124A4
:104D60008BEDE82E8FEFF82EE00EF11E68E870E074
:104D7000C7010E94AE24682F98012D593F4F8FB371
:104D80009927AC014270507081FDF9CF32BD21BD31
:104D9000F89A80B5861711F0CA0121C08FB3992700
:104DA0009C012270307081FDF9CFF2BCE1BCF89A11
:104DB00080B5873611F0C90112C089E8C89FC001CB
:104DC0001124859729E834E249E850E0BC018DE2DE
:104DD00096E00E94B36E0E94AB6181E090E0CF91BB
:104DE0001F910F91FF90EF900895282F863010F0BB
:104DF00025E003C0882309F421E020930101F999FB
:104E0000FECF1FBA82E090E092BD81BD20BD0FB6FB
:104E1000F894FA9AF99A0FBE0895CF93C82F80910B
:104E20002D06873609F04FC0C63010F0C5E003C02C
:104E3000CC2309F448C00E94AC6D8091A80682FF83
:104E400007C080915206843618F080E580935206A0
:104E500068E870E08DE296E00E949D248093B5069C
:104E600089E8C89FC001112421E934E249E850E0F3
:104E70006DE276E085970E94F06E21E934E24CE025
:104E800050E06EE276E080E590E00E94F06E6CE02B
:104E900070E08EE296E00E949D24282FF999FECFC3
:104EA0001FBA8CE590E092BD81BD20BD0FB6F8948D
:104EB000FA9AF99A0FBE8C2F0E94F5260E94AB61D8
:104EC00081E090E002C080E090E0CF9108956DE431
:104ED00070E088EE93E00E94AE24482F8FB39927AC
:104EE0009C012270307081FDF9CF85E394E092BD82
:104EF00081BDF89A80B5841779F48FB399279C0106
:104F00002270307081FDF9CF88EE93E092BD81BDB3
:104F1000F89A80B5813011F0C901089529E834E28A
:104F20004EE450E068EE73E086EB96E00E94B36ECC
:104F300081E090E008958091B6068130A9F46DE497
:104F400070E086EB96E00E949D248093030721E9A0
:104F500034E24EE450E066EB76E088EE93E00E94A7
:104F6000F06E81E090E0089580E090E00895CF93A6
:104F7000DF9381E08093B606E6EBF6E08FE01586DE
:104F800016861786108A8150349687FFF8CF80E402
:104F90008093C3068093C4061092C5068093C6060C
:104FA0008093C70690EC9093C8061092C906809330
:104FB000CA068093CB061092CC069093CD069093B0
:104FC000CE068093CF061092D0068093D1069093A0
:104FD000D206A7EBB6E08CE0ECE2F1E0ED01019047
:104FE00009928A95E1F76DE470E0CD0101970E9486
:104FF0009D2480930307DF91CF910895F999FECF07
:1050000082E090E092BD81BDF89A80B5282F86306D
:1050100078F023E0322FF999FECF1FBA82E090E0BA
:1050200092BD81BD30BD0FB6F894FA9AF99A0FBEC1
:1050300020930101822F992708951F93CF93C82FA2
:10504000162F863010F0C5E003C0882309F4C1E0B4
:105050008C2F99278230910541F08330910544F4DB
:10506000019731F40E94E52505C00E941A2602C06E
:105070000E9450261123E1F06CE070E080E590E0A2
:105080000E94AE24282FF999FECF8CE590E092BDC6
:1050900081BDF89A80B5821759F429E834E24CE0D2
:1050A00050E060E570E08EE296E00E94B36E02C0D0
:1050B0000E94C6248C2F0E940D27CF911F91089526
:1050C000DF92EF92FF920F931F93CF93FF24DF2C79
:1050D000EF2C81E090E00E948426873611F031E0C9
:1050E000E32E6CE070E080E590E00E94AE24C82FD3
:1050F000F999FECF8CE590E092BD81BDF89A80B51C
:105100008C1711F421E0D22EC1E001E010E0EE2076
:1051100029F48C2F0E94A2268823B9F591E0F92E5C
:105120001F930F9380EE96E09F938F938EED91E106
:105130009F938F93E0918903F0918A0309952DB78E
:105140003EB72A5F3F4F2DBF0130110521F00230DD
:10515000110521F006C00E94E52505C00E941A260F
:1051600002C00E945026DD2059F029E834E24CE0CC
:1051700050E060E570E08EE296E00E94B36E02C0FF
:105180000E94C6248C2F0E940D27CF5F0F5F1F4FF8
:10519000C63008F4BCCFFF2019F083E00E94F5264A
:1051A0000E94FE27C82F0E94A2268C2F99279F932A
:1051B0008F9386E097E09F938F930EED11E11F93FD
:1051C0000F93E0918903F0918A03099581E090E0C3
:1051D0000E9484262DB73EB72A5F3F4F2DBF8F3FD9
:1051E00021F00E946727882399F48FE197E09F932D
:1051F0008F931F930F93E0918903F0918A03099590
:105200000E94B7270E949B270F900F900F900F903E
:10521000EE2029F067E681E090E00E948C26109253
:105220002C0690E0E3ECF6E0CFE08081349618168F
:105230000CF49F5FC150C7FFF8CF90932C06892FC5
:1052400099279F938F9387EB96E09F938F9380E4AA
:1052500097E09F938F931F930F93E0918903F091B1
:105260008A0309950E940A058DB79EB708968DBFDF
:10527000CF911F910F91FF90EF90DF900895982F9D
:105280002FB7F8943998389A88B1836088B980919B
:10529000B9008C7F8093B9008AE28093B8001092A5
:1052A000400210923E0210923D029923B1F0E8E4D0
:1052B000F7E08BE010821182128213821482158231
:1052C0001682178216861086118612861386148619
:1052D000158681503F9687FFEDCF78942FBF0895B4
:1052E0001092400284E98093BC0080E88093BC0067
:1052F0001092BD001092BA001092BB001092B9003B
:105300001092B80010923C0280E00E943F29109257
:10531000BB0085E88093BC0080913A028260809354
:105320003A0208951F920F920FB60F9211242F93F5
:105330003F936F937F938F939F93EF93FF9380910E
:105340004002282F33278F5F80934002233031059E
:1053500009F41CC1243031055CF42130310509F415
:1053600054C0223031050CF099C0232B71F02EC3AC
:105370002530310509F470C1253031050CF41EC10A
:105380002630310509F434C221C381E080933C0208
:1053900009C080913E028C3090F480913E028F5F74
:1053A00080933E0280913E02E82FFF27EE0FFF1F01
:1053B000EE0FFF1FEA54F94F8585181654F78091B8
:1053C0003E026CE00E94697090933E02809146021A
:1053D0008F5F8093460290913B01981770F4109272
:1053E0004602109239021092380285E08093400202
:1053F00080913D02880F8D5A04C080913E02880F33
:105400008E5A8093BB0085E824C180913E02992783
:10541000FC0124E0EE0FFF1F2A95E1F7E81BF90BD2
:10542000E85BF84F81818093BB0085E88093BC00E6
:1054300080913E029927FC01E295F295F07FFE27CC
:10544000E07FFE27E81BF90BE85BF84F808180FFC7
:105450009BC080913E029927FC01E295F295F07F76
:10546000FE27E07FFE27E81BF90BE85BF84F8281FF
:10547000882329F080912C06873008F4BDC28091E2
:10548000380290913902892B09F0B6C28091360218
:1054900090913702892B09F0AFC276C080913E020D
:1054A00021E030E002C0220F331F8A95E2F780919D
:1054B00036029091370228233923232B81F08091E3
:1054C0003E029927FC0174E0EE0FFF1F7A95E1F789
:1054D000E81BF90BE85BF84F80E184830EC08091F4
:1054E0003E029927FC0164E0EE0FFF1F6A95E1F789
:1054F000E81BF90BE85BF84F148280913E02992774
:10550000FC01E295F295F07FFE27E07FFE27E81B85
:10551000F90BE85BF84F8481282F3327220F331FC4
:10552000220F331F220F331F80913E029927FC0167
:1055300034E0EE0FFF1F3A95E1F7E81BF90BE85B4B
:10554000F84F82818770822B8093BB0085E880931F
:10555000BC0020913E0281E090E002C0880F991FBC
:105560002A95E2F720913802309139028223932361
:10557000892B51F080E497E090934402809343029A
:1055800088E08093450238C284E01DC2E091430266
:10559000F091440281918093BB0085E88093BC0028
:1055A000F0934402E093430280914502815080933E
:1055B0004502882309F420C283E005C28091B90026
:1055C000803379F580914102882329F480913E024D
:1055D0008F5F8093410280913E029927FC01E29502
:1055E000F295F07FFE27E07FFE27E81BF90BE85BD2
:1055F000F84F838199278F7790708F3791058CF4BE
:1056000080913E029927FC01E295F295F07FFE27FA
:10561000E07FFE27E81BF90BE85BF84F83818F5F83
:1056200083831092400284E98093BC008AE090E07A
:1056300090933A018093390180913E028F5F80936D
:105640003E021092400280913A028E7F80933A028D
:1056500085EA8093BC00D0C18091B9008034D1F13B
:1056600080913D029927FC0174E0EE0FFF1F7A95AF
:10567000E1F7E81BF90BE85BF84F83818F778383B1
:1056800080913D028F5F80933D0280913D028C307E
:10569000A0F010923D0210923702109236028091D3
:1056A00042028F5F809342028C3038F010924202A7
:1056B00080913A028D7F80933A0280913A02816014
:1056C00080933A021092400284E98093BC001092C9
:1056D0003C0287C080913D029927FC0164E0EE0FF7
:1056E000FF1F6A95E1F7E81BF90BE85BF84F838130
:1056F0008068838380913D029927FC01E295F295B1
:10570000F07FFE27E07FFE27E81BF90BE85BF84FF0
:10571000808180FF42C080913D029927FC01E29583
:10572000F295F07FFE27E07FFE27E81BF90BE85B90
:10573000F84F848199270097D9F0409709F048C025
:1057400080E497E0909344028093430288E0809342
:10575000450280913D029927FC0134E0EE0FFF1FC6
:105760003A95E1F7E81BF90BE85BF84F148230C07B
:1057700090913D028FE0989FC0011124835B984F68
:10578000909344028093430290913D0280914202A3
:105790009817D9F480913C0119C090913D028FE097
:1057A000989FC0011124835B984F9093440280938B
:1057B000430280913A0281FD06C090913D028091A2
:1057C0004202981711F482E001C081E08093450203
:1057D00080914502813011F485E801C085EC809309
:1057E000BC008091410280933B021092410204C1AF
:1057F000E0914302F09144028091BB00808380914C
:105800004302909144020196909344028093430294
:1058100080914502815080934502823010F085ECE2
:10582000CFC0813011F485E8CBC080913A0281FF6E
:105830007BC080915B0280FD77C080913D029927FB
:10584000FC0124E0EE0FFF1F2A95E1F7E81BF90B9E
:10585000E85BF84F868199278C7F9070883F91058F
:1058600091F480913D029927FC01E295F295F07F39
:10587000FE27E07FFE27E81BF90BE85BF84F8081ED
:10588000816080830FC080913D029927FC01E295E1
:10589000F295F07FFE27E07FFE27E81BF90BE85B1F
:1058A000F84F108280913D029927FC0174E0EE0FC1
:1058B000FF1F7A95E1F7E81BF90BE85BF84F86814B
:1058C000883F81F480913D029927FC0164E0EE0F4E
:1058D000FF1F6A95E1F7E81BF90BE85BF84F808141
:1058E000866021C080913D029927FC01E295F295E6
:1058F000F07FFE27E07FFE27E81BF90BE85BF84FFF
:105900008681893F89F480913D029927FC01E295C7
:10591000F295F07FFE27E07FFE27E81BF90BE85B9E
:10592000F84F80818460808380915B0281FF20C07A
:1059300080913D029927FC0134E0EE0FFF1F3A955C
:10594000E1F7E81BF90BE85BF84F86818E3F80F4A6
:1059500080913D029927FC0124E0EE0FFF1F2A955C
:10596000E1F7E81BF90BE85BF84F86858F5F8687C8
:1059700080913D028F5F80933D0280913D028C308B
:10598000A0F010923D0210923702109236028091E0
:1059900042028F5F809342028C3038F010924202B4
:1059A00080913A028D7F80933A021092400284E9FE
:1059B0008093BC0080913A02816080933A021AC0C1
:1059C0008093BC0086E08093400216C01092400293
:1059D00084E98093BC0080913A02816080933A020E
:1059E0008AE090E090933A018093390110923E0250
:1059F00010923D0210923C02FF91EF919F918F9186
:105A00007F916F913F912F910F900FBE0F901F903C
:105A100018950F931F93CF93DF93182F80919302C4
:105A2000882321F48091C501882319F081E090E05A
:105A300091C01D3008F08CC01123C9F0812F992727
:105A4000FC0144E0EE0FFF1F4A95E1F7E81BF90B5C
:105A5000E85BF84F3C9780813C9688230CF078C037
:105A60003F97808180FD03C083E090E073C0809108
:105A7000400799278B709070029719F084E090E0AE
:105A800069C067E070E080E497E00E949D249091F7
:105A90004707891719F085E090E05CC000913B0151
:105AA0008CE080933B0184E690E090933A018093F0
:105AB00039010E94B415EC0180913A0280FD05C0C5
:105AC000CE010E94BD158823B9F3112319F48FEF7D
:105AD0009FE00BC0212F33272150304081E090E020
:105AE00002C0880F991F2A95E2F79093390280939C
:105AF000380210923E0210923D0288EE93E00E941E
:105B0000B415EC011092400280913A028E7F80938E
:105B10003A0285EA8093BC0080913A0280FD05C07C
:105B2000CE010E94BD158823B9F38091380290916F
:105B30003902892B29F0CE010E94BD15882311F36B
:105B400000933B018091380290913902009711F047
:105B500082E090E0DF91CF911F910F9108950F9314
:105B60001F93CF93DF93982F80919302882321F482
:105B70008091C501882319F081E090E07BC09D30C1
:105B8000B0F4992319F486E090E074C0C92FDD27A2
:105B9000FE0154E0EE0FFF1F5A95E1F7EC1BFD0BE1
:105BA000E85BF84F3C9780813C9687FD03C082E01C
:105BB00090E060C03F97808180FD03C083E090E06B
:105BC00059C088EE93E00E94B4158C0180913A028E
:105BD00080FD05C0C8010E94BD158823B9F3219737
:105BE00081E090E002C0880F991FCA95E2F7909378
:105BF00037028093360210923E0210923D021092BC
:105C00004007109247071092400280913A028E7F1F
:105C100080933A0285EA8093BC0080913A0280FD2D
:105C200005C0C8010E94BD158823B9F380913602D2
:105C300090913702892B29F0C8010E94BD15882355
:105C400011F38091400799278B709070029719F09B
:105C500084E090E00FC067E070E080E497E00E948D
:105C60009D2490914707891719F085E090E002C0C4
:105C700080E090E0DF91CF911F910F910895CF9335
:105C8000DF9380E021E83FEFC3E4D8E0EDEFF7E0F9
:105C9000DF01853020F411961C921E9202C03183E0
:105CA00020831982188222968F5F12963296833251
:105CB00080F38FE790E090933C0880933B0881E865
:105CC0009FEF90933A088093390810923E08109203
:105CD0003D081092E5021092E4021092E702109241
:105CE000E6021092E9021092E802DF91CF91089546
:105CF0001F920F920FB60F9211240F931F932F93A1
:105D00003F934F935F936F937F938F939F93AF9343
:105D1000BF93CF93DF93EF93FF9340918600509111
:105D200087008091480290914902481B590B80914D
:105D30008600909187009093490280934802CA019F
:105D40008D549440A0914A02B0914B02835F9A41D6
:105D500058F480914A028093FC07149714F0109233
:105D60003F0181E090E0C1C0A131B1050CF0C1C09C
:105D7000CA018B5F9040845B914008F0B1C0809174
:105D80003D0190913E01481B590BE0919706EE238F
:105D900051F0FF27EE0FFF1FE350F84F80819181F4
:105DA00084369105ECF4FD01EA0FFB1FE350F84F38
:105DB00080819181FA01E81BF90BCF01F7FF03C045
:105DC000909581959F4F06975CF480919402883C52
:105DD00020F480919402865F01C088EC8093940245
:105DE000FD01EA0FFB1FE350F84F808191819C0178
:105DF000220F331F280F391F240F351F37FF02C012
:105E00002D5F3F4FE901D595C795D595C795CA0137
:105E100001968C179D0714F4219706C041505040FD
:105E2000C417D5070CF4219680919402833CD8F0D6
:105E30008D010A0F1B1FF801E350F84F80819181FB
:105E40009E01281B390BC90163E070E00E94897034
:105E5000CB01880F991F860F971F0D5B174FF80115
:105E60009183808307C0AA0FBB1FAD5BB74F11960C
:105E70001C921E92E0914A02F0914B02EE0FFF1F1E
:105E8000E350F84FD183C08380919402823340F570
:105E900080912E06E82FFF27EE0FFF1FE350F84FEB
:105EA0001182108280912F06E82FFF27EE0FFF1F2F
:105EB000E350F84F1182108280913106E82FFF27BE
:105EC000EE0FFF1FE350F84F1182108280913006D1
:105ED000E82FFF27EE0FFF1FE350F84F11821082CB
:105EE00080914A0290914B02019690934B028093CD
:105EF0004A02FF91EF91DF91CF91BF91AF919F91B6
:105F00008F917F916F915F914F913F912F911F9151
:105F10000F910F900FBE0F901F9018958091000960
:105F200090910109909389058093880580910209D9
:105F30009091030990938B0580938A058091D408F2
:105F40009091D50897FD039695958795959587959A
:105F500090938D0580938C058091E6089091E708D9
:105F600097FD0396959587959595879590938F05C1
:105F700080938E058091E4029091E50220910E02BB
:105F800030910F02821B930B9093910580939005A3
:105F900080918E0290918F02A0919002B091910217
:105FA000BC01CD012AE030E040E050E00E94BE702C
:105FB00030939305209392058091CD059091CE0565
:105FC000909395058093940580918F019091900115
:105FD00090939905809398058091230190912401D5
:105FE00090939B0580939A058091940299279093B2
:105FF0009D0580939C0580919508909196089093BB
:106000009F0580939E058091490799279093A1054C
:106010008093A0058091580799279093A3058093BA
:10602000A2058091670799279093A5058093A40501
:106030008091760799279093A7058093A605809174
:10604000E0019091E1019093B1058093B0058091BA
:106050007802909179029093B3058093B205809174
:106060007209909173099093B5058093B40580915E
:106070007609909177099093B7058093B605809142
:106080008A0290918B02A0918C02B0918D02BC018A
:10609000CD012AE030E040E050E00E94BE70309335
:1060A000B9052093B8058091780999279093C30585
:1060B0008093C20580913403909135039093C50578
:1060C0008093C40580913203909133039093C70568
:1060D0008093C6058091A203882321F48091A303B5
:1060E000882321F080918705816003C08091870516
:1060F0008E7F809387050895EF92FF921F93CF9331
:10610000DF93182F7B0180919302882371F5809192
:106110000301893111F4299801C0299A11501F3FB8
:10612000E9F0F092E801E092E701E7018091E701F0
:106130009091E801892B11F4209781F38091EB0174
:106140008823A1F31092EB018091E7019091E8017F
:10615000892B09F421970E94C26DE8CF8091030139
:10616000893111F4299A01C02998DF91CF911F91AB
:10617000FF90EF900895EF92FF920F931F9310926C
:106180007A00809112029091130290939C08809360
:106190009B08809110029091110290939108809336
:1061A000900880910E0290910F029093DC088093EA
:1061B000DB0820910A0230910B02C901880F991F58
:1061C000880F991F820F931F820F931F9093D508FA
:1061D0008093D40820910C0230910D02C901880FE0
:1061E000991F880F991F820F931F820F931F9093FF
:1061F000E7088093E6088FEC80937A0080916E0622
:106200009927AA27BB2744ECE42E49E0F42E012D60
:10621000112DBC01CD01A80197010E944A70DC013B
:10622000CB018093870190938801A0938901B0935B
:106230008A0180916F069927AA27BB27BC01CD014F
:106240000E944A70DC01CB0180938301909384010A
:10625000A0938501B09386011F910F91FF90EF905D
:106260000895A0E0B0E0E7E3F1E30C94DD70782E50
:1062700091E0692EEE24FF24570147018701109217
:10628000A203F092DF02E092DE02F092DD02E092E1
:10629000DC02F092D902E092D8021092D702F0927A
:1062A000E902E092E802F092E702E092E602F09260
:1062B000E502E092E40210926901109268011092E6
:1062C000030223E0821729F48091590282608093AF
:1062D00059020E94BB3084E690E00E94D6150E94CD
:1062E000BB3080913A0680FF14C0809119019091D3
:1062F0001A01875B934058F48091190190911A011B
:106300008E5E924020F080910302882311F00E945B
:10631000171AC0911901D0911A0187B5865F87BD00
:1063200087B5809588BD8FE1C82E8AE090E00E94F5
:10633000D61580910E0290910F02E80EF91E809101
:10634000120290911302A80EB91E80911002909132
:106350001102880E991E8091CD059091CE05080FEF
:10636000191FCA94C7FEE1CF8091190190911A01BB
:10637000825F934080F48091190190911A014597B2
:1063800050F08091190190911A01C81BD90BD0933C
:106390001401C093130187B58A5087BD87B58095D6
:1063A00088BD9501205F3F4F3695279536952795F7
:1063B0003093E9022093E802C401409696958795B0
:1063C000969587959093E7028093E60240E150E02E
:1063D000E40EF51EA5E0F694E794AA95E1F7F09295
:1063E000E502E092E402040F151FF5E0169507950B
:1063F000FA95E1F71093D9020093D8029093E30243
:106400008093E2023093E1022093E00252E075169D
:1064100009F051C08091D4089091D50897FF03C02E
:10642000909581959F4F6CE070E00E9489709B0170
:106430007093DF026093DE028091E6089091E70896
:1064400097FF03C0909581959F4F6CE070E00E948C
:1064500089707093DD026093DC02B90184E090E002
:106460000E949D266091DC027091DD0286E090E042
:106470000E949D266091D8027091D90288E090E038
:106480000E949D266091E8027091E90282E190E00D
:106490000E949D266091E6027091E70284E190E0FF
:1064A0000E949D266091E4027091E50286E190E0F1
:1064B0000E949D269CC084E090E00E9498269093C4
:1064C000DF028093DE0286E090E00E9498269C0125
:1064D0009093DD028093DC028091DE029091DF02D6
:1064E0008150984018F421503840A0F181E697E09F
:1064F0009F938F938EED91E19F938F93E09189030A
:10650000F0918A0309958091D4089091D50897FF5E
:1065100003C0909581959F4F6CE070E00E94897058
:106520007093DF026093DE028091E6089091E708A5
:1065300097FF03C0909581959F4F6CE070E00E949B
:1065400089707093DD026093DC0266240F900F90D7
:106550000F900F908091590281FF49C082E190E035
:106560000E9498268C0184E190E00E949826EC011C
:1065700086E190E00E9498269C01C80180509941D4
:1065800081589C4080F455E2C138D50760F489E118
:10659000C030D80740F044E0213B340720F453E0FA
:1065A00020323507C0F489E797E09F938F938EEDF3
:1065B00091E19F938F93E0918903F0918A0309956C
:1065C0006624809159028D7F809359020F900F901D
:1065D0000F900F900CC01093E9020093E802D09343
:1065E000E702C093E6023093E5022093E40212BC76
:1065F00011BC10929C0810929B0810929108109266
:1066000090081092DC081092DB0888EC90E00E9461
:10661000D61580910A0290910B029C01220F331F24
:10662000220F331F280F391F280F391F3093D50829
:106630002093D40880910C0290910D028C01000FE0
:10664000111F000F111F080F191F080F191F10939A
:10665000E7080093E60880914906C82EDD24EE2461
:10666000FF24442737FD4095542FC701B6010E94EF
:106670004A704B015C016093D2027093D302809305
:10668000D4029093D5029801442737FD4095542FAA
:10669000C701B6010E944A70DC01CB018093CE0293
:1066A0009093CF02A093D002B093D1028092C60201
:1066B0009092C702A092C802B092C9028093C2020F
:1066C0009093C302A093C402B093C5021092BE027D
:1066D0001092BF021092C0021092C10200918F016D
:1066E000109190011093AD020093AC0284E690E00B
:1066F00090938C0180938B0180916E069927AA2735
:10670000BB27BC01CD0124EC39E040E050E00E9401
:106710004A70DC01CB018856954CAF4FBF4F809338
:10672000870190938801A0938901B0938A01809199
:106730006F069927AA27BB27BC01CD010E944A708A
:10674000DC01CB018856954CAF4FBF4F809383013E
:1067500090938401A0938501B09386011092460125
:1067600010924501C801AA2797FDA095BA2F209144
:106770004101309142014091430150914401BC01DB
:10678000CD010E944A70DC01CB018093E208909316
:10679000E308A093E408B093E5081092A9021092D0
:1067A000A8020E94AB61772029F080915B0284608F
:1067B00080935B028FEF809362091092630980E2FD
:1067C0008093640984E6809394028091E501882394
:1067D00011F0579A17C08091A606992780FF05C02F
:1067E00082FF03C080EE9EE202C080E091E19093C0
:1067F0000A018093090181E0809311010E947716BC
:106800000E94771688E090E00E9498269093D90223
:106810008093D80212BC11BC8091E8029091E902E9
:1068200080569940815C9B4228F08091A203816050
:106830008093A2038091E6029091E70280569940EE
:10684000815C9B4228F08091A20382608093A20326
:106850008091E4029091E5028C52914089579540D5
:1068600028F08091A20384608093A2038091DE02CD
:106870009091DF028C529140835C914028F080918E
:10688000A20388608093A2038091DC029091DD02D4
:106890008C529140835C914028F08091A2038061EA
:1068A0008093A2038091D8029091D90280509240A7
:1068B0008355914028F08091A20380628093A203C7
:1068C0008091A2038111662486E480937E018091E9
:1068D0001B0190911C01A0911D01B0911E0180939C
:1068E000CF059093D005A093D105B093D205109217
:1068F00002021092010210920402109205021092FC
:106900000602109207021092AE021092AF0210928D
:10691000B0021092B1021092C1051092C0050E94FF
:10692000DF198091590281FF07C080917106882389
:1069300019F484E080937106862D9927EEE0CDB797
:10694000DEB70C94F970A3E1B0E0E9EAF4E30C944B
:10695000D9708091E4029091E50220910E0230916D
:106960000F02821B930B9093DC088093DB088091CD
:1069700018029091190297FD07969C0183E03595C6
:1069800027958A95E1F730939C0820939B08809186
:1069900016029091170297FD079603E0959587954B
:1069A0000A95E1F790939108809390083093A4089A
:1069B0002093A30890939F0880939E088091D40809
:1069C0009091D508AC01440F551F480F591F2091D5
:1069D0000A0230910B02C901880F991F880F991F75
:1069E000820F931F820F931F480F591F57FF02C03A
:1069F0004D5F5F4F55954795559547955093D508F1
:106A00004093D4088091E6089091E708AC01440FC8
:106A1000551F480F591F20910C0230910D02C901DA
:106A2000880F991F880F991F820F931F820F931F42
:106A3000480F591F57FF02C04D5F5F4F559547954F
:106A4000559547955093E7084093E6088091AD0827
:106A50009091AE0820910A0230910B02820F931F91
:106A60009093AE088093AD088091DE089091DF0886
:106A700020910C0230910D02820F931F9093DF083A
:106A80008093DE088091DA029091DB020196909368
:106A9000DB028093DA028091F3019091F401A091DE
:106AA000F501B091F60180938E0290938F02A0932E
:106AB0009002B09391028093F7019093F801A09314
:106AC000F901B093FA018FEC80937A0010921501CE
:106AD0002091C2023091C3024091C4025091C5027C
:106AE00029873A874B875C8729543B464140504071
:106AF0002CF028E43BE641E050E00DC089859A8502
:106B0000AB85BC85885B9449AE4FBF4F4CF428EBF6
:106B100034E94EEF5FEF2D833E834F83588708C0E3
:106B200089859A85AB85BC858D839E83AF83B88725
:106B30002091C6023091C7024091C8025091C9020B
:106B40002D873E874F87588B29543B464140504004
:106B50002CF028E43BE641E050E00DC08D859E8599
:106B6000AF85B889885B9449AE4FBF4F4CF428EB92
:106B700034E94EEF5FEF29833A834B835C8308C08F
:106B80008D859E85AF85B88989839A83AB83BC83C5
:106B9000A091DB08B091DC08BB8BAA8BFD01CF0173
:106BA000AA2797FDA095BA2FA090BE02B090BF0271
:106BB000C090C002D090C102A80EB91ECA1EDB1E32
:106BC000A092BE02B092BF02C092C002D092C10297
:106BD000E090E208F090E3080091E4081091E508E5
:106BE000E80EF91E0A1F1B1FE092E208F092E3086C
:106BF0000093E4081093E508F0917702F98BFF23E6
:106C000009F098C180917602882309F093C18091A0
:106C1000D00886FF8FC18091900890919108AA2793
:106C200097FDA095BA2FBC01CD0129813A814B81F6
:106C30005C810E944A709B01AC0197FF04C0215007
:106C4000384F4F4F5F4F6BE05595479537952795D8
:106C50006A95D1F780916801682E77248824992459
:106C6000CA01B901A40193010E944A70DC01CB0161
:106C70008093F4029093F502A093F602B093F7028A
:106C8000B7FF04C08150904FAF4FBF4F1C012D0183
:106C90003CE055944794379427943A95D1F7209245
:106CA000F4023092F5024092F6025092F70280917F
:106CB0009B0890919C08AA2797FDA095BA2FBC012C
:106CC000CD012D813E814F8158850E944A7097FFEA
:106CD00004C06150784F8F4F9F4F2BE0959587955B
:106CE000779567952A95D1F7A40193010E944A7080
:106CF000DC01CB018093F8029093F902A093FA0291
:106D0000B093FB02B7FF04C08150904FAF4FBF4F0D
:106D10009C01AD018CE055954795379527958A954F
:106D2000D1F72093F8023093F9024093FA0250937E
:106D3000FB028091F4029091F50290938A0880936F
:106D400089088091F8029091F90290938C088093C1
:106D50008B0822193309440955092093F80230930E
:106D6000F9024093FA025093FB02E20EF31E041F55
:106D7000151FE092E208F092E3080093E4081093F4
:106D8000E508809167018823B1F457FF04C02F5FA5
:106D90003F4F4F4F5F4F5595479537952795A21A0F
:106DA000B30AC40AD50AA092BE02B092BF02C09232
:106DB000C002D092C1022A893B8979010027F7FCE1
:106DC0000095102F8091F8029091F902A091FA029B
:106DD000B091FB02E80EF91E0A1F1B1FC801B70184
:106DE00029813A814B815C810E944A709B01AC01F0
:106DF00097FF04C02150384F4F4F5F4FBBE0559570
:106E0000479537952795BA95D1F780916901A82EB6
:106E1000BB24CC24DD24CA01B901A60195010E943E
:106E20004A70DC01CB018093EC029093ED02A093B9
:106E3000EE02B093EF02B7FF04C08150904FAF4F06
:106E4000BF4F3C014D01ACE09594879477946794D3
:106E5000AA95D1F76092EC027092ED028092EE0258
:106E60009092EF02C801B7012D813E814F81588574
:106E70000E944A7097FF04C06150784F8F4F9F4F18
:106E8000FBE09595879577956795FA95D1F7A601DB
:106E900095010E944A70DC01CB018093F00290932F
:106EA000F102A093F202B093F302B7FF04C0815045
:106EB000904FAF4FBF4FAC01BD01ECE075956795AA
:106EC00057954795EA95D1F74093F0025093F10218
:106ED0006093F2027093F3022A893B8937FF03C063
:106EE000309521953F4F21343105E4F1D401C301A0
:106EF00097FE07C0B095A095909581959F4FAF4F95
:106F0000BF4F81389105A105B10584F4DB01CA01A9
:106F100077FF07C0B095A095909581959F4FAF4F93
:106F2000BF4F81389105A105B105E4F081E0809360
:106F3000AA0218C010928C0810928B0810928A082E
:106F4000109289081092F0021092F1021092F2024F
:106F50001092F3021092EC021092ED021092EE02E7
:106F60001092EF028091F0029091F102A091F20252
:106F7000B091F302BC01CD0124E630E040E050E0E6
:106F80000E94BE70E090EC02F090ED02E21AF30A6B
:106F9000F0929A08E09299088091EC029091ED02AB
:106FA000A091EE02B091EF02BC01CD0124E630E0E9
:106FB00040E050E00E94BE70DA01C9012091F00269
:106FC0003091F1028C01021B130B10939308009374
:106FD00092088091410190914201A0914301B091AA
:106FE0004401BC01CD0128E631E040E050E00E94C0
:106FF0004A702091E2083091E3084091E4085091F2
:10700000E508261737074807590764F0261B370B92
:10701000480B590B2093E2083093E3084093E408AF
:107020005093E5082091E2083091E3084091E4088C
:107030005091E50857FF0CC0260F371F481F591FF6
:107040002093E2083093E3084093E4085093E50866
:1070500080919008909191088E0D9F1D20917C0247
:1070600030917D02821B930BAA2797FDA095BA2F22
:1070700029853A854B855C85820F931FA41FB51F18
:107080008093C2029093C302A093C402B093C5023E
:10709000C0908301D0908401E0908501F09086013A
:1070A000C816D906EA06FB0684F488EA91E6A0E051
:1070B000B0E08C199D09AE09BF098093C20290937C
:1070C000C302A093C402B093C50222273327A901AB
:1070D0002C193D094E095F098091C2029091C302AB
:1070E000A091C402B091C50282179307A407B50707
:1070F00084F488E59EE9AFEFBFEFC80ED91EEA1E03
:10710000FB1EC092C202D092C302E092C402F0926F
:10711000C50280919B0890919C08800F911F20913F
:107120007A0230917B02821B930BAA2797FDA095D0
:10713000BA2F2D853E854F855889820F931FA41F36
:10714000B51F8093C6029093C702A093C802B09364
:10715000C902E0908701F0908801009189011091A7
:107160008A01E816F9060A071B0784F488EA91E603
:10717000A0E0B0E08E199F09A00BB10B8093C6026E
:107180009093C702A093C802B093C9022227332765
:10719000A9012E193F09400B510B8091C602909115
:1071A000C702A091C802B091C90282179307A40731
:1071B000B50784F488E59EE9AFEFBFEFE80EF91E4E
:1071C0000A1F1B1FE092C602F092C7020093C8027A
:1071D0001093C9028091BE029091BF02A091C0029B
:1071E000B091C1028093CA029093CB02A093CC02CB
:1071F000B093CD028091C6029091C702A091C802BF
:10720000B091C9028093D2029093D302A093D4028A
:10721000B093D5028091C2029091C302A091C402A2
:10722000B091C5028093CE029093CF02A093D0027A
:10723000B093D102809121019091220197FD079690
:1072400033E0959587953A95E1F790939C08809364
:107250009B0880911F019091200197FD079623E0E4
:10726000959587952A95E1F79093910880939008DA
:1072700080911202909113020F9734F488E19CEFF1
:1072800090939C0880939B08809112029091130226
:10729000079734F480E398EF90939C0880939B08C1
:1072A0008091120290911302815D974034F088EE34
:1072B00093E090939C0880939B0880911202909198
:1072C0001302805E974034F080ED97E090939C0825
:1072D00080939B0880911002909111020F9734F4D3
:1072E00088E19CEF90939108809390088091100220
:1072F00090911102079734F480E398EF90939108EE
:10730000809390088091100290911102815D9740C6
:1073100034F088EE93E090939108809390088091E8
:10732000100290911102805E974034F080ED97E05A
:10733000909391088093900860917601662309F4F8
:10734000AFC040912101509122018091FC029091A7
:10735000FD02481B590B50930303409302032091F5
:10736000210130912201280F391F37FF02C02F5F02
:107370003F4F359527953093FD022093FC0241380D
:1073800051051CF080E890E005C040585F4F34F490
:1073900080E89FEF909303038093020340911F01C5
:1073A000509120018091FE029091FF02481B590BE1
:1073B000509301034093000320911F01309120015D
:1073C000280F391F37FF02C02F5F3F4F3595279594
:1073D0003093FF022093FE02413851051CF080E8F3
:1073E00090E005C040585F4F34F480E89FEF9093E1
:1073F000010380930003462F55278091020390914B
:107400000303849FB001859F700D949F700D11241C
:107410009B0177FF02C0215F3F4FB4E03595279570
:10742000BA95E1F780919B0890919C08820F931F79
:1074300090939C0880939B08809100039091010396
:10744000849FD001859FB00D949FB00D1124AD0194
:107450009D01B7FF02C0215F3F4FA4E035952795FE
:10746000AA95E1F78091900890919108820F931F5F
:10747000909391088093900880912101909122012E
:10748000860F971F909322018093210180911F0105
:1074900090912001840F951F9093200180931F01EC
:1074A00000919E0810919F088091890890918A0808
:1074B000101611065CF59C0197FF04C022273327A4
:1074C000281B390BC901AA2797FDA095BA2F209137
:1074D0006701332744275527BC01CD010E944A701C
:1074E0009B01AC0197FF04C0215C3F4F4F4F5F4FA2
:1074F000F6E05595479537952795FA95D1F7809100
:10750000990890919A08820F931F27C097FF03C094
:10751000909581959F4FAA2797FDA095BA2F20910E
:107520006701332744275527BC01CD010E944A70CB
:107530009B01AC0197FF04C0215C3F4F4F4F5F4F51
:10754000E6E05595479537952795EA95D1F78091CF
:10755000990890919A08821B930B90939A088093B4
:107560009908E090A308F090A40880918B0890916E
:107570008C081E141F045CF59C0197FF04C0222791
:107580003327281B390BC901AA2797FDA095BA2FCD
:1075900020916701332744275527BC01CD010E9464
:1075A0004A709B01AC0197FF04C0215C3F4F4F4FD5
:1075B0005F4F76E055954795379527957A95D1F7A2
:1075C0008091920890919308820F931F27C097FF94
:1075D00003C0909581959F4FAA2797FDA095BA2F3C
:1075E00020916701332744275527BC01CD010E9414
:1075F0004A709B01AC0197FF04C0215C3F4F4F4F85
:107600005F4F66E055954795379527956A95D1F771
:107610008091920890919308821B930B909393080A
:10762000809392088091D00887FF44C0B989BB231A
:1076300009F040C0809176028823E1F5E1E0EE1682
:10764000E1E0FE064CF080919B0890919C088E0D25
:107650009F1D805091400DC0F0E0EF16FFEFFF0638
:1076600064F480919B0890919C088E0D9F1D805022
:107670009F4F90939C0880939B0821E00130120754
:107680004CF08091900890919108800F911F80504C
:1076900091400CC03FEF0030130764F480919008D4
:1076A00090919108800F911F80509F4F9093910867
:1076B00080939008E2E1CD5E0C94F5708091930286
:1076C000882329F580915B028C7F80935B028091F7
:1076D0005A028F7D80935A02A7EAB3E0E8E4F7E00C
:1076E0009BE08091C501882309F48C938D9181835F
:1076F000128291503F9697FFF4CF8091C501882365
:1077000059F08091C50181508093C50105C08091D9
:107710005B02816080935B0280913C02882319F0B8
:1077200010923C0208958093400280913A028E7F2D
:1077300080933A0285EA8093BC000895882319F467
:1077400080E090E00895E82FFF27EE0FFF1FE35041
:10775000F84F8081918181589F4F8F3F910521F093
:107760001CF08FEF90E004C097FF02C080E090E033
:1077700099270895CF93DF93A5E9B2E0C2E3D6E05D
:1077800057E08991E82FFF27EE0FFF1FE350F84FD6
:107790000190F081E02DE158FF4FEF3FF10521F01E
:1077A0001CF0EFEFF0E004C0F7FF02C0E0E0F0E013
:1077B000893111F4EC931BC04C91242F3327E2172D
:1077C000F307A9F0CF01821B930B97FD03969595C4
:1077D000879595958795242F280F2C93822F99278D
:1077E000E817F90714F4215001C02F5F2C93515072
:1077F000119657FFC6CF80913C06883F38F0EFEFD7
:10780000F0E0E81BF109EB56FD4F808180937B018E
:1078100080917B01882329F0843618F084E68093D8
:107820007B0180913E06883F38F0EFEFF0E0E81BE7
:10783000F109EB56FD4F808180937A0180917A01A6
:10784000882329F0843618F084E680937A018091A9
:107850004B06883F38F0EFEFF0E0E81BF109EB56FC
:10786000FD4F808180937501809175018B3010F4FC
:107870008AE002C08F3F11F48093750180917806F1
:10788000883F38F0EFEFF0E0E81BF109EB56FD4FD1
:1078900080818093AF088091AF08863010F485E036
:1078A00002C08F3F11F48093AF0880917A06883F21
:1078B00038F0EFEFF0E0E81BF109EB56FD4F808167
:1078C0008093D7088091D708863010F485E002C0F5
:1078D0008F3F11F48093D70880916506873F19F494
:1078E000429905C007C0863F41F4439B03C0809185
:1078F0009A0616C080919B0613C0883F38F0EFEFC0
:10790000F0E0E81BF109EB56FD4F80818093AC0855
:107910008091AC08893110F488E102C08F3F11F4E6
:107920008093AC0880916606873F19F4429905C0A0
:1079300007C0863F41F4439B03C080919C0616C05C
:1079400080919D0613C0883F38F0EFEFF0E0E81B10
:10795000F109EB56FD4F808180938D0880918D0851
:10796000893110F488E102C08F3F11F480938D08B3
:1079700080916706883F38F0EFEFF0E0E81BF109EF
:10798000EB56FD4F80818093B5088091B508893111
:1079900010F488E102C08F3F11F48093B508809104
:1079A0003D060E949E3B8093710280914006883F75
:1079B00038F0EFEFF0E0E81BF109EB56FD4F808166
:1079C0008093790180914206883F38F0EFEFF0E034
:1079D000E81BF109EB56FD4F808180937701809180
:1079E0004A06883F38F0EFEFF0E0E81BF109EB566C
:1079F000FD4F80818093780180914C06883F38F05C
:107A0000EFEFF0E0E81BF109EB56FD4F808180932A
:107A1000740180914D06883F38F0EFEFF0E0E81BED
:107A2000F109EB56FD4F80818093760180914E06DF
:107A3000883F38F0EFEFF0E0E81BF109EB56FD4F1F
:107A400080818093730180914F06883F38F0EFEF7B
:107A5000F0E0E81BF109EB56FD4F80818093720145
:107A600080915506883F38F0EFEFF0E0E81BF10910
:107A7000EB56FD4F80818093700180915606883FC0
:107A800038F0EFEFF0E0E81BF109EB56FD4F808195
:107A90008093700280915706883F38F0EFEFF0E056
:107AA000E81BF109EB56FD4F808180936F028091B6
:107AB0005806883F38F0EFEFF0E0E81BF109EB568D
:107AC000FD4F808180936E0280915906883F38F087
:107AD000EFEFF0E0E81BF109EB56FD4F808180935A
:107AE0006D0280917306883F38F0EFEFF0E0E81BFD
:107AF000F109EB56FD4F808180936C0280917406F2
:107B0000883F38F0EFEFF0E0E81BF109EB56FD4F4E
:107B1000808180936B0280917506883F38F0EFEF8B
:107B2000F0E0E81BF109EB56FD4F808180936A027B
:107B300080917606883F38F0EFEFF0E0E81BF1091E
:107B4000EB56FD4F80818093690280915A06883FF1
:107B500038F0EFEFF0E0E81BF109EB56FD4F8081C4
:107B600080936E0180915E06883F38F0EFEFF0E081
:107B7000E81BF109EB56FD4F808180936D018091E8
:107B80005B06883F38F0EFEFF0E0E81BF109EB56B9
:107B9000FD4F808180936C0180915F06883F38F0B3
:107BA000EFEFF0E0E81BF109EB56FD4F8081809389
:107BB0006B0180916806883F38F0EFEFF0E0E81B3A
:107BC000F109EB56FD4F808180936A0180916B062D
:107BD000883F38F0EFEFF0E0E81BF109EB56FD4F7E
:107BE00080818093690180916C06883F38F0EFEFC7
:107BF000F0E0E81BF109EB56FD4F808180936801AE
:107C000080916D06883F38F0EFEFF0E0E81BF10956
:107C1000EB56FD4F80818093670180919606883FE7
:107C200038F0EFEFF0E0E81BF109EB56FD4F8081F3
:107C30008093980880913A068093D0088091A70697
:107C40008093B40880917206883F38F0EFEFF0E03F
:107C5000E81BF109EB56FD4F80818093660180910E
:107C60008F06883F38F0EFEFF0E0E81BF109EB56A4
:107C7000FD4F80818093E90880917001282F332780
:107C80002F5F3F4F8CE398E2B9010E948970709397
:107C90007D0160937C01809148068093D808809193
:107CA00047068093A008E0919106EE23D9F181E088
:107CB00080936802FF27EE0FFF1FE350F84F80818B
:107CC0009181805C9F4F14F41092680280917E0134
:107CD000209168028217B1F0833088F4222319F0D2
:107CE0008CED95E002C088EC90E09093E8018093E1
:107CF000E70185E080937E0220937E0103C08150DE
:107D000080937E018091290990912A0997FF0FC0E5
:107D100080916802882359F08091A2038068809343
:107D2000A20305C0E09368028AE080937E018091FF
:107D3000290990912A0997FF1DC0809193028823F9
:107D4000C9F0809168028823A9F080910B0190917D
:107D50000C018F5F9F4F71F488E99AE39093E801DB
:107D60008093E70180E094EA90930C0180930B01EB
:107D70001092680280916802882321F080915A0253
:107D8000816003C080915A028E7F80935A02DF91F6
:107D9000CF91089580914306882301F56091780280
:107DA0007091790277FF02C06D5F7F4F759567957F
:107DB00075956795409123015091240180910201AE
:107DC000282F3327649FC001659F900D749F900DED
:107DD0001124B9010E947570CB0101C099279093BD
:107DE0008201809381018091810190918201873489
:107DF000910538F486E490E09093820180938101AC
:107E000008958F3A910530F08FEA90E090938201C7
:107E1000809381010895ABE0B0E0E1E1FFE30C94D1
:107E2000D9700E94A33480915B029927847190706D
:107E3000892B91F58091A80682FF27C08091780256
:107E4000909179020097F1F022E088359207D4F4FE
:107E50009C0197FF02C02D5F3F4F359527953595C3
:107E60002795809152069927289FA001299F500DA0
:107E7000389F500D1124CA0164E670E00E94897099
:107E8000CB0106C08DE290E003C080915206992795
:107E900090935802809357022091550230915602D8
:107EA00055E72033350759F410929F0210929E0235
:107EB0008091A0089927909358028093570260916F
:107EC0009E0270919F027A8369838091A00899270E
:107ED0000A966817790714F49A838983809194022B
:107EE0008436B0F580915A0282FD32C08091100331
:107EF00090911103009731F00197909311038093B3
:107F000010030BC01092930290935D0280935C0269
:107F100080915B028D7E80935B02289A80915C0247
:107F200090915D02895E934080F08091780985365A
:107F300060F080915702909158029A8389838091D2
:107F40005B02806180935B02B0C410929302ADC467
:107F5000809194028D3808F47EC480915B028F7EFC
:107F600080935B029091530682E3989FC001112495
:107F70009093110380931003A981BA8199978CF093
:107F800080919302882369F080915C0290915D0258
:107F9000BFEF8F3F9B0729F0019690935D0280937E
:107FA0005C0220915C0230915D022F3F310509F0A7
:107FB00030F51092B6021092B7021092B8021092E9
:107FC000B9021092B2021092B3021092B40210924F
:107FD000B50210920403109205031092060310924A
:107FE00007031092BE021092BF021092C0021092BC
:107FF000C10280915A02806280935A024DC08091E2
:108000005B02826080935B0280915A0285FF44C0CC
:108010008091F7019091F801A091F901B091FA01D6
:1080200087399105A105B1058CF480918E0290915C
:108030008F02A0919002B0919102825A9E4FAF4F51
:10804000BF4F24F08091D00880FD05C080915A0276
:108050008F7180935A021092B6021092B70210925A
:10806000B8021092B9021092B2021092B3021092AA
:10807000B4021092B5021092BE021092BF0210928A
:10808000C0021092C102295E334030F088EE93E0C6
:1080900090935D0280935C0280913006E82FFF2769
:1080A000EE0FFF1FE350F84F8081918181359105DC
:1080B0000CF483C120919302222309F07EC18091A8
:1080C0003E039927AC014071507084FD76C18091C8
:1080D0003106E82FFF27EE0FFF1FE350F84F808196
:1080E00091810190F081E02DF7FF03C0F095E195BB
:1080F000FF4FEC34F1050CF45EC1809112038F5FE9
:1081000080931203893C08F458C1122F2093120364
:1081100050935D0240935C0230912E06E32FFF27BF
:10812000EE0FFF1FE350F84F808191818734910556
:10813000B4F480912F06E82FFF27EE0FFF1FE350C6
:10814000F84F808191810190F081E02DF7FF03C00D
:10815000F095E195FF4FE734F1050CF48DC02091C7
:108160002F06E22FFF27EE0FFF1FE350F84F80810D
:108170009181873491058CF0E32FFF27EE0FFF1FCD
:10818000E350F84F808191818634910534F48081E9
:1081900091818B5B9F4F0CF011E0E22FFF27EE0FD8
:1081A000FF1FE350F84F808191818734910574F06F
:1081B00080912E06E82FFF27EE0FFF1FE350F84FA8
:1081C00080819181873491050CF012E0E22FFF2726
:1081D000EE0FFF1FE350F84F8081918186349105A7
:1081E00074F480912E06E82FFF27EE0FFF1FE35057
:1081F000F84F80819181873491050CF013E0E22FD4
:10820000FF27EE0FFF1FE350F84F808191818A5BBB
:108210009F4F74F480912E06E82FFF27EE0FFF1F6B
:10822000E350F84F80819181873491050CF014E080
:10823000E22FFF27EE0FFF1FE350F84F808191815F
:108240008A5B9F4FA4F480912E06E82FFF27EE0F44
:10825000FF1FE350F84F80819181863491053CF4F3
:10826000808191818B5B9F4F14F015E002C0112338
:1082700019F0812F0E94F52680912F06E82FFF2705
:10828000EE0FFF1FE350F84F808191810190F08144
:10829000E02DF7FF03C0F095E195FF4F7E97CCF4FA
:1082A00080912E06E82FFF27EE0FFF1FE350F84FB7
:1082B000808191818A5B9F4F64F481E08093BD034C
:1082C00010927F0288EE93E09093E8018093E7019B
:1082D00074C0809101010E94A22680E00E944A059C
:1082E000809154060E94466C8091D00880FF10C097
:1082F0008091190190911A01875B934038F4809125
:10830000190190911A018E5E924010F40E94171A82
:10831000112309F040C080912F06E82FFF27EE0FB0
:10832000FF1FE350F84F808191818A5B9F4F7CF45F
:1083300080912E06E82FFF27EE0FFF1FE350F84F26
:10834000808191818634910514F483E025C0809169
:108350003106E82FFF27EE0FFF1FE350F84F808113
:108360009181855B9F4FBCF480912E06E82FFF27FB
:10837000EE0FFF1FE350F84F808191810190F08153
:10838000E02DF7FF03C0F095E195FF4FE634F105CE
:1083900014F482E001C081E00E94313180937F02B9
:1083A00081E08093E501579A68E770E080910101D0
:1083B0000E947C3002C02093120380913006E82F87
:1083C000FF27EE0FFF1FE350F84F808191818C59FA
:1083D0009F4F0CF039C220919206E22FFF27EF77D2
:1083E000F070EE0FFF1FED5BF74F808191810697D4
:1083F00014F084E606C0808191818B5F9F4F1CF44E
:108400008CE98093150380919302E09131068823D3
:1084100009F068C1FF27EE0FFF1FE350F84F80817E
:1084200091818C599F4F9CF48091A80683FD0BC0CD
:10843000E22FFF27EE0FFF1FE350F84F808191815D
:10844000855B9F4FDCF0809192068823B9F0809184
:10845000A80683FF44C180919206E82FFF27EE0F04
:10846000FF1FE350F84F80819181875F9F4F0CF48D
:1084700036C180911503843609F031C180913E03E5
:1084800084FD2DC180917F02882329F080915B02B9
:10849000886080935B0280911B0190911C01A091E8
:1084A0001D01B0911E018093CF059093D005A0933C
:1084B000D105B093D20510928E0210928F021092C5
:1084C0009002109291021092F3011092F401109216
:1084D000F5011092F60188E592E0909356028093A0
:1084E0005502109204021092050210920602109298
:1084F000070280912E06E82FFF27EE0FFF1FE350A3
:10850000F84F808191818D599F4FACF480912F0657
:10851000E82FFF27EE0FFF1FE350F84F8081918176
:108520000190F081E02DF7FF03C0F095E195FF4F3A
:10853000E436F10534F480919206882311F4809397
:108540001303809113038F5F809313038E3F08F40E
:108550005EC1809159022091DB083091DC0881FFD7
:1085600021C0C90137FF04C088279927821B930BBC
:1085700081349105ACF580919B0890919C0897FF00
:1085800003C0909581959F4FCD9754F580919008A9
:108590009091910897FF03C0909581959F4FCD973B
:1085A0000CF11EC0C90137FF03C0909581959F4F04
:1085B0008197B4F480919B0890919C0897FF03C029
:1085C000909581959F4F45975CF48091900890918C
:1085D000910897FF03C0909581959F4F459714F0A0
:1085E00010927F02109213038091A203882309F056
:1085F00073C080917F02882309F46EC0809142038A
:10860000882309F069C081E090E090935D02809337
:108610005C0281E0809393021092040310920503A0
:1086200010920603109207031092BE021092BF022E
:108630001092C0021092C1021092BA021092BB02B4
:108640001092BC021092BD0280914906E82EFF24D0
:10865000002711278091D4089091D5089C014427C8
:1086600037FD4095542FC801B7010E944A70DC01C4
:10867000CB018093C6029093C702A093C802B09327
:10868000C9028091E6089091E7089C01442737FDD4
:108690004095542FC801B7010E944A70DC01CB01FC
:1086A0008093C2029093C302A093C402B093C50208
:1086B0001092B6021092B7021092B8021092B9024C
:1086C0001092B2021092B3021092B4021092B5024C
:1086D00084E680937E029BC08CED95E091C0109261
:1086E000130395C0FF27EE0FFF1FE350F84F808163
:1086F0009181853691059CF08091A80683FD0BC081
:10870000E22FFF27EE0FFF1FE350F84F808191818A
:10871000855B9F4FDCF0809192068823B9F08091B1
:10872000A80683FF72C080919206E82FFF27EE0F04
:10873000FF1FE350F84F808191818E5C9F4F0CF0BA
:1087400064C0809115038C3909F05FC080912E06BA
:10875000E82FFF27EE0FFF1FE350F84F8081918134
:108760008D599F4FACF480912F06E82FFF27EE0F15
:10877000FF1FE350F84F808191810190F081E02D3F
:10878000F7FF03C0F095E195FF4FE436F1053CF4A7
:1087900080919206882319F48093140318C01092D4
:1087A000B6021092B7021092B8021092B90210925B
:1087B000B2021092B3021092B4021092B50210925B
:1087C000A5021092A4021092A3021092A20280911C
:1087D00014038F5F809314038B3F70F01092930209
:1087E0001092140310925D0210925C0280915A0262
:1087F0008F7180935A020BC0843649F48CEA9DE055
:108800009093E8018093E70102C010921403209135
:10881000550230915602F3E0283E3F0708F045C06C
:1088200080910102909102028B569F4F1CF02F5FA6
:108830003F4F05C021153105C1F121503040309323
:1088400056022093550231C0109215031092560221
:10885000109255022AC02E5E324038F18091F10804
:108860009091F2088059914000F580918E0290918C
:108870008F02A0919002B09191028C5D9540A04032
:10888000B0409CF480E395E79093560280935502A4
:1088900080915C0290915D028A5E934030F089EE97
:1088A00093E090935D0280935C0280913F01815040
:1088B00080933F0180913F018F3F21F080915B02C7
:1088C00084FFDFC30E94BA3BA09044068091160348
:1088D000909117039C01220F331F280F391FB0906E
:1088E0002E06AB2DBB27AA0FBB1FFD01E350F84F8F
:1088F0004A2D552780819181849FF001859FF00D3D
:10890000949FF00D11242E0F3F1F37FF02C02D5FE3
:108910003F4FB9017595679575956795AD5BB74FF5
:1089200080914506082F11278D919C91809F900181
:10893000819F300D909F300D1124620F731F709333
:1089400017036093160380911803909119039C01FB
:10895000220F331F280F391FE0902F06AE2DBB27A3
:10896000AA0FBB1FFD01E350F84F80819181849FC6
:10897000F001859FF00D949FF00D11242E0F3F1FE5
:1089800037FF02C02D5F3F4FA9015595479555957B
:108990004795AD5BB74F8D919C91809F9001819FD2
:1089A000300D909F300D1124420F531F5093190327
:1089B0004093180380916802882309F448C0CB01D2
:1089C00077FD0396DC01B595A795B595A795CA01E6
:1089D00057FD0396FC01F595E795F595E795809190
:1089E000A101682F772767FD70956A9F90016B9FA3
:1089F000300D7A9F300D112480914503482F552763
:108A000047FD50954E9FC0014F9F900D5E9F900D6A
:108A10001124280F391F37FF02C0295F3F4F03E0A1
:108A2000359527950A95E1F73093A5022093A40286
:108A30006E9F90016F9F300D7E9F300D11244A9FD5
:108A4000C0014B9F900D5A9F900D11243FC0809103
:108A50009006E82FFF27E95BFE4F86818093A101F6
:108A6000908190934503A82FBB27A7FDB095A69FA3
:108A70009001A79F300DB69F300D1124E92FFF27DD
:108A8000E7FDF095E49FC001E59F900DF49F900DE8
:108A90001124280F391F37FF02C0295F3F4F13E011
:108AA000359527951A95E1F73093A5022093A402F6
:108AB000A49F9001A59F300DB49F300D1124E69F17
:108AC000C001E79F900DF69F900D1124281B390BD4
:108AD00037FF02C0295F3F4F73E0359527957A95A0
:108AE000E1F73093A3022093A20280913106E82F90
:108AF000FF27EE0FFF1FE350F84F80819181909583
:108B000081959F4F9093A1028093A002853091059B
:108B100014F0049705C03FEF8C3F930734F404969C
:108B20009093A1028093A00204C01092A10210921F
:108B3000A00280915502909156028150924078F1A6
:108B40008091A4029091A50297FD079663E0959508
:108B500087956A95E1F79093A5028093A40280918E
:108B6000A2029091A30297FD079653E095958795F1
:108B70005A95E1F79093A3028093A2021092B60255
:108B80001092B7021092B8021092B9021092B2027B
:108B90001092B3021092B4021092B50243C08091B9
:108BA0003103882309F43EC0282F33278091A40283
:108BB0009091A50297FD079643E0959587954A9574
:108BC000E1F7289FB001299F700D389F700D112487
:108BD000CB0177FD0F9604E0959587950A95E1F70F
:108BE0009093A5028093A4028091A2029091A30287
:108BF00097FD079613E0959587951A95E1F7289FBD
:108C0000D001299FB00D389FB00D1124CD01B7FDC3
:108C10000F96B4E095958795BA95E1F79093A302E6
:108C20008093A2028090A4029090A50280913403C8
:108C300090913503881A990A9092A5028092A40215
:108C40000091A2021091A30280913203909133030C
:108C5000081B190B1093A3020093A2028091300607
:108C6000E82FFF27EE0FFF1FE350F84FC080D180A1
:108C7000EFE7F0E0CE0EDF1ED0929F02C0929E0280
:108C8000809175019927AA2797FDA095BA2FBC015D
:108C9000CD010E94BE6FDC01CB0120E030E040E25C
:108CA00051E4BC01CD010E942C6FDC01CB01BC0161
:108CB000CD010E94906FDC01CB018093E008809190
:108CC00074018093B608809173019927AA2797FDB4
:108CD000A095BA2FBC01CD010E94BE6FDC01CB0173
:108CE00020E030E040E251E4BC01CD010E942C6F55
:108CF000DC01CB01BC01CD010E94906FDC01CB01F6
:108D000080939708809172018093A5088091C90390
:108D100080FF59C08091E908813808F454C08091DF
:108D2000C203992787FD90952A2D3327829FA001A2
:108D3000839F500D929F500D1124840E951E90928A
:108D4000A5028092A4028091C303992787FD909584
:108D5000829FB001839F700D929F700D1124060FAA
:108D6000171F1093A3020093A2028091C403282F1F
:108D7000332727FD30958091A0029091A102820FA8
:108D8000931F9093A1028093A0028091C603282F85
:108D9000332727FD309580913F069927289FD001E2
:108DA000299FB00D389FB00D1124B0934601A093B8
:108DB00045018091C50399278C159D0524F4909356
:108DC0009F0280939E0280919E0290919F0297FF46
:108DD00004C010929F0210929E028091D00882FFE0
:108DE00002C01092B6084091A4025091A502CA0197
:108DF00057FD03969C01359527953595279537FFA7
:108E000003C0309521953F4F80916002909161029F
:108E100082179307B4F4CA0157FF03C09095819558
:108E20009F4F97FD03969595879595958795909378
:108E30006102809360028536910544F084E690E0FB
:108E400001C0019790936102809360024091A20259
:108E50005091A302CA0157FD03969C0135952795B1
:108E60003595279537FF03C0309521953F4F809169
:108E70005E0290915F0282179307B4F4CA0157FF14
:108E800003C0909581959F4F97FD03969595879583
:108E90009595879590935F0280935E028536910544
:108EA00044F084E690E001C0019790935F028093C4
:108EB0005E0280915B0284FF08C0109261021092F2
:108EC000600210925F0210925E02EE2DFF27EE0FFD
:108ED000FF1FE350F84F40916906242F332780810C
:108EE00091812817390744F48091A50682FF04C0B8
:108EF00081E08093750213C0EE2DFF27EE0FFF1F58
:108F0000E350F84F842F992720916A06821B91091C
:108F1000208131812817390714F41092750240918D
:108F20002F06E42FFF27EE0FFF1FE350F84F50915D
:108F30006906852F992722273327281B390B808123
:108F400091818217930744F48091A50683FF04C0A2
:108F500081E08093740216C080917402882391F09E
:108F6000E42FFF27EE0FFF1FE350F84F80916A06B2
:108F70009927851B9109208131818217930714F469
:108F800010927402EB2DFF27EE0FFF1FE350F84FF6
:108F900040916906242F3327808191812817390752
:108FA00044F48091A50680FF04C081E080937202A2
:108FB00017C080917202882399F0EB2DFF27EE0FE6
:108FC000FF1FE350F84F842F992720916A06821BD8
:108FD0009109208131812817390714F41092720207
:108FE00040912E06E42FFF27EE0FFF1FE350F84FAE
:108FF00050916906852F992722273327281B390B83
:10900000808191818217930744F48091A50681FFA6
:1090100004C081E08093730216C08091730288239C
:1090200091F0E42FFF27EE0FFF1FE350F84F8091E0
:109030006A069927851B9109208131818217930740
:1090400014F41092730280917502882319F48091B0
:109050007402811181E080937602809172028823EC
:1090600021F480917302882351F081E0809377028C
:1090700010927602109275021092740202C08093D0
:10908000770280917602882321F4809177028823E9
:1090900069F0809168069927E981FA818E179F0708
:1090A00014F49A83898381E08093AA0280915A0202
:1090B00099279C012470307082FF31C08091340365
:1090C00090913503909581959F4F9093A502809341
:1090D000A4028091320390913303909581959F4F24
:1090E0009093A3028093A2028091810190918201CA
:1090F00090939F0280939E021092A1021092A00270
:109100008091D0088B778B668093D0088091B408CB
:109110008C7B8093B40888EC809371021EC0809190
:109120005B0284FF1AC03093A1022093A002309307
:10913000A5022093A4023093A3022093A2029AE5F1
:109140009093E00888E78093B608909397088093FF
:10915000A50810927602109277028091A80890914B
:10916000A908A091AA08B091AB082091D202309131
:10917000D3024091D4025091D502820F931FA41FB5
:10918000B51F8093A8089093A908A093AA08B0934C
:10919000AB088091B0089091B108A091B208B0914D
:1091A000B3082090CE023090CF024090D002509071
:1091B000D102820D931DA41DB51D8093B00890931C
:1091C000B108A093B208B093B308F0917702FB8383
:1091D000FF2321F480917602882301F11092A808E0
:1091E0001092A9081092AA081092AB081092B00829
:1091F0001092B1081092B2081092B30810920002B7
:109200001092FF0110927B0210927A0210927D025E
:1092100010927C026B81662309F0ECC1809176028A
:10922000882309F0E7C18091CD059091CE0581504A
:1092300092402CF480919302882309F4DBC1909032
:109240006209A09049068091D4089091D5089B8727
:109250008A87A091E608B091E708B987A887191412
:109260000CF0BDC0BB24CC24DD24CA01B901A60189
:1092700095010E94BE7079018A0180912B0990911D
:109280002C09EA85FB85E81BF90BCF01AA2797FD7E
:10929000A095BA2FE81AF90A0A0B1B0BC201B101FB
:1092A000A60195010E94BE7059016A0180912D09A5
:1092B00090912E0928853985281B390BC901AA27C9
:1092C00097FDA095BA2FA81AB90ACA0ADB0A292C59
:1092D000332427FC3094432C532CC801B701A2013E
:1092E00091010E944A7097FF04C061507E4F8F4FDA
:1092F0009F4F3B014C0169E0959487947794679464
:109300006A95D1F7C601B501A20191010E944A7088
:1093100097FF04C061507E4F8F4F9F4F5B016C01E0
:1093200059E0D594C794B794A7945A95D1F78091F2
:10933000600290916102813491053CF480915E025B
:1093400090915F0281349105D4F0D401C30197FE5E
:1093500003C00196A11DB11D3C014D019594879458
:1093600077946794D601C501D7FE03C00196A11D6D
:10937000B11D5C016D01D594C794B794A7948091F9
:109380006409282F332727FD3095432F532F2615A7
:1093900037054805590514F439014A01992787FD15
:1093A0009095909581959F4FAA2797FDA095BA2FEC
:1093B000681679068A069B0614F43C014D012A15AD
:1093C0003B054C055D0514F459016A01A816B90660
:1093D000CA06DB060CF0D2C05C016D01CFC0EA2CDE
:1093E000FF2400271127CA01B901A80197010E9493
:1093F000BE7039014A014A855B85CA01AA2797FDDB
:10940000A095BA2F681A790A8A0A9B0AC201B1018B
:10941000A80197010E94BE7059016A01688579858B
:10942000CB01AA2797FDA095BA2FA81AB90ACA0A94
:10943000DB0AD401C30197FE03C00F96A11DB11D25
:109440003C014D0124E095948794779467942A9584
:10945000D1F7D601C501D7FE03C00F96A11DB11DDE
:109460005C016D0194E0D594C794B794A7949A9544
:10947000D1F78091600290916102813491053CF4B2
:1094800080915E0290915F0281349105A4F0C40145
:10949000B30123E030E040E050E00E94BE703901AB
:1094A0004A01C601B50123E030E040E050E00E94EF
:1094B000BE7059016A0180913106E82FFF27EE0F37
:1094C000FF1FE350F84F808191810190F081E02DE2
:1094D000F7FF03C0F095E195FF4F7A97A4F0C40120
:1094E000B30123E030E040E050E00E94BE7039015B
:1094F0004A01C601B50123E030E040E050E00E949F
:10950000BE7059016A0189E180938D0171E267168D
:109510007104810491042CF080E2682E712C812C5E
:10952000912C80EE68168FEF78068FEF88068FEF0C
:10953000980644F400EE602E0FEF702E0FEF802E91
:109540000FEF902E91E2A916B104C104D1042CF0C2
:1095500010E2A12EB12CC12CD12CA0EEAA16AFEF97
:10956000BA06AFEFCA06AFEFDA0644F4B0EEAB2EA0
:10957000BFEFBB2EBFEFCB2EBFEFDB2E8091C6021D
:109580009091C702A091C802B091C90286199709AB
:10959000A809B9098093C6029093C702A093C80294
:1095A000B093C9028091C2029091C302A091C402FB
:1095B000B091C5028A199B09AC09BD098093C2020A
:1095C0009093C302A093C402B093C50280914E024F
:1095D00090914F02860D971D90934F0280934E02FB
:1095E00080914C0290914D028A0D9B1D90934D02EB
:1095F00080934C028091FF01909100028F3F910572
:1096000009F008F461C120917106222309F40EC10A
:109610008091D4089091D508815E9C4F8F539640DD
:1096200008F004C18091E6089091E708815E9C4FA4
:109630008F53964008F0FAC08091AA02882309F05F
:10964000F5C08091DB089091DC084F96CF9708F029
:10965000EDC0822F99279093A9058093A805FC015E
:10966000A6E0EE0FFF1FAA95E1F720914E02309180
:109670004F02C901BF010E947570261B370B309342
:109680004F0220934E0220914C0230914D02C901AD
:10969000BF010E947570261B370B30934D0220933B
:1096A0004C022091A8023091A902C901BF010E9479
:1096B0007570261B370B3093A9022093A802809166
:1096C00060029091610281349105DCF480915E0228
:1096D00090915F0281349105A4F480913106E82FC6
:1096E000FF27EE0FFF1FE350F84F8081918101901B
:1096F000F081E02DF7FF03C0F095E195FF4F7A97D9
:10970000E4F080914E0290914F0297FD019695955D
:10971000879590934F0280934E0280914C029091D6
:109720004D0297FD01969595879590934D028093F4
:109730004C021092A9021092A80280914E029091C0
:109740004F02895B9B406CF010924F0210924E02C8
:109750008091E8029091E90201969093E90280934A
:10976000E80280914E0290914F028854944F6CF41D
:1097700010924F0210924E028091E8029091E902FD
:1097800001979093E9028093E80280914C029091B6
:109790004D02895B9B406CF010924D0210924C027E
:1097A0008091E6029091E70201969093E702809300
:1097B000E60280914C0290914D028854944F6CF4D3
:1097C00010924D0210924C028091E6029091E702B5
:1097D00001979093E7028093E6028091A80290910E
:1097E000A9028D5A9D406CF01092A9021092A80215
:1097F0008091E4029091E50201969093E5028093B6
:10980000E4028091A8029091A9028455924FD4F469
:109810001092A9021092A8028091E4029091E502B0
:1098200001979093E5028093E4020CC010924F02DE
:1098300010924E0210924D0210924C021092A90208
:109840001092A8021092AA028091B608882341F4CF
:1098500010927D0210927C0210927B0210927A028A
:109860008091A8089091A908A091AA08B091AB088E
:1098700080931A0390931B03A0931C03B0931D03C2
:109880008091B0089091B108A091B208B091B3084E
:1098900080931E0390931F03A0932003B093210392
:1098A0001092A8081092A9081092AA081092AB086A
:1098B0001092B0081092B1081092B2081092B3083A
:1098C000109200021092FF018090A0029090A102DD
:1098D000C40197FE04C0882799278819990904971D
:1098E0003CF08091D00884FD03C082E380937E0227
:1098F00010914606A12EBB24CC24DD24B401882778
:1099000077FD8095982F940197FE04C02227332776
:1099100028193909442737FD4095542F0E944A7071
:109920009B01AC01C601B5010E944A7097FF04C0BB
:1099300061507E4F8F4F9F4F59E095958795779552
:1099400067955A95D1F79B01812F9927889DD00162
:10995000899DB00D989DB00D1124CD01B7FD0396E2
:109960009595879595958795280F391F8091550274
:10997000909156028150924010F020E030E08091AA
:10998000800290918102820F931F9C01442737FD32
:109990004095542F2093040330930503409306030E
:1099A000509307038091BE029091BF02A091C00224
:1099B000B091C102821B930BA40BB50B8093BE0226
:1099C0009093BF02A093C002B093C1028155934C03
:1099D000A040B04064F080E593ECA0E0B0E080935C
:1099E000BE029093BF02A093C002B093C1028091C7
:1099F000BE029091BF02A091C002B091C102805BF3
:109A00009C43AF4FBF4F64F480EB9CE3AFEFBFEFDD
:109A10008093BE029093BF02A093C002B093C10294
:109A200080908F019090900197FCFAC08091D008AF
:109A300083FFF6C080918E01815080938E01882330
:109A400009F0F2C08DE080938E018091D202909156
:109A5000D302A091D402B091D502B7FF04C08150C7
:109A60009E4FAF4FBF4F39E0B595A7959795879516
:109A70003A95D1F78C0197FF03C0109501951F4FC0
:109A80008091CE029091CF02A091D002B091D102EC
:109A9000B7FF04C081509E4FAF4FBF4F29E0B5952F
:109AA000A795979587952A95D1F79C0197FF03C0B5
:109AB000309521953F4F021713070CF48901B80127
:109AC00017FF02C0695F7F4F3B01A3E07594679465
:109AD000AA95E1F722E030E0620E731EA090E20842
:109AE000B090E308C090E408D090E50820914101CF
:109AF000309142014091430150914401C601B501AA
:109B00000E94BE7019012A0130939608209395088F
:109B1000821A930AC401845E9D4F68E671E00E9438
:109B20008970AC01445B504020917E02222321F0D9
:109B30003092AD022092AC0280918B0190918C0109
:109B4000009731F0019790938C0180938B0112C0A4
:109B5000093111057CF48091A8029091A902840F2B
:109B6000951F9093A9028093A802222319F02150F7
:109B700020937E0280918B0190918C01892BF9F4C6
:109B800080918D019927489FB001499F700D589F82
:109B9000700D1124CB01B3010E948970CB01AA275B
:109BA00097FDA095BA2FA80EB91ECA1EDB1EA09263
:109BB000E208B092E308C092E408D092E5088091F0
:109BC0007E02882369F58091AC029091AD022091CC
:109BD000950830919608821B930B845E9D4F68E632
:109BE00071E00E9489709C01245B30408091780173
:109BF00086959927289FD001299FB00D389FB00DD9
:109C000011249D01B7FF02C0215F3F4FF4E035955D
:109C10002795FA95E1F7309381022093800204C0E2
:109C200010928102109280028091AA02882381F012
:109C30001092B2021092B3021092B4021092B502C6
:109C40001092B6021092B7021092B8021092B902A6
:109C5000BB81BB23F1F48091B608282F332744271A
:109C600055278091D2029091D302A091D402B09155
:109C7000D502BC01CD010E944A70DC01CB01BC01C0
:109C8000CD0128EF3AE240E050E00E94BE70390179
:109C900002C066247724809176028823F1F48091B3
:109CA000B608282F3327442755278091CE0290915C
:109CB000CF02A091D002B091D102BC01CD010E948F
:109CC0004A70DC01CB01BC01CD0128EF3AE240E053
:109CD00050E00E94BE70290102C0442455248091A6
:109CE000920890919308893C91051CF088EC90E0D3
:109CF00005C088539F4F34F488E39FEF90939308F7
:109D0000809392088091990890919A08893C9105D6
:109D10001CF088EC90E005C088539F4F34F488E332
:109D20009FEF90939A088093990880919B08909157
:109D30009C08AA2797FDA095BA2F2091E008A22E93
:109D4000BB24CC24DD24BC01CD01A60195010E94D9
:109D50004A709B01AC018091920890919308AA27C8
:109D600097FDA095BA2FE7E0880F991FAA1FBB1F88
:109D7000EA95D1F7280F391F4A1F5B1F57FF04C010
:109D8000215C3F4F4F4F5F4F76E055954795379594
:109D900027957A95D1F78301020F131F10939C0822
:109DA00000939B088091900890919108AA2797FDB5
:109DB000A095BA2FBC01CD01A60195010E944A7061
:109DC0009B01AC018091990890919A08AA2797FD70
:109DD000A095BA2F67E0880F991FAA1FBB1F6A952D
:109DE000D1F7280F391F4A1F5B1F57FF04C0215CA2
:109DF0003F4F4F4F5F4FA6E05595479537952795B5
:109E0000AA95D1F74201820E931E909291088092FA
:109E100090088091DB089091DC08880F991FAA2791
:109E200097FDA095BA2F20919708332744275527EF
:109E3000BC01CD010E944A705B016C0197FF08C014
:109E40002FE330E040E050E0A20EB31EC41ED51E4A
:109E5000F6E0D594C794B794A794FA95D1F780917A
:109E6000A508282F3327442755278091CA029091AF
:109E7000CB02A091CC02B091CD02BC01CD010E94D9
:109E80004A70DC01CB01BC01CD0120EF35E540E09B
:109E900050E00E94BE70B501620F731F7093DC0822
:109EA0006093DB080150104134F080E090E1909322
:109EB0009C0880939B0880919B0890919C088050FF
:109EC000904F34F480E090EF90939C0880939B082F
:109ED00051E0851650E1950634F080E090E19093D2
:109EE00091088093900880919008909191088050FB
:109EF000904F34F480E090EF909391088093900815
:109F00006150704134F080E090E19093DC088093E0
:109F1000DB088091DB089091DC088050904F34F48E
:109F200080E090EF9093DC088093DB0880915B02E7
:109F300085FD16C08091020199272091230130915F
:109F4000240169817A81689FA001699F500D789FE3
:109F5000500D1124CA01B9010E9475707A8369837A
:109F6000809122038150809322038F3F09F05EC0CD
:109F70008091230390912403892B41F48091230144
:109F800090912401909324038093230380912301D3
:109F9000909124012091230330912403281739073D
:109FA00018F42F5F3F4F09C0809123019091240145
:109FB0008217930730F421503040309324032093CC
:109FC000230384E6809322038091B901282F33274D
:109FD00040912303509124034217530710F48AE061
:109FE0000CC080910001280F311D2417350738F46B
:109FF00080915102882319F0815080935102809101
:10A00000B801282F33274217530710F489E10CC0F9
:10A0100080910001280F311D2417350738F48091F5
:10A020005002882319F08150809350028091510290
:10A030008823D1F08091840290918502A0918602BC
:10A04000B0918702B7FD10C080919F068093830274
:10A0500080EE91EBAFEFBFEF809384029093850287
:10A06000A0938602B09387028091E601882311F4C1
:10A070000E944E5C89819A81880F991F880F991FD1
:10A080009A8389838091D00880FFE4C7809176020B
:10A09000882309F0DFC740917702442309F0DAC72B
:10A0A0008091A20399278F779070009709F0D2C70B
:10A0B0004C012091EA023091EB022115310509F0A3
:10A0C00044C08091190190911A018959934058F028
:10A0D00087B5853F20F480910302815011C081E053
:10A0E0008093300353C08091190190911A018436F6
:10A0F000910530F587B58B30F8F0809103028F5FC2
:10A10000809303029AE08902900111248091D9057D
:10A11000821B87BD87B5809588BD8CE291E09093C6
:10A12000E8018093E7018EE591E09093EB02809344
:10A13000EA020E94DF192AC081E080932F0326C023
:10A1400040932F034093300321C0909302028093E9
:10A15000010280918E0290918F02A0919002B091A5
:10A16000910274E0880F991FAA1FBB1F7A95D1F73F
:10A170008093040290930502A0930602B093070215
:10A18000215030403093EB022093EA028091D008B6
:10A190002091710281FF25C02233E8F48091910162
:10A1A0008150809391018F3FE1F51092AB02809135
:10A1B0008E0290918F02A0919002B09191028093B3
:10A1C0008A0290938B02A0938C02B0938D0281E05F
:10A1D0008093910126C0273420F188EC809391016F
:10A1E0001DC08091450190914601820F911D2091E3
:10A1F0003F063327829FF001839FF00D929FF00D61
:10A200001124CF01AA2797FDA095BA2F80938A0227
:10A2100090938B02A0938C02B0938D0281E0809387
:10A22000AB028091D2029091D302A091D402B0915E
:10A23000D502E0904101F09042010091430110915C
:10A240004401BC01CD01A80197010E94BE705901D3
:10A250006A018091CE029091CF02A091D002B0917C
:10A26000D102BC01CD01A80197010E94BE70B901C5
:10A27000C5010E94A567209177013327829FA00125
:10A28000839F500D929F500D1124CA0164E670E027
:10A290000E9489709B016C33710514F02CE330E04F
:10A2A000C9010E94CF659093A2088093A10880E223
:10A2B0008093400110928902109288028091AB0233
:10A2C000882309F46EC580915B0299279C01207157
:10A2D000307084FD66C580915A02826080935A0274
:10A2E0007091B408872F992761E0C62ED12CC8221F
:10A2F000D92280FD04C08091D00881FD10C0098161
:10A300001A813093260320932503309389022093EA
:10A31000880280915B02806C80935B02CFC2809147
:10A320005B0281FF9EC20091810110918201C801F0
:10A330000F96A0909E02B0909F028A159B0508F090
:10A3400079C080912F03882309F074C080915B024B
:10A3500087FF15C080915B028F7780935B028091AD
:10A36000F7019091F801A091F901B091FA01809361
:10A370008A0290938B02A0938C02B0938D02E0909E
:10A380009808EE20F9F080918A0290918B02A091BA
:10A390008C02B0918D02BC01CD0124E630E040E09A
:10A3A00050E00E94BE708E2D9927AA27BB278217E6
:10A3B0009307A407B50734F4D0928902C0928802AB
:10A3C0008DE378C08091270390912803459784F00E
:10A3D0008091F7019091F801A091F901B091FA01F3
:10A3E00080938A0290938B02A0938C02B0938D028B
:10A3F00080915B02806480935B029501201B310B8E
:10A400002F50304037FF03C0309521953F4F309398
:10A4100089022093880280915102882349F0C90162
:10A4200063E070E00E9489707093890260938802F3
:10A430008BE240C0C8010F97A816B90608F03FC0CC
:10A44000809130038823D9F580915B0286FD07C097
:10A450008091270390912803845D9E4FACF48091F6
:10A460005B028F7B80935B028091F7019091F801F2
:10A47000A091F901B091FA0180938A0290938B0226
:10A48000A0938C02B0938D0280915B0280688093D0
:10A490005B02C501801B910B0F9697FF03C090953F
:10A4A00081959F4F909581959F4F909389028093BE
:10A4B00088028DE28093400110928202D9C08DE320
:10A4C0008093400160918302662371F120918402A0
:10A4D00030918502409186025091870280918A02D4
:10A4E00090918B02A0918C02B0918D0282179307FC
:10A4F000A407B507CCF480915B02806480935B0273
:10A50000862F992790938902809388028AE080930E
:10A5100082028EE58093400180915B0287FFA8C094
:10A5200080915B028F7733C0662309F443C020918A
:10A530008402309185024091860250918702809179
:10A540008A0290918B02A0918C02B0918D02281703
:10A5500039074A075B0774F580915B028068809336
:10A560005B02862F9927909581959F4F9093890242
:10A570008093880286EF8093820286E78093400171
:10A5800080915B0286FF74C080915B028F7B809319
:10A590005B028091F7019091F801A091F901B091CF
:10A5A000FA0180938A0290938B02A0938C02B0935D
:10A5B0008D025EC080915B02807C09F459C080915D
:10A5C0008202882379F5A090F701B090F801C0903D
:10A5D000F901D090FA01D601C501885C9040A040F5
:10A5E000B04020918A0230918B0240918C025091B0
:10A5F0008D0282179307A407B5075CF4D601C50145
:10A6000088539F4FAF4FBF4F281739074A075B0743
:10A610005CF080938A0290938B02A0938C02B0939B
:10A620008D0202C01092820280915B028F73809330
:10A630005B02109226031092250371FF06C084EF7F
:10A6400091E09093E8018093E70180919202882342
:10A6500079F480918E0290918F02A0919002B09136
:10A660009102C397A105B1051CF081E0809392028D
:10A670006091250370912603809188029091890250
:10A68000680F791F7093260360932503CB0177FF32
:10A6900004C088279927861B970B855F91400CF48F
:10A6A000C9C040918202442389F180918402909133
:10A6B000850220918A0230918B02821B930B0996AE
:10A6C000439748F48091840290918502A09186027C
:10A6D000B091870212C0242F332727FD3095432FD6
:10A6E000532F80918A0290918B02A0918C02B0919D
:10A6F0008D02820F931FA41FB51F80938A0290932F
:10A700008B02A0938C02B0938D0224C080913F06EF
:10A7100020918A0230918B0240918C0250918D02DF
:10A720001616170644F463E00E946970280F311D65
:10A73000411D511D07C063E00E946970281B31094B
:10A740004109510920938A0230938B0240938C0275
:10A7500050938D021092260310922503A0908E0232
:10A76000B0908F02C0909002D0909102D601C501A6
:10A7700080509440A040B0402091F7013091F80102
:10A780004091F9015091FA0182179307A407B50788
:10A790005CF4D601C50180509C4FAF4FBF4F2817C6
:10A7A00039074A075B0744F08093F7019093F8015B
:10A7B000A093F901B093FA01A090F701B090F801CD
:10A7C000C090F901D090FA01D601C50180509440A3
:10A7D000A040B04020918A0230918B0240918C02BF
:10A7E00050918D0282179307A407B5075CF4D60138
:10A7F000C50184529A4FAF4FBF4F281739074A07F8
:10A800005B0744F080938A0290938B02A0938C02A2
:10A81000B0938D028091B40881FF06C084E690E079
:10A820009093E8018093E70180918302882311F4DB
:10A830000E94CA3E8091EA029091EB02892BD1F1ED
:10A840008091F7019091F801A091F901B091FA017E
:10A8500080938A0290938B02A0938C02B0938D0216
:10A8600029C08091F7019091F801A091F901B09170
:10A87000FA01805D9740A040B04080938A02909397
:10A880008B02A0938C02B0938D02809143068823A3
:10A8900011F0992702C08FE790E090938201809396
:10A8A0008101E981FA81F0937902E09378028EE2E6
:10A8B000809340010091780210917902A090F701F5
:10A8C000B090F801C090F901D090FA0120918A026D
:10A8D00030918B0240918C0250918D022A153B05DC
:10A8E0004C055D0524F08091B40880FD6CC2809118
:10A8F0005202882309F067C28091EA029091EB022C
:10A90000892B49F000917802109179021092280366
:10A9100010922703DCC0D601C501821B930BA40B48
:10A92000B50B8093080390930903A0930A03B09397
:10A930000B038230F0E89F07FFEFAF07FFEFBF0781
:10A940002CF481E090E8AFEFBFEF09C08F5F9F4725
:10A95000A040B04064F08FEF9FE7A0E0B0E08093AC
:10A96000080390930903A0930A03B0930B0380910B
:10A970000803909109039093280380932703809103
:10A980007A01282F33274427552780910803909177
:10A990000903A0910A03B0910B03BC01CD010E94F1
:10A9A0004A7097FF04C0615E7F4F8F4F9F4F55E005
:10A9B00095958795779567955A95D1F76093080394
:10A9C0007093090380930A0390930B0365303EEF65
:10A9D00073073FEF83073FEF93072CF484E09EEF6C
:10A9E000AFEFBFEF09C0605074408040904064F00A
:10A9F00080E094E0A0E0B0E0809308039093090326
:10AA0000A0930A03B0930B0380900803909009036E
:10AA1000609101027091020277FF02C0695F7F4F6F
:10AA20009B0143E0359527954A95E1F75FEF223882
:10AA300035071CF421E83FEF05C02038310514F03C
:10AA400020E830E0C901AA2797FDA095BA2F2091F0
:10AA50007B01332744275527BC01CD010E944A7052
:10AA600097FF04C06D5F7F4F8F4F9F4F22E09595FA
:10AA70008795779567952A95D1F79B016FEF2130E0
:10AA800036071CF420E03FEF06C02F3F310519F0D8
:10AA900014F020E031E080915B02807C49F0C90134
:10AAA00037FD03969C0135952795359527950DC063
:10AAB0008091B40880FF09C0C90137FD07969C0149
:10AAC00083E0359527958A95E1F7820E931E2091B4
:10AAD0007901222309F454C06091AE027091AF0253
:10AAE0008091B0029091B10297FF04C061587F4FEE
:10AAF0008F4F9F4FB7E09595879577956795BA9556
:10AB0000D1F73327442755270E944A7097FF04C086
:10AB1000615E7F4F8F4F9F4FA5E095958795779505
:10AB20006795AA95D1F76093080370930903809302
:10AB30000A0390930B036138AFEF7A07AFEF8A07F0
:10AB4000AFEF9A072CF480E89FEFAFEFBFEF0AC09A
:10AB50006F3F71058105910569F064F080E091E037
:10AB6000A0E0B0E08093080390930903A0930A0348
:10AB7000B0930B038091080390910903880E991EEE
:10AB8000C401AA2797FDA095BA2FC0907802D09053
:10AB900079029601442737FD4095542FBC01CD0121
:10ABA0000E944A7097FF04C061507E4F8F4F9F4FA5
:10ABB000F9E09595879577956795FA95D1F7061BF6
:10ABC000170B8091880290918902892B09F064C04B
:10ABD0001C141D040CF060C0209127033091280341
:10ABE000C90137FF03C0309521953F4F2D33310503
:10ABF00040F48091A6029091A7028017910774F506
:10AC000026C02C533040E5E036952795EA95E1F7CC
:10AC10002031310510F02FE030E04091A602509134
:10AC2000A70218161906E4F480E190E0821B930B4A
:10AC3000489F9001499F300D589F300D112474E0BA
:10AC4000369527957A95E1F72017310720F5809101
:10AC50007F019091800108171907F4F08C011CC046
:10AC6000205F3F4F80917F0190918001829FF00192
:10AC7000839FF00D929FF00D11249F0164E03695A3
:10AC800027956A95E1F74017510714F08A0104C02F
:10AC90000217130708F08901C801AA2797FDA0959C
:10ACA000BA2F5DE0880F991FAA1FBB1F5A95D1F7D5
:10ACB0002091A1083091A208442737FD4095542FD8
:10ACC000BC01CD010E94BE7020930C0330930D0394
:10ACD00040930E0350930F0300910C0310910D034A
:10ACE0008091290390912A039C01220F331F280F82
:10ACF000391F200F311F37FF02C02D5F3F4FA901C1
:10AD0000559547955595479550932A0340932903A8
:10AD100080913B06282F3327220F331F220F331F2A
:10AD2000241735076CF48091D808282F3327220F79
:10AD3000331F220F331F205530404217530724F092
:10AD400030932A03209329038091B40880FF14C014
:10AD50008091290390912A0329813A8182179307D0
:10AD600024F030932A032093290340912903509122
:10AD70002A035A83498327C029813A812C193D0926
:10AD800037FF02C02D5F3F4F3595279535952795A5
:10AD90006091290370912A03620F731F7A8369837C
:10ADA00012C00E94CA3E89819A8190932A0380939F
:10ADB000290380915B02806C80935B0280915A0230
:10ADC0008D7F80935A0280915B0299279C012270AB
:10ADD000307081FF30C180912B0390912C03A091A2
:10ADE0002D03B0912E030097A105B10521F08091AC
:10ADF00092028130B9F48091780290917902AA2769
:10AE000097FDA095BA2F1EE0880F991FAA1FBB1FA0
:10AE10001A95D1F780932B0390932C03A0932D03C5
:10AE2000B0932E0380919202813019F482E08093D6
:10AE30009202A981BA817D010027F7FC0095102FAD
:10AE40008091A1089091A2089C01442737FD40956C
:10AE5000542FC801B7010E944A70DC01CB018093D6
:10AE60000C0390930D03A0930E03B0930F03B7FF51
:10AE700004C08150904EAF4FBF4F5C016D01FDE0AB
:10AE8000D594C794B794A794FA95D1F7A0920C03E0
:10AE9000B0920D03C0920E03D0920F0360915C023A
:10AEA00070915D02BFE0603A7B0750F580912B0303
:10AEB00090912C03A0912D03B0912E039C01AD0124
:10AEC000EAE05695479537952795EA95D1F7821B85
:10AED000930BA40BB50BA601950104E0220F331FC1
:10AEE000441F551F0A95D1F7820F931FA41FB51F4A
:10AEF00080932B0390932C03A0932D03B0932E03E8
:10AF000060547F4118F580912B0390912C03A09100
:10AF10002D03B0912E039C01AD011CE05695479581
:10AF2000379527951A95D1F7821B930BA40BB50B78
:10AF3000A6019501F2E0220F331F441F551FFA9519
:10AF4000D1F7820F931FA41FB51F38C08091010253
:10AF500090910202809101029091020297FF03C03A
:10AF6000909581959F4F8436910584F58091F701E6
:10AF70009091F80120918A0230918B02821B930BF1
:10AF800081509F4F8F5F914008F580912B039091E6
:10AF90002C03A0912D03B0912E039C01AD01EEE096
:10AFA0005695479537952795EA95D1F7821B930BD0
:10AFB000A40BB50B8A0D9B1DAC1DBD1D80932B03EF
:10AFC00090932C03A0932D03B0932E0380912B0319
:10AFD00090912C03A0912D03B0912E037EE0B695A5
:10AFE000A795979587957A95D1F790937902809355
:10AFF000780240914106442399F055279C01BA01FB
:10B000000E948970C901861B970B9093A7028093B9
:10B01000A602260F371F3093800120937F011FC0A7
:10B020001092A7021092A6028FEF93E090938001F6
:10B0300080937F0114C01092920210922B03109201
:10B040002C0310922D0310922E033093790220933B
:10B05000780205C080915B02806C80935B028091D6
:10B060003E0381FF37C089819A8197FD03969595AC
:10B07000879595958795209157023091580228170A
:10B08000390760F48091780290917902892B31F030
:10B09000220F331F220F331F3A8329838091F70138
:10B0A0009091F801A091F901B091FA0180938A0280
:10B0B00090938B02A0938C02B0938D0288E99AE35F
:10B0C0009093E8018093E70180E09EE090930C016B
:10B0D00080930B012091A008822F9927880F991F38
:10B0E000880F991F889649815A818417950714F013
:10B0F0009A8389838091D8089927880F991F880F90
:10B10000991F8055904069817A818617970714F4BA
:10B110009A83898380913B02882341F48091780946
:10B120008E3F20F0809142038823D9F080915C0209
:10B1300090915D020297C097A0F489819A811816B8
:10B1400019067CF481E090E090935D0280935C02AC
:10B15000A22FBB27AA0FBB1FAA0FBB1F9896BA83AB
:10B16000A9838091E601882311F40E944E5CE98155
:10B17000FA81F0939705E0939605809104039091EE
:10B180000503A0910603B091070312E0880F991FF1
:10B19000AA1FBB1F1A95D1F70091DB081091DC089C
:10B1A000081B190BE13AF1058CF0CF01F7FD019670
:10B1B00095958795801791070CF48C019095819552
:10B1C0009F4F081719076CF48C010BC0013511054E
:10B1D00014F000E510E0FFEF003B1F0714F400EB54
:10B1E0001FEF8091D808282F3327220F331F220FFB
:10B1F000331FC90149815A81841B950B8017910720
:10B200000CF48C0169817A81621B730B0617170796
:10B210000CF48B0180919B0890919C086091A40292
:10B220007091A502861B970B9093A7088093A608A0
:10B23000D090B6082091B6023091B7024091B80282
:10B240005091B902DD2041F0661A770AC301AA279E
:10B2500097FDA095BA2F04C0AA2797FDA095BA2FF5
:10B26000280F391F4A1F5B1F2093B6023093B70285
:10B270004093B8025093B9028091B6029091B70200
:10B28000A091B802B091B90281509A4FA040B0404D
:10B2900064F080E09AEFA0E0B0E08093B602909373
:10B2A000B702A093B802B093B9028091B602909110
:10B2B000B702A091B802B091B90280509640AF4F4A
:10B2C000BF4F64F480E096E0AFEFBFEF8093B6022B
:10B2D0009093B702A093B802B093B902C090500601
:10B2E0002091A6083091A70878E07C1598F08C2D65
:10B2F0009927829FD001839FB00D929FB00D11249A
:10B30000CD01B7FD07965C0163E0B594A7946A95FB
:10B31000E1F712C08C2D86959927829FF001839FBB
:10B32000F00D929FF00D1124CF01F7FD03965C0103
:10B33000B594A794B594A79480907C0190907D01DA
:10B340009401442737FD4095542F8091B602909187
:10B35000B702A091B802B091B902BC01CD010E9420
:10B36000BE70A20EB31EE09066016E2D772788276F
:10B370009927980117FF04C022273327201B310B80
:10B3800037FF02C02F5F3F4F3595279549815A817E
:10B39000240F351F442737FD4095542F0E944A70D3
:10B3A00097FF04C0615C7F4F8F4F9F4F26E09595BC
:10B3B0008795779567952A95D1F79B016A157B0547
:10B3C0000CF45B0166277727621B730BA616B70682
:10B3D0000CF45B0180919008909191086091A20219
:10B3E0007091A302861B970B90938F0880938E0811
:10B3F0002091B2023091B3024091B4025091B50253
:10B40000DD2041F0461A570AC201AA2797FDA095F0
:10B41000BA2F04C0AA2797FDA095BA2F280F391F6D
:10B420004A1F5B1F2093B2023093B3024093B402D1
:10B430005093B5028091B2029091B302A091B402F0
:10B44000B091B50281509A4FA040B04064F080E0C6
:10B450009AEFA0E0B0E08093B2029093B302A09381
:10B46000B402B093B5028091B2029091B302A09160
:10B47000B402B091B50280509640AF4FBF4F64F414
:10B4800080E096E0AFEFBFEF8093B2029093B302FB
:10B49000A093B402B093B50220918E0830918F082A
:10B4A00078E07C1598F08C2D9927829FD001839F9E
:10B4B000B00D929FB00D1124CD01B7FD07966C0120
:10B4C000B3E0D594C794BA95E1F712C0C6948C2D19
:10B4D0009927829FF001839FF00D929FF00D112418
:10B4E000CF01F7FD03966C01D594C794D594C7940A
:10B4F0009401442737FD4095542F8091B2029091DA
:10B50000B302A091B402B091B502BC01CD010E947A
:10B51000BE70C20ED31E6E2D7727882799279801FB
:10B5200017FF04C022273327201B310B37FF02C02F
:10B530002F5F3F4F3595279549815A81240F351F3D
:10B54000442737FD4095542F0E944A7097FF04C04E
:10B55000615C7F4F8F4F9F4FE6E09595879577957C
:10B560006795EA95D1F79B016C157D050CF46B018D
:10B5700066277727621B730BC616D7060CF46B0180
:10B580008091E601882311F40E944E5C8091A0080E
:10B59000682F77277D836C838091D808A82FBB27DD
:10B5A000BF83AE83E090930668E4862E67E0962E14
:10B5B00053EC652E56E0752E4BE0342E37EB432EC0
:10B5C00038E0532EF301208112160CF030C12034E4
:10B5D00029F429813A813B872A871FC049815A81F2
:10B5E000CA01AA2797FDA095BA2F332727FD3095CA
:10B5F000432F532FBC01CD010E944A7097FF04C016
:10B60000615C7F4F8F4F9F4F26E09595879577958B
:10B6100067952A95D1F77B876A87F30121812034CA
:10B6200039F42A853B852A0D3B1D3B872A872AC092
:10B63000203C39F44A855B854A195B095B874A8758
:10B6400021C0C501AA2797FDA095BA2F332727FD52
:10B650003095432F532FBC01CD010E944A7097FFB4
:10B6600004C0615C7F4F8F4F9F4FB6E095958795E3
:10B6700077956795BA95D1F7AA85BB85A60FB71FB1
:10B68000BB87AA87F3012281203439F42A853B85C0
:10B690002C0D3D1D3B872A872AC0203C39F44A8562
:10B6A0005B854C195D095B874A8721C0C601AA27C3
:10B6B00097FDA095BA2F332727FD3095432F532FA1
:10B6C000BC01CD010E944A7097FF04C0615C7F4FAE
:10B6D0008F4F9F4FA6E09595879577956795AA958B
:10B6E000D1F7AA85BB85A60FB71FBB87AA87F30131
:10B6F0002381203439F42A853B85200F311F3B8775
:10B700002A872AC0203C39F44A855B85401B510BAF
:10B710005B874A8721C0C801AA2797FDA095BA2F49
:10B72000332727FD3095432F532FBC01CD010E94B5
:10B730004A7097FF04C0615C7F4F8F4F9F4FF6E0C8
:10B740009595879577956795FA95D1F7AA85BB85E5
:10B75000A60FB71FBB87AA87F401808181FD08C0AF
:10B76000D2018D919C91EA85FB858E179F0774F419
:10B77000D2018D919C91EA85FB858E0F9F1F97FDCD
:10B780000196959587959B878A871EC0EE2049F480
:10B790002A853B85220F331F281B390B3B872A87BD
:10B7A00013C031E03E1580F42E2D33274A855B858A
:10B7B000841B950BB9010E948970CB016A857B853A
:10B7C000680F791F7B876A878C819D81880F991FFD
:10B7D000880F991FAA85BB858A179B075CF48E8109
:10B7E0009F81880F991F880F991FEA85FB85E817AD
:10B7F000F90714F09B878A878A859B8597FD0396B6
:10B800009595879595958795F4018183880F991F64
:10B81000880F991F2A853B85281B390BC901880F82
:10B820008283EA85FB85D201ED93FC9303C0F4018A
:10B83000118212823A9422E030E0420E531E44E01C
:10B8400050E0640E751E6FE070E0860E971E37FEA6
:10B85000B9CEE2E1C55F0C94F57084B1806A84B919
:10B860003D9A82E58CBD1DBC459A81E08093EC0831
:10B870008AEA8093FD0883E88093FE088AE080933B
:10B88000FF0810920109109200091092030910920A
:10B890000209109265091092210908953091EC086F
:10B8A000332309F070C00DB407FE6DC085E08093AE
:10B8B000E601459A2EB5809146039927813091057E
:10B8C00089F0823091051CF4892B21F03EC002974B
:10B8D000B9F03BC030932009209347032138A9F5E4
:10B8E00081E008C0253549F480914703820F809399
:10B8F000470382E08093460328C03093460325C067
:10B9000080912009E82FFF27EE5BF64F20838F5FA1
:10B9100080932009909147038032A0F0291769F4A1
:10B9200080E2A2E4B9E0E2E2F9E00D9001928A95AA
:10B93000E1F781E08093210902C030932109109240
:10B94000460303C0920F909347032091FC082232D4
:10B95000A0F445980000000000000000E091F50808
:10B96000F091F608E20FF11D80818EBD80911E09D5
:10B970009081890F80931E0903C081E08093EC08B9
:10B980002F5F2093FC080895EF92FF920F931F936F
:10B99000CF93DF93809149069927880F991F880FCD
:10B9A000991F7C010027F7FC0095102F8091D2028F
:10B9B0009091D302A091D402B091D502BC01CD01E7
:10B9C000A80197010E94BE703093010920930009DD
:10B9D0008091CE029091CF02A091D002B091D1027D
:10B9E000BC01CD01A80197010E94BE7030930309EC
:10B9F000209302092091E2083091E3084091E40885
:10BA00005091E508DA01C90163E0880F991FAA1F68
:10BA1000BB1F6A95D1F7820F931FA41FB51F820F1A
:10BA2000931FA41FB51F2091410130914201409105
:10BA3000430150914401BC01CD010E94BE7030937E
:10BA4000090920930809C091E402D091E502809190
:10BA50000E0290910F029E01281B390B30930F09A3
:10BA600020930E09E091DA02F091DB028091AD089B
:10BA70009091AE08BF010E9489709B01220F331F75
:10BA8000220F331F260F371F260F371F37FF02C025
:10BA90002D5F3F4F359527953595279530930509AF
:10BAA000209304098091DE089091DF08BF010E9475
:10BAB00089709B01220F331F220F331F260F371F60
:10BAC000260F371F37FF02C02D5F3F4F3595279553
:10BAD0003595279530930709209306091092DB02CC
:10BAE0001092DA021092AE081092AD081092DF08A0
:10BAF0001092DE088091FF089927AA27BB27FC0136
:10BB00003A97EA30F10508F088C2E35AFF4F0C94E7
:10BB10001071809170028093120980916F0280935E
:10BB2000130980916E028093140980916D028093B5
:10BB3000150980916C028093160980916B028093A5
:10BB4000170980916A028093180980916902809395
:10BB5000190980915B0280931A0980915B02837FAF
:10BB600080935B028091010180931B0980912301E6
:10BB70009091240180931C0980915A0280931D09A1
:10BB800042994BC280915A02877F80935A0245C2E4
:10BB9000809172099091730990931309809312090F
:10BBA0008091480380931409809178098093150946
:10BBB00080917E060E949E3B8093160980914001F1
:10BBC0008093170920914803822F9927FC01C4E034
:10BBD000EE0FFF1FCA95E1F7E81BF90BE85BF84F82
:10BBE00086858093180980818093190986818093C6
:10BBF0001A09838180931B09878180931C098581A1
:10BC000080931D092F5F20934803E22FFF27EE0F3B
:10BC1000FF1FEE0FFF1FEA54F94F858518160CF42D
:10BC2000FCC1222309F4F9C1822F992701966DE006
:10BC300070E00E948970AC01282FE82FFF27EE0FDB
:10BC4000FF1FEE0FFF1FEA54F94F8585181614F0F9
:10BC5000442351F740934803E0C18091490388236E
:10BC6000A9F58DE08093FF0881E0809349038091DE
:10BC700002018093120980917F06809313098091BD
:10BC80008006809314098091810680931509809124
:10BC90008206809316098091860680931709809109
:10BCA00087068093180980918806809319098091EE
:10BCB0008B0680931A098091890680931B098091D5
:10BCC0008A0680931C0980918C06A5C182E180932D
:10BCD000FF08109249038091E8029091E902909345
:10BCE0001309809312098091E6029091E7029093E4
:10BCF000150980931409D0931709C09316098091F0
:10BD0000710680931809809178029091790297FDCD
:10BD10000396959587959595879580931909109227
:10BD20001A0910921B0910921C0910921D0975C165
:10BD300080917D06809312091092130980919F06CD
:10BD40008093140980919406809315098091500284
:10BD50008093160980916B03809317098091690382
:10BD600080931809809168038093190910926B03DE
:10BD7000109269031092680380917801882329F05A
:10BD80008091AC029091AD0204C080919508909191
:10BD9000960890931B0980931A098091A3068093BB
:10BDA0001C098091A40637C1F89480913006E82FD1
:10BDB000FF27EE0FFF1FE350F84F0190F081E02DB9
:10BDC000E038F1051CF0EFE7F0E006C03FEFE138A6
:10BDD000F30714F4E1E8FFEFE093120980913106D4
:10BDE000E82FFF27EE0FFF1FE350F84F0190F0817F
:10BDF000E02DE038F1051CF0EFE7F0E006C07FEF42
:10BE0000E138F70714F4E1E8FFEFE09313098091BC
:10BE10002F06E82FFF27EE0FFF1FE350F84F01908A
:10BE2000F081E02DE038F1051CF0EFE7F0E006C00E
:10BE30008FEFE138F80714F4E1E8FFEFE09314091D
:10BE400080912E06E82FFF27EE0FFF1FE350F84FDB
:10BE50000190F081E02DE038F1051CF0EFE7F0E013
:10BE600006C02FEFE138F20714F4E1E8FFEF789411
:10BE7000E0931509809195028093160980919602AE
:10BE800080931709809197028093180980919802F6
:10BE9000809319098091990280931A0980919A02DE
:10BEA00080931B0980919B0280931C0980919C02C6
:10BEB000B2C08091BD03853018F01092BD0385E0BB
:10BEC0008093120980918D068093130980918E02D0
:10BED00090918F02A0919002B0919102BC01CD018E
:10BEE00025E030E040E050E00E94BE70309315093C
:10BEF0002093140980918A0290918B02A0918C0268
:10BF0000B0918D02BC01CD0125E030E040E050E071
:10BF10000E94BE7030931709209316098091830602
:10BF20008093180980918406809319098091850671
:10BF300080931A098091940280931B0980914A038F
:10BF400080931C09809196059091970597FD039623
:10BF500095958795959587955EC082E080931209A7
:10BF600088E0809313091092140987E480931509DF
:10BF700080910301809316098091A2038093170991
:10BF80009091A303909318098F778093A2039071E7
:10BF90009093A3038091A006809319098091D00803
:10BFA00080931A098091B40880931B0980919006B0
:10BFB00080931C098091A8062EC0809176099091EB
:10BFC0007709909313098093120980916E018093F1
:10BFD000140980916D01809315098091C0058093AB
:10BFE0001609809159028093170980918E068093DB
:10BFF000180980919808809319098091B401909153
:10C00000B50190931B0980931A098091640680936F
:10C010001C098091A50380931D0980912109882323
:10C0200009F45FC1609122098091A201681719F09B
:10C030008AEF8093A0016093A20181E080938E013A
:10C040004091230950912409CA0181509E4F8F5F6E
:10C050009340B0F42091250930912609C9018150FF
:10C060009E4F8F5F934060F480913A0685FF08C031
:10C0700050933503409334033093330320933203BA
:10C080008091290990912A0921E08936920724F4A8
:10C090009093900180938F0120913309309134095E
:10C0A0008091E7019091E8018217930740F4809115
:10C0B000BA01882321F43093E8012093E701862F09
:10C0C00099278836910509F453C08936910524F4DF
:10C0D0008736910551F00DC18936910509F47DC06F
:10C0E0008B36910509F4D8C004C18091350980933D
:10C0F00062098091360980936409809137098093A1
:10C1000063098091380980938D018091390980936A
:10C11000660980913A098093A10180913B0980933F
:10C12000450380913C098093310380916802882304
:10C1300051F080913D0990913E0997FD04C0909384
:10C14000AD028093AC0220913C0330913D0380917D
:10C150003F0990914009280F391F37FF02C02F5F18
:10C160003F4F3595279530933D0320933C03C1C045
:10C17000809135098093F708809136098093F808FB
:10C18000809137098093F908809138098093FA08E3
:10C19000809139098093FB088091860590913A0936
:10C1A000892B8093860590918705937080913B0938
:10C1B0008C70982B9093870580913C098093420363
:10C1C00080913D098093920180913E098093650999
:10C1D00080913F0980933E038CC080913509809304
:10C1E000ED08809136098093EE088091370980939D
:10C1F000EF08809138098093F00880913909909177
:10C200003A099093F2088093F10880913B0990914C
:10C210003C099093F4088093F3088091370890913B
:10C220003808813849F480914403882329F48091A7
:10C230003D0981588093440380913D09992787FDEA
:10C240009095909338088093370880913E098093A9
:10C25000830280913F09909140099C01442737FD5A
:10C260004095542FDA01C90163E0880F991FAA1F76
:10C27000BB1F6A95D1F7820F931FA41FB51F820FB2
:10C28000931FA41FB51F8093840290938502A093EF
:10C290008602B09387022DC08091350980934103B7
:10C2A00080913609809340038091370980933F0342
:10C2B0008091390980936E0380913A0980936D03D0
:10C2C00080913D0980936C0380913E0980936A03BD
:10C2D00080913F09909140099093DA088093D908A2
:10C2E00008C0109235031092340310923303109259
:10C2F0003203E6E0CDB7DEB70C9401718091EC0813
:10C30000882319F480E090E0089545988DEF98E037
:10C310009093F6088093F50890914303E92FFF2747
:10C32000ED56FE4F9F5F9093430380818093FF08FB
:10C330009D3010F0109243031092EC080E94C45CF0
:10C3400081E08093FC088091FD0880931E098EBDDA
:10C3500081E090E0089587B18C6087B94298439856
:10C3600010924C0380E88093A40110924B038093B9
:10C37000A301089540914403442311F040935603D0
:10C38000809151038150809351038F3F09F054C134
:10C3900080917706809352038091790680935303AE
:10C3A00089E08093510380915B029927807390709C
:10C3B000892B21F48091A30380FF1DC080917B060F
:10C3C000882351F080915403882319F484E08093EA
:10C3D0004C0381E08093540380917C06882379F09C
:10C3E00080915503882319F484E080934B0381E006
:10C3F0008093550304C0109254031092550380910A
:10C400005403882309F084C08091A506282F332780
:10C4100024FF07C080919302882319F425FD91C061
:10C4200092C090917806983F48F08091AF088D3D7A
:10C4300028F08091520388236CF00AC0983F78F06E
:10C440008091AF08853059F48091520387FF02C074
:10C45000429A01C0429881E08093A40156C0809125
:10C460004C03815080934C038F3F09F06DC0809145
:10C47000A80685FF31C090915603892F8695809339
:10C480004C03992361F490934A038091520387FFF0
:10C4900002C0429A01C042981092A40155C081E0A6
:10C4A00080934A038091A40190915203882359F408
:10C4B000409356038093440380E48093A40199231E
:10C4C0000CF43FC040C0982311F0429A01C042983A
:10C4D00086958093A40138C08091AF08869580939B
:10C4E0004C038091A401813021F41092560380E422
:10C4F00001C086958093A4018091A401909152037C
:10C50000892311F0429A01C0429810924A031CC03C
:10C5100080914C03815080934C038F3FA9F489E0B4
:10C5200080934C038091A401813011F480E801C014
:10C5300086958093A4018091A40190917B06892324
:10C5400011F0429A01C0429880915503882309F066
:10C5500043C09091A50697FF07C08091930288235E
:10C5600019F496FD52C053C090917A06983F48F056
:10C570008091D7088D3D28F08091530388236CF07B
:10C580000AC0983F78F08091D708853059F480919F
:10C59000530387FF02C0439A01C0439881E0809310
:10C5A000A30136C080914B03815080934B038F3F92
:10C5B00079F58091D708869580934B038091A301EC
:10C5C000813011F480E401C086958093A3018091AD
:10C5D000A3019091530317C080914B038150809326
:10C5E0004B038F3FA9F489E080934B038091A30113
:10C5F000813011F480E801C086958093A301809179
:10C60000A30190917C06892311F0439A01C04398BD
:10C61000429B05C080915A02886080935A02439BD6
:10C6200006C080915A02806180935A0208958091D9
:10C630005A028F7E80935A0208950F931F93CF93CF
:10C64000DF93482FEB0180919402E42FFF27843B76
:10C65000D8F08F010E0F1F1FF801E350F84F8081B3
:10C6600091819B01281B390BC90163E070E00E9496
:10C670008970CB01880F991F860F971F0D5B174F8D
:10C68000F8019183808306C0EE0FFF1FED5BF74F2B
:10C6900011821082E42FFF27EE0FFF1FE350F84FA7
:10C6A000D183C083DF91CF911F910F9108954FB730
:10C6B00024E130E0F8948091C9008F778093C9001D
:10C6C0008091C9008F7B8093C9008091C9008F7DC4
:10C6D0008093C900832F99278093CD002093CC00AD
:10C6E0008091C80082608093C80080E18093C90077
:10C6F0008091CA008F778093CA008091CA008F7B97
:10C700008093CA008091CA008F7D8093CA00809177
:10C71000CA008F7E8093CA008091CA00877F809371
:10C72000CA008091C9008B7F8093C9008091CA00A4
:10C7300084608093CA008091CA0082608093CA009E
:10C740008091C80087FF03C08091CE00F9CF80910F
:10C75000C90080688093C9004FBF0895EF92FF928F
:10C760000F931F93CF93DF93482F00E010E0809149
:10C77000A501813061F41092A50184E480935903EE
:10C7800010925B0310925A0310925C0303C28091D3
:10C790005903882319F421E030E001C098019091F9
:10C7A0005A03992371F4232B11F081E010C084E423
:10C7B0008093590390935B0390935A0390935C0387
:10C7C000D2C1913069F4232B09F0C3C182E0809378
:10C7D0005A0380915B038F5F80935B0383E0C1C149
:10C7E0009230D1F4232B09F0B4C183E08093590334
:10C7F00040935C0390915B03923039F410925D0397
:10C8000047FF03C081E080935D0383E080935A0378
:10C810009F5F90935B03A7C1933009F09AC1232BCC
:10C8200009F097C19093590382E080935A03809155
:10C830005B038F5F80935B0320915C03822F9927BA
:10C84000782F6627842F9927682B792B809154069F
:10C85000813051F47370CB018050924063E070E0FE
:10C860000E948970EB0119C0823069F47770CB01A6
:10C870008050944066E070E00E948970EB0126953C
:10C88000269526950CC0EB01D370C856D140CE0139
:10C89000D7FD0196EC01D595C79526952695022FD3
:10C8A00011270F7010700F5F1F4F0D30110508F02A
:10C8B00049C10230110519F404E010E005C004304C
:10C8C000110511F402E010E0D801A00FB11FFD0125
:10C8D000E350F84F808191819E01281B390BC901DB
:10C8E00037FF03C0909581959F4F069704F5E0911F
:10C8F0009706EE2351F0FF27EE0FFF1FE350F84F8E
:10C90000808191818436910594F480919402883CD1
:10C9100030F480919402865F8093940208C088EC82
:10C920008093940280916F008F7D80936F00A3505D
:10C93000B84F8D919C91BC01660F771F680F791FCE
:10C940006C0F7D1F77FF02C06D5F7F4F7B01F594F9
:10C95000E794F594E794CE0101968E159F0524F493
:10C960000894E108F10808C0CE010197E816F9061D
:10C970001CF40894E11CF11C0630110509F0CEC02E
:10C98000C536D1050CF4A5C090915803E92FFF27B7
:10C99000E959F64FE081ED3729F4809157038095EE
:10C9A00080935703963061F480915703882311F0E8
:10C9B000E338B9F0882309F088C0ED3791F085C0DD
:10C9C000993009F082C080915703882329F480911F
:10C9D0007009833831F079C0809170098D3709F082
:10C9E00074C0809168098D3739F480916909833862
:10C9F00099F463E87FEF0DC0833871F48091690981
:10CA0000833819F460E070E004C08D3729F46DE7D5
:10CA100070E085E00E941D6380916A09992787FD77
:10CA20009095BC0186E00E941D6380916B09992757
:10CA300087FD9095BC018BE00E941D6380916C097D
:10CA4000992787FD9095BC018CE00E941D63809121
:10CA500058038930D1F580916E098D3749F4809162
:10CA60000D0890910E080596BC0188E00E941D6398
:10CA700080916F098D3749F480910D0890910E08CF
:10CA80000597BC0188E00E941D6380910D0890917C
:10CA90000E0883589F4F1CF483E89FEF09C08091D4
:10CAA0000D0890910E088E37910534F08DE790E0D7
:10CAB00090930E0880930D0880916D09992787FD4A
:10CAC0009095BC018AE00E941D6310925803109259
:10CAD0005703CA30D1055CF4809158038F5F80936F
:10CAE0005803E82FFF27E959F64F83E880838091A8
:10CAF00058038A3011F4109258038FEFCC39D807BD
:10CB00006CF480915803E82FFF27E959F64F8DE721
:10CB100080838091570380958093570305301105DA
:10CB200018F4B701802F0BC00530110519F4BE01B0
:10CB300087E005C007301105B1F4BE0189E00E940D
:10CB40001D6311C00231110570F081E08093A501D1
:10CB50000AC081E08093A50110925B0310925D03EF
:10CB600084E48093590380915B03803198F0809135
:10CB70005D03882331F48091A501882311F480930B
:10CB80003F0110925B0310925D0310925A0384E4FC
:10CB900080935903E6E0CDB7DEB70C940171CF93D3
:10CBA000EAE5F0E0E81BF90BF7FF05C0CFEFF095E1
:10CBB000E195FF4F01C0C1E028E631E0CF01B901A6
:10CBC0000E948970FC018B35910554F08B55904083
:10CBD0008A35910538F484EB90E08E1B9F0BFC01A5
:10CBE00041E00DC0CF01855B90408A35910518F476
:10CBF000E45BF04003C02E1B3F0BF9014FEFEE0F3B
:10CC0000FF1FE356F84F259134918C2F992787FD0C
:10CC10009095289FB001299F700D389F700D1124A9
:10CC2000842F992787FD9095689FA001699F500DDB
:10CC3000789F500D1124CA01CF9108950895089549
:10CC4000089508950895089508950895089580E039
:10CC500090E008951092730910927209109277096A
:10CC60001092760910927509109274091092780941
:10CC700082E390E00E94B41590935F0380935E037B
:10CC800008959927FC0124E0EE0FFF1F2A95E1F794
:10CC9000E81BF90BE85BF84F95819F3F19F480E0A2
:10CCA00090E00895993C18F4892F99270895808180
:10CCB00082FF07C08AE0989FC001112488509740E6
:10CCC0000895892F99270895A0E0B0E0EAE6F6E6F6
:10CCD0000C94E27080915E0390915F030E94BD15F9
:10CCE000882309F4D5C080915E0390915F03C296BA
:10CCF00090935F0380935E03C0E0D0E07E01BB248D
:10CD00007FEFC72E809178098E3F21F480915902E0
:10CD1000816005C08F3F29F4809159028E7F8093F6
:10CD20005902DD2408E417E0F801838187FF1AC067
:10CD3000B3948581893C30F08D2D0E944166C80FE7
:10CD4000D91F02C0C80FD11DF8018181E80EF11C66
:10CD50008681C81610F0C82E05C0809159028E7FBA
:10CD600080935902D394015F1F4FFBE0FD15E0F65D
:10CD7000C0927809EF2841F5209164033091650352
:10CD80004091660350916703BB27A52F942F832FF3
:10CD90009093630380936203AA27BB27281B390B58
:10CDA0004A0B5B0BCE01AA27BB27280F391F4A1F4E
:10CDB0005B1F209364033093650340936603509395
:10CDC0006703C5E0D0E013C08091620390916303D4
:10CDD0008C179D0718F4C81BD90B02C0C0E0D0E027
:10CDE0008B2D9927880F991FC80FD91F2596D0938F
:10CDF0007309C0937209CF3FD10578F48091230164
:10CE0000909124018C9F90018D9F300D9C9F300D3F
:10CE10001124C90164E670E013C0CE019695879590
:10CE2000969587952091230130912401289FA00198
:10CE3000299F500D389F500D1124CA0169E170E0FF
:10CE40000E947570709375096093740980916003F6
:10CE5000909161038C0F9D1F9093610380936003F9
:10CE600052E0813D9507A0F0209176093091770935
:10CE70002F5F3F4F805D9240E2E0813D9E07C0F70B
:10CE80009093610380936003309377092093760930
:10CE9000E9E0CDB7DEB70C94FE7008950895002444
:10CEA00022273327442751E0BB27EE27FF27A0E1A5
:10CEB000660F771F881F991F001C221F331F441FF6
:10CEC000660F771F881F991F001C221F331F441FE6
:10CED0002AF4050E2B1F3E1F4F1F04C0051A2B0BF3
:10CEE0003E0B4F0B550FBB1FEE1F587F556047FD84
:10CEF0005250AA95E9F6E695B7955795E695B795F8
:10CF00005795852F9B2F08952227332741E05527DA
:10CF100068E0880F991F221F331F880F991F221F57
:10CF2000331F1AF4240F351F02C0241B350B440F86
:10CF3000551F487F456037FD42506A9551F7569519
:10CF4000479556954795842F0895AA2797FF04C0C3
:10CF5000809590958A1F9A1F77FF04C06095709501
:10CF60006A1F7A1F669F9001779FA001679F300D0F
:10CF7000411D5A1F300D411D5A1F889FF001999F76
:10CF80002E0F3F1F401D511D899F300D411D5A1FFF
:10CF9000300D411D5A1FCA01B901112480CF909153
:10CFA0007203933240F4E92FFF27ED57F64F808349
:10CFB0009F5F909372030895833218F48D5F80937E
:10CFC0007203089590E2E6E8F9E08FE191938150D1
:10CFD00087FFFCCF0895CF93CFB723E031E0F894DB
:10CFE0008091C9008F778093C9008091C9008F7BA1
:10CFF0008093C9008091C9008F7D8093C900832FE1
:10D0000099278093CD002093CC008091C800826046
:10D010008093C80088E18093C9008091CA008F770F
:10D020008093CA008091CA008F7B8093CA00809150
:10D03000CA0080628093CA008091CA008061809398
:10D04000CA008091CA0088608093CA008091C9009C
:10D0500084608093C9008091CA0084608093CA0074
:10D060008091CA0082608093CA008091C80087FFC7
:10D0700003C08091CE00F9CF8091C9008068809371
:10D08000C9008091C90080648093C9000E94E26752
:10D09000CFBFCF910895282F99278F709070892B3B
:10D0A00031F4209580917103822B80937103089550
:10D0B0008091AC01882309F44BC080915B0285FD0F
:10D0C00004C08091B001882381F082E980938309B4
:10D0D00083E2809384098091B001882309F485E577
:10D0E000809385091092B00102C0809383098091DA
:10D0F000AD018F3071F4809171030E9427668823FF
:10D1000041F081E9809383098093840981E38093CE
:10D1100085091092AC018091C80085FFFCCF8091F9
:10D12000C9008F7E8093C9008091C9008E7F809353
:10D13000C90080918309882311F48EEF01C08EE726
:10D140008093CE00809171038093AD0110927103A2
:10D1500008951F920F920FB60F9211248F939F93F1
:10D16000EF93FF939091AC01992309F040C0809117
:10D170007303882361F480918309882311F483E089
:10D1800003C0813999F481E0809373030FC0833029
:10D1900099F480918309882349F0909383098091C1
:10D1A000C9008E7F8093C9008EEF1EC08091C90098
:10D1B00081608093C9000EC0833261F48091C90000
:10D1C0008E7F8093C9008FEF8093CE0081E08093A3
:10D1D000AC0118C080917303E82FFF27ED57F64F7D
:10D1E0008F5F8093730380818093CE000BC0109279
:10D1F000730310927403109275038091C9008061CB
:10D200008093C900FF91EF919F918F910F900FBE76
:10D210000F901F901895EF92FF920F931F93CF934B
:10D22000DF937C018B01EA01452B39F0F8018191F4
:10D230008F01F70109952197C9F7E6E0CDB7DEB771
:10D240000C940171EF92FF920F931F93CF93DF9392
:10D250007C018B01EA01452B41F0F8010F5F1F4F64
:10D260008491F70109952197C1F7E6E0CDB7DEB7C4
:10D270000C9401710F931F93CF938C01C62F161638
:10D2800034F480E2F8010995C1501C16D4F3CF9113
:10D290001F910F9108950F931F93CF938C01C62F69
:10D2A000161634F480E3F8010995C1501C16D4F326
:10D2B000CF911F910F910895A5E3B0E0E2E6F9E662
:10D2C0000C94D9702E96EEADFFAD2E97882499243C
:10D2D000540180917003882321F42C961FAE1EAE5A
:10D2E0002C97AEE44A2E512C4C0E5D1E6F01B601F8
:10D2F00005C0153239F00894C11CD11CF6011491F7
:10D300001123B9F7A601461B570B31F02C968EADB1
:10D310009FAD2C970E942269112309F46AC20894D8
:10D32000C11CD11CFF24FDA6FCA67FEFE72EF9A6A9
:10D33000F6010894C11CD11C1491153721F0812FDE
:10D3400080628837B1F4F0FE0AC0F20124E030E0D8
:10D35000420E531E80809180A280B3800AC0F201E9
:10D3600042E050E0440E551E808191814C01AA2478
:10D37000BB24103221F489A58823D1F61DC01332B5
:10D3800019F458E0F52AD4CF1A3211F01D3291F475
:10D390001A3259F4F20182E090E0480E591EE08101
:10D3A000ECA7EE232CF6E195ECA790E1F92AAFED7E
:10D3B000FA22BECF1B3211F419A7BACF1E32C1F523
:10D3C000F6010894C11CD11C14911A3279F4F201AF
:10D3D00022E030E0420E531E408151813FEF4F3F2B
:10D3E000530714F44FEF5FEFE42EA2CF40E050E07C
:10D3F000812F80538A30A0F4CA0163E0880F991FFF
:10D400006A95E1F7840F951F480F591F410F511D71
:10D4100040535040F6010894C11CD11C1491E8CF30
:10D420008FEF4F3F580714F44FEF5FEFE42E85CF97
:10D43000103329F4F4FC7CCF90E2F92A79CF812FC4
:10D4400081538930D8F440E050E0CA0133E0880FBE
:10D45000991F3A95E1F7840F951F480F591F410F07
:10D46000511D40535040F6010894C11CD11C149129
:10D47000812F80538A3048F34CA75FCF183619F4B8
:10D48000A4E0FA2A55CF1C3619F4B1E0FB2A50CF9C
:10D49000133661F43E010894611C711CF20122E014
:10D4A00030E0420E531E808189833CC1143421F048
:10D4B000143611F0193651F5143411F431E0F32A11
:10D4C000F0FE0AC0F20144E050E0440E551E808098
:10D4D0009180A280B3800CC0F20182E090E0480EFF
:10D4E000591E808191814C01AA2497FCA094BA2CEA
:10D4F000B7FE0AC0B094A09490948094811C911CB3
:10D50000A11CB11C8DE289A70AE06FC01F3411F085
:10D510001F3631F41F3411F491E0F92A08E064C099
:10D52000103779F4F201A2E0B0E04A0E5B1E808170
:10D5300091814C01AA24BB2400E1B0E4FB2A18E746
:10D5400053C01337C1F5F20122E030E0420E531E02
:10D55000608071806114710489F43E010894611C3B
:10D56000711C88E289838EE6F301818385E78B83D2
:10D570008CE68C838D8389E28E831F82E7FC13C047
:10D580008E2D992787FD9095AC0160E070E0C30176
:10D590000E94A66E009729F0382E3618E3140CF07E
:10D5A000C3C03E2CC1C0F30101900020E9F73197C0
:10D5B0003E2E3618B9C0153511F0153731F4153532
:10D5C00011F4F1E0FF2A0AE00FC0183519F01837FE
:10D5D00009F0A0C000E1F3FE07C081149104A1048A
:10D5E000B10411F020E4F22A19A6EDA6E7FC02C06E
:10D5F0003FEDF32229E2622E712C6C0E7D1E811408
:10D600009104A104B10421F44DA5442309F47BC085
:10D61000802F9927AA27BB278EA79FA7A8ABB9ABB6
:10D62000202E332490E0891690E0990691E0A90617
:10D6300090E0B90648F0C501B4012EA53FA548A960
:10D6400059A90E949C7017C0AFEF8A169104A104DB
:10D65000B10449F040F0C401B1010E9475709B0112
:10D660004427552708C0882D602F0E946970282FF5
:10D670003327442755272AAB3BAB4CAB5DAB0A3075
:10D6800059F48AA9880F880F880F9AA9990F890FD2
:10D69000382D381B832F10C0003139F48AA98295A8
:10D6A000807F482D481B842F07C08AA9880F880FC8
:10D6B000880F582D581B852F90E02EA53FA548A90F
:10D6C00059A982169306A406B50608F091E08AA827
:10D6D0009BA8ACA8BDA88A3010F4805D04C0895A0C
:10D6E000183509F48F7DD3018E933D01992309F0FC
:10D6F00099CF083041F4F3FE06C0803321F080E377
:10D70000FD0182933F01CE010196382E3618F8E2D2
:10D710003F0E0BC0112309F46CC03E010894611C3C
:10D72000711C198391E0392E19A6032D2DA42318FD
:10D7300027FC222489A5882311F00F5F02C0F6FC84
:10D740000E5F020DEF2CFF24C70180739070892BB0
:10D7500049F48CA5801B682F2C968EAD9FAD2C971D
:10D760000E943A6989A5882331F041E050E0BE016A
:10D77000675D7F4F0AC0E6FE0EC080E38AA71BA745
:10D7800042E050E0BE01665D7F4F2C968EAD9FADAE
:10D790002C970E940B69C70180739070809749F4A1
:10D7A0008CA5801B682F2C968EAD9FAD2C970E9468
:10D7B0004B69622D2C968EAD9FAD2C970E944B69C4
:10D7C000832D992787FD9095AC01B3012C968EADE2
:10D7D0009FAD2C970E940B69E4FE89CD2CA5201BE0
:10D7E0002CA7622F2C968EAD9FAD2C970E943A6984
:10D7F0007ECDE2E1CB5C0C94F5702FB740E0F8945D
:10D80000E0E0F0E081E2809357009491E2E0F0E004
:10D81000809357003491E4E0F0E0809357008491C6
:10D820002FBF9E3199F4363941F4893011F441E02B
:10D830000DC08A3059F442E009C0373939F48630D6
:10D8400011F443E003C0853009F444E0842F9927A4
:10D8500008959FB7F8948091C900877F8093C9008D
:10D860008091C9008F7E8093C9008091C9008F7715
:10D870008093C9008091C9008F7B8093C9008091FB
:10D88000C9008F7D8093C9009FBF08951F93CF93D8
:10D89000DF93182F80917003882309F4A0C0809132
:10D8A000AB01181709F49BC080916F03882321F402
:10D8B0000E94FD6B80936F0382ED91E090933E0197
:10D8C00080933D0182EF98E09F938F93CEEDD1E15D
:10D8D000DF93CF93E0918903F0918A0309950F902C
:10D8E0000F900F900F90812F992784309105F1F0C0
:10D8F000853091051CF4892B51F00CC086309105C0
:10D90000D9F086309105ACF0089741F12AC08EEE2F
:10D9100098E002C085EE98E09F938F93DF93CF93BA
:10D92000E0918903F0918A03099527C080EE98E081
:10D93000F3CF88ED98E0F0CF80ED98E09F938F9340
:10D94000DF93CF93E0918903F0918A03099588EDE5
:10D9500091E090933E0180933D010FC08BEC98E0E5
:10D96000DBCF8FEF98E09F938F93DF93CF93E0917E
:10D970008903F0918A03099510E00F900F900F90A2
:10D980000F9080916F03843011F0823099F40E94DF
:10D99000296C812F8150833018F40E9457631DC079
:10D9A000143019F40E94EB6718C01830B1F40E94CB
:10D9B0004D6713C0112389F085E199E09F938F9300
:10D9C0008EED91E19F938F93E0918903F0918A030B
:10D9D00009950F900F900F900F901093AB01DF916E
:10D9E000CF911F9108950F931F93082F81E080938B
:10D9F00070034091AA01EBE7F8E020E030E05FE43B
:10DA0000849199272F5F3F4F829FB001839F700DB4
:10DA1000929F700D112446275150319657FFF0CF39
:10DA20004093AA01E3E5F8E020E030E057E284917A
:10DA300099272F5F3F4F829FB001839F700D929F68
:10DA4000700D112446275150319657FFF0CF409367
:10DA5000AA0180916F03882321F40E94FD6B8093BB
:10DA60006F038CE599E690938A03809389038091F4
:10DA7000AA01833459F088E190E029E20FB6F894C6
:10DA8000A895809360000FBE20936000073091F04E
:10DA900080E399E09F938F938EED91E19F938F9315
:10DAA000E0918903F0918A0309950F900F900F90F0
:10DAB0000F90EECF0E940A0581E690E09F938F932E
:10DAC00088E090E09F938F9382E090E09F938F9304
:10DAD000809103016AE00E946970892F99279F93C2
:10DAE0008F93809103010E94697099279F938F9370
:10DAF0008DE499E09F938F930EED11E11F930F93A7
:10DB0000E0918903F0918A0309958BE798E09F9350
:10DB10008F931F930F93E0918903F0918A030995E6
:10DB200083E598E09F938F931F930F93E091890370
:10DB3000F0918A0309950E940A0583EC8093810085
:10DB400080916F00806280936F008DB79EB746967C
:10DB50008DBF1F910F910895809195068D3338F0F8
:10DB60008091ED0887FD03C08CE38093950680913A
:10DB70004306882331F08055853618F08FE780936F
:10DB80004306089580917003882309F482C0809130
:10DB90008603815080938603882309F069C089E158
:10DBA00080938603809195068E3338F08091ED083E
:10DBB00087FD03C08DE3809395068091940282389F
:10DBC000A0F580915C0290915D02805D974020F00D
:10DBD00080917809843620F410928803109287038C
:10DBE000209187033091880321153105B1F1C901D6
:10DBF00001979093880380938703419798F18091D0
:10DC0000ED0884FF2FC080915A02846080935A02ED
:10DC10008091FB0887FF26C080916E03882311F155
:10DC200030938803209387031DC080919402853B25
:10DC3000C8F09091950684E1989FC0011124409608
:10DC400020918703309188032817390730F42F5F1C
:10DC50003F4F309388032093870380915A028B7F34
:10DC600080935A028091AA01833411F010927003BC
:10DC70008091AE01882321F081508093AE010895F8
:10DC80008BE48093AE018091AB01843011F40E944B
:10DC9000586808951F920F920FB60F9211242F9378
:10DCA0003F934F935F936F937F938F939F93AF9324
:10DCB000BF93EF93FF932091CE008091BC01882306
:10DCC000B1F02093C6008091BC01823029F52F3F2E
:10DCD00019F58FEF94E3ACE0B0E0C297A109B10968
:10DCE000B7FFFBCF8091CC038093CE0015C09091FD
:10DCF000AB01892F8150833020F4822F0E94AE63C4
:10DD00000BC0943021F4822F0E944B6805C09830DC
:10DD100019F4822F0E944E67FF91EF91BF91AF914E
:10DD20009F918F917F916F915F914F913F912F9133
:10DD30000F900FBE0F901F901895FB01DC0102C0E1
:10DD400005900D9241505040D8F70895FC01415084
:10DD5000504030F001900616D1F73197CF01089569
:10DD6000882799270895A0E0B0E0E9EBFEE60C943F
:10DD7000E1706C017B01EA01590121978FEFCF3FE0
:10DD8000D80789F086010894C11CD11CC7010894EA
:10DD9000E11CF11CF5010995F80180832197FFEF43
:10DDA000CF3FDF0779F7EAE0CDB7DEB70C94FD701F
:10DDB000CF92DF92EF92FF920F931F937C016B0142
:10DDC000FB010995082FC7010196F6010995182F47
:10DDD000C8011F910F91FF90EF90DF90CF900895B1
:10DDE000A0E0B0E0E6EFFEE60C94E3708C017B016E
:10DDF000EA01690121978FEFCF3FD80771F0F70152
:10DE000021917F01C8010F5F1F4F622FF601099515
:10DE10002197FFEFCF3FDF0791F7E8E0CDB7DEB7FF
:10DE20000C94FF70CF92DF92EF92FF920F931F93AB
:10DE30006C018B017A01FA010995812F9927682FCE
:10DE4000C6010196F70109951F910F91FF90EF9080
:10DE5000DF90CF9008955058BB27AA270ED0E0C07E
:10DE6000D1D030F0D6D020F031F49F3F11F41EF421
:10DE7000C6C00EF4E095E7FBBCC0E92FE2D080F30A
:10DE8000BA17620773078407950718F071F49EF5B7
:10DE9000FAC00EF4E0950B2EBA2FA02D0B01B9019C
:10DEA00090010C01CA01A0011124FF27591B99F010
:10DEB000593F50F4503E68F11A16F040A22F232F1C
:10DEC000342F4427585FF3CF469537952795A7956C
:10DED000F0405395C9F77EF41F16BA0B620B730B13
:10DEE000840BBAF09150A1F0FF0FBB1F661F771F84
:10DEF000881FC2F70EC0BA0F621F731F841F48F439
:10DF0000879577956795B795F7959E3F08F0B3CFBE
:10DF10009395880F08F09927EE0F979587950895A8
:10DF200098D088F09F5790F0B92F9927B751A0F05B
:10DF3000D1F0660F771F881F991F1AF0BA95C9F79D
:10DF400012C0B13081F09FD0B1E008959CC0672F1E
:10DF5000782F8827B85F39F0B93FCCF3869577954D
:10DF60006795B395D9F73EF4909580957095619536
:10DF70007F4F8F4F9F4F0895E89409C097FB3EF461
:10DF800090958095709561957F4F8F4F9F4F992306
:10DF9000A9F0F92F96E9BB279395F6958795779584
:10DFA0006795B795F111F8CFFAF4BB0F11F460FF44
:10DFB0001BC06F5F7F4F8F4F9F4F16C0882311F09C
:10DFC00096E911C0772321F09EE8872F762F05C0B0
:10DFD000662371F096E8862F70E060E02AF09A954B
:10DFE000660F771F881FDAF7880F9695879597F940
:10DFF000089597F99F6780E870E060E008959FEFCB
:10E0000080EC089500240A941616170618060906CF
:10E01000089500240A94121613061406050608959E
:10E02000092E0394000C11F4882352F0BB0F40F426
:10E03000BF2B11F460FF04C06F5F7F4F8F4F9F4F66
:10E04000089557FD9058440F551F59F05F3F71F0E8
:10E050004795880F97FB991F61F09F3F79F087954F
:10E060000895121613061406551FF2CF4695F1DFD8
:10E0700008C0161617061806991FF1CF8695710568
:10E08000610508940895E894BB2766277727CB019C
:10E0900097F90895629FD001739FF001829FE00D70
:10E0A000F11D649FE00DF11D929FF00D839FF00D17
:10E0B000749FF00D659FF00D9927729FB00DE11DC3
:10E0C000F91F639FB00DE11DF91FBD01CF011124A0
:10E0D0000895991B79E004C0991F961708F0961BC4
:10E0E000881F7A95C9F780950895AA1BBB1B51E13B
:10E0F00007C0AA1FBB1FA617B70710F0A61BB70BB8
:10E10000881F991F5A95A9F780959095BC01CD015C
:10E11000089597FB092E07260AD077FD04D0E5DF86
:10E1200006D000201AF4709561957F4F0895F6F798
:10E13000909581959F4F0895A1E21A2EAA1BBB1BB3
:10E14000FD010DC0AA1FBB1FEE1FFF1FA217B307C3
:10E15000E407F50720F0A21BB30BE40BF50B661FD9
:10E16000771F881F991F1A9469F76095709580959D
:10E1700090959B01AC01BD01CF01089597FB092E3D
:10E1800005260ED057FD04D0D7DF0AD0001C38F486
:10E1900050954095309521953F4F4F4F5F4F0895D3
:10E1A000F6F790958095709561957F4F8F4F9F4FB3
:10E1B00008952F923F924F925F926F927F928F922B
:10E1C0009F92AF92BF92CF92DF92EF92FF920F9306
:10E1D0001F93CF93DF93CDB7DEB7CA1BDB0B0FB610
:10E1E000F894DEBF0FBECDBF09942A8839884888CD
:10E1F0005F846E847D848C849B84AA84B984C88463
:10E20000DF80EE80FD800C811B81AA81B981CE0F59
:10E21000D11D0FB6F894DEBF0FBECDBFED0108953E
:0EE22000EE0FFF1F0590F491E02D0994FFCF43
:10E22E0004035E0A010164FF010020FFFFC01FC04E
:10E23E001F0101F40101737373FF03007D0000C41D
:10E24E0009C4099600134167696C650051756164D4
:10E25E00726F0000000000000064000C09D2010182
:10E26E00200B050000ECFF00020406070808080753
:10E27E0006040200FEFCFAF9F8F8F8F9FAFCFE00C2
:10E28E000204060708086440415A46553264646425
:10E29E000A02969696960864403A1030380132FF7C
:10E2AE00037F0090D0030090D0030032002064FF63
:10E2BE00FF64200B0A130B0E100B0A0C0F0B111020
:10E2CE00FA2068010101F7FFFCFF70FF010F6400E7
:00000001FF
